:020000040000FA
:0408000090EF07F07E
:020808003BD0E3
:0808180087D0E26BE36BE46B97
:10082000E56BF86A080EF76E000EF66A0900F550DF
:10083000E527E86AE423E323E223FF0EF762F6D715
:10084000FA0EF662F3D7E51FE41FE31FE21FE52B64
:0A085000E86AE423E323E223FFD764
:10088000026ED8CF03F0D9CF05F0DACF04F0E1CF74
:1008900007F0E2CF06F0E9CF09F0EACF08F09EBA00
:1008A0000BD0F2B201D030D0F292A081A0A32CD014
:1008B00091C092F0916B28D0AECFC9F03D8E0A0E58
:1008C000C95D22E00D0EC9630BD06B511DE022EE15
:1008D00000F0D926C9C0DFFF6B6BA6EC5DF014D029
:1008E00022EE00F06B51D926C9C0DFFF6B2B3E0E04
:1008F000C96302D03F8008D03FA006D0200EC96354
:1009000003D03F823F906B6B05C0D9FF04C0DAFF74
:1009100007C0E1FF06C0E2FF09C0E9FF08C0EAFF27
:10092000025003C0D8FF1000006ED8CF01F0E9CF0D
:100930000AF0EACF0BF0A4AA18D0A49A1AEE00F09D
:100940006ECFF7F00A0EF75DD8B4AED2F851E126BB
:10095000F7C0E7FF0D0EF76306D0E12AE76AF86BF0
:100960005EEC67F0A1D2F82B9FD2F0A203D0F092F8
:1009700035809AD2F2A498D2F294AA2F1ED00A0EF1
:10098000AA6FA0B3912B39B002D0809816D083AE55
:10099000808883BE809883AE678983BE67996739F4
:1009A0006719010BE8A009D067A904D067816785A2
:1009B000679303D0679167956783AB67AB07B167B0
:1009C000B107AD5305E0AE0703E1640EAE6FAD07AE
:1009D000AF5305E0B00703E1640EB06FAF07B25349
:1009E00005E0B40703E10A0EB46FB207B35305E0A4
:1009F000B50703E1640EB56FB307B65305E0B7075B
:100A000003E10A0EB76FB607B85305E0B90703E173
:100A1000640EB96FB80760EC07F036B462D036B236
:100A200024D036B00DD035A06FD03590C26BC36BDB
:100A3000366A376A36800A0EB46F050EB26F64D01C
:100A4000B26702D0366A60D035A05ED0359036905D
:100A50003682C26BC46BC36B0A0EB46F140EB26FD6
:100A6000640EB56F2D0EB36F4FD0C22B35B017D0BB
:100A7000B2674AD036923684369636A80CD0358284
:100A8000358635843698640EB56F2D0EB36FC46B02
:100A9000C26BC36B39D035923594359635D03590CD
:100AA0000A0EB46F140EB26F36B605D0C2C0C3F0D2
:100AB000C26B367629D03676C251C327430EC36146
:100AC0000BD00F0EC36508D0C36BC26BC42B050ED1
:100AD000C4651AD0368818D03696C46BC26BC36B07
:100AE00013D0B36704D0366AC00E35160DD035A0CA
:100AF0000BD03590C46BC26BC36B3682369436967E
:100B00000A0EB46F1E0EB26F3AA6E3EF05F03AB0CC
:100B1000BDEF05F03AB2A1EF05F06C2FE3EF05F061
:100B2000140E6C6F80746D2FE3EF05F01D50D8B478
:100B30003A841BC06DF03A828086809480828090D7
:100B400042D06C2FE3EF05F0140E6C6F6D2FE3EFC6
:100B500005F01C5008E06D6F3A923A8080868094D0
:100B60008092808030D01AC06DF03A923A90C52BB6
:100B7000808680948092808026D03AB2D2EF05F0B1
:100B80006C2FE3EF05F0140E6C6F80746D2FE3EFA4
:100B900005F01DC06DF03A823A8480868094808290
:100BA000809011D06C2FE3EF05F0140E6C6F6D2F59
:100BB000E3EF05F01AC06DF03A923A90C52B8086AB
:100BC000809480928080BFAF6FD1010EC06308D047
:100BD000000EC16304D0B5EC61F0C12B65D164D1C6
:100BE000020EC06345D0000EC1630BD0C12BE0C91B
:100BF000E8FFFF0BD8B458D15CEC07F0C0EC61F013
:100C000053D1010EC1630DD0B6674ED1C12BE1C9DE
:100C1000E8FFFF0BD8B448D15CEC07F0F5EC61F0CD
:100C200043D1020EC1630DD0B6673ED1C12BE2C9DC
:100C3000E8FFFF0BD8B438D15CEC07F0C0EC61F0F2
:100C400033D1030EC1630DD0B6672ED1C12BE3C9DA
:100C5000E8FFFF0BD8B428D15CEC07F0F5EC61F0AD
:100C600023D1040EC16320D1B6671ED1C16B1CD144
:100C7000030EC06345D0000EC1630BD0C12BE4C985
:100C8000E8FFFF0BD8B410D15CEC07F0CBEC61F0BF
:100C90000BD1010EC1630DD0B66706D1C12BE5C9DA
:100CA000E8FFFF0BD8B400D15CEC07F0F5EC61F085
:100CB000FBD0020EC1630DD0B667F6D0C12BE6C9DA
:100CC000E8FFFF0BD8B4F0D05CEC07F0CBEC61F0A0
:100CD000EBD0030EC1630DD0B667E6D0C12BE7C9D8
:100CE000E8FFFF0BD8B4E0D05CEC07F0F5EC61F066
:100CF000DBD0040EC163D8D0B667D6D0C16BD4D0D8
:100D0000040EC06345D0000EC1630BD0C12BE8C9EF
:100D1000E8FFFF0BD8B4C8D05CEC07F0D6EC61F06C
:100D2000C3D0010EC1630DD0B667BED0C12BE9C9D7
:100D3000E8FFFF0BD8B4B8D05CEC07F0F5EC61F03D
:100D4000B3D0020EC1630DD0B667AED0C12BEAC9D5
:100D5000E8FFFF0BD8B4A8D05CEC07F0D6EC61F04C
:100D6000A3D0030EC1630DD0B6679ED0C12BEBC9D3
:100D7000E8FFFF0BD8B498D05CEC07F0F5EC61F01D
:100D800093D0040EC16390D0B6678ED0C16B8CD067
:100D9000050EC06363D0000EC16307D0C12B0A0EDD
:100DA0005CEC07F0B5EC61F07FD0010EC16309D0B7
:100DB000B6677AD0F5EC61F0C12B0A0E5CEC07F057
:100DC00073D0020EC16309D0B6676ED0B5EC61F086
:100DD000C12B0A0E5CEC07F067D0030EC16309D08B
:100DE000B66762D0F5EC61F0C12B0A0E5CEC07F03F
:100DF0005BD0040EC16309D0B66756D0C12BB5ECE9
:100E000061F00A0E5CEC07F04FD0050EC16309D00B
:100E1000B6674AD0F5EC61F0C12B0A0E5CEC07F026
:100E200043D0060EC16309D0B6673ED0B5EC61F081
:100E3000C12BFA0E5CEC07F037D0070EC16307D068
:100E4000B66732D0C12BF00E5CEC07F02DD0080E47
:100E5000C1632AD0B66728D0C16B26D0060EC06306
:100E600023D0000EC16307D0E1EC61F0C12B0A0E64
:100E70005CEC07F019D0010EC16309D0B66714D03D
:100E8000F5EC61F0C12B0A0E5CEC07F00DD0020E00
:100E9000C1630AD0B66708D0E1EC61F0010EC16F02
:100EA0000A0E5CEC07F000D00AC0E9FF0BC0EAFFB5
:100EB000005001C0D8FF1000B66F0A0EB76F1200C5
:100EC0000001D42BFA0ED46324D0D46BD32B040EA0
:100ED000D3631FD0D36BD52BBA67BA07010EBB5FA4
:100EE000E86ABC5BBB6707D0BC6705D026C0BBF017
:100EF00027C0BCF06481010EBD5FE86ABE5BBD67C0
:100F000007D0BE6705D065C0BDF066C0BEF0648581
:100F100034801200D880EF50E75ED8A0E76C120052
:100F2000C26A0F0EC16E070EB46E806A816A826A51
:100F3000836A846A856A866A000E926E070E936ED3
:100F4000B80E946EA10E956E090E966E000E976EF9
:100F5000140E986E82928290838684888492848410
:100F6000808A8186D66AD76A530ED56ED58E336A4B
:100F7000326A0001D36BD46BD56BF86BA16B996BA4
:100F8000A66BA76B346A646BBF6B356A366A376AC7
:100F9000386A396A3A6A3B6A576A586A596A5A6AB9
:100FA000676B3D6A3F6AA06B6B6B426A8A6B140E7B
:100FB000976F00EE43F0EE6A972FFDD7400E976FC4
:100FC00004EEC0F0EE6A972FFDD7976B0DEE00F0A0
:100FD0001EEE00F0EE68E668972FFCD7120E976FB2
:100FE00001EE8CF011EE9EF0200EEE6EE66E972F65
:100FF000FBD77BEC64F08EEC63F08E6F9DEC63F0BE
:101000008F6FABEC63F08388690EAF6E260EAC6E0B
:10101000920EAB6E080E6F6E260E6C6E920E6B6E9D
:10102000D08EF28AF194F294F288F292F16AF06A28
:10103000F0889F8A9D8A9F989D98A59AA38AA598D3
:10104000A398F28CF28EF28C34EC66F095EC66F09C
:10105000A66BA76B53EC63F08086809480828090AF
:101060008690E30EF76E4E0EF66E20EED6F0F5EC9F
:1010700065F0FF0EF76E4C0EF66E20EEE6F0F5EC26
:1010800065F013EC66F0640EAE6F0A0EAD6FAD67DF
:1010900047EF08F029EC62F071EC34F030A280ECFC
:1010A00034F030B213D039AE09D0F80EF76ECE0E50
:1010B000F66E20EEE6F0F5EC65F008D0F80EF76E6F
:1010C000DE0EF66E20EEE6F0F5EC65F039AC09D0F8
:1010D000F80EF76EAE0EF66E20EED6F0F5EC65F07B
:1010E00008D0F80EF76EBE0EF66E20EED6F0F5ECD8
:1010F00065F013EC66F0640EAE6F140EAD6FAD6765
:10110000FED721EC62F0A5EC62F0A66BA76B53EC66
:1011100063F0A68753EC63F0A78953EC63F0300EBD
:101120002414E86664873994F80EF76EEE0EF66EB6
:1011300020EED6F0F5EC65F0E30EF76EBE0EF66E1F
:1011400020EEE6F0F5EC65F013EC66F08280576A6D
:10115000640EAE6F050EAD6FAD67FED78290640E64
:10116000AE6F140EAD6FAD67FED7050E976F3D9055
:101170003D92DF0EF76EB40EF66E23EE00F0EEEC4D
:1011800065F0DE6ADFEC65F0640EAE6F140EAD6FD5
:101190003DB0E2EF08F0AD67FBD7972FE8D7E40E3C
:1011A000F76E0E0EF66E20EED6F0F5EC65F0E40E5E
:1011B000F76E1E0EF66E20EEE6F0F5EC65F013EC21
:1011C00066F0FFD73D903D92E00EF76E120EF66E80
:1011D00023EE00F0EEEC65F0DE6ADFEC65F0640E05
:1011E000AE6F320EAD6F3DB0FCEF08F03DB2CFEF09
:1011F00008F0AD67F8D7D3D7640EAE6F0A0EAD6FA7
:10120000AD67FED73D903D92E00EF76E2E0EF66E66
:1012100023EE00F0EEEC65F0DE6ADFEC65F0640EC4
:10122000AE6F320EAD6F3DB01CEF09F03DB2CFEFA7
:1012300008F0AD67F8D7B3D7640EAE6F140EAD6F7C
:10124000AD67FED73D903D92E00EF76E460EF66E0E
:1012500023EE00F0EEEC65F0DE6ADFEC65F0640E84
:10126000AE6F320EAD6F3DB03CEF09F03DB2CFEF47
:1012700008F0AD67F8D793D73D903D92E00EF76E3A
:10128000FA0EF66E23EE00F0EEEC65F0DE6ADFECAF
:1012900065F0640EAE6F640EAD6F3DB056EF09F0B1
:1012A0003DB2CFEF08F0AD67F8D779D7640EAE6FD7
:1012B0000A0EAD6FAD67FED73D903D92E00EF76E22
:1012C0009A0EF66E23EE00F0EEEC65F0DE6ADFECCF
:1012D00065F0640EAE6F640EAD6F57B678EF09F02F
:1012E00057B078EF09F03DB03D90AD67F6D757D7CE
:1012F0005796E40EF76EBE0EF66E20EEE6F0F5ECB5
:1013000065F013EC66F03D903D92E00EF76EBE0E78
:10131000F66E23EE00F0EEEC65F0DE6ADFEC65F0D1
:10132000640EAE6F320EAD6F3DB09FEF09F03DB26F
:101330009CEF09F0AD67F8D73D92CFEF08F03D90F4
:101340003D92DF0EF76ECA0EF66E23EE00F0EEEC65
:1013500065F0DE6ADFEC65F0640EAE6F320EAD6FE5
:101360003DB0BBEF09F03DB2B8EF09F0AD67F8D77B
:101370003D92CFEF08F0388C3D903D92E00EF76E35
:10138000600EF66E23EE00F0EEEC65F0DE6ADFEC48
:1013900065F0640EAE6F320EAD6F3DB0D7EF09F061
:1013A0003DB2D5EF09F0AD67F8D73D92F8D63D9044
:1013B000389C100E976F08EE52F018EE22F0EECF28
:1013C000E6FF972FFCD703EE00F0410EEE6E540EB1
:1013D000EE6E2B0EEE6E570EEE6E4D0EEE6E420E54
:1013E000EE6E530EEE6E3D0EEE6E1FC084F059ECA5
:1013F00061F07FC0EEFF80C0EEFF81C0EEFFEE6ABD
:101400003D6ADFEC65F0640EAE6F320EAD6F3DB03D
:1014100011EF0AF03DB20FEF0AF0AD67F8D73D9239
:10142000BED63D90E50EF76EFE0EF66E20EED6F0BF
:10143000F5EC65F020C084F059EC61F0200EE16F0E
:10144000E46F300E806380C0E1F081C0E2F021C023
:1014500084F059EC61F0300E806380C0E4F081C00C
:10146000E5F01FC0F4F147EC5DF013EC66F0640E9C
:10147000AE6F320EAD6FAD67FED7E30EF76EDE0EC8
:10148000F66E20EED6F0F5EC65F0E30EF76EEE0E9C
:10149000F66E20EEE6F0F5EC65F0310EE96F13EC38
:1014A00066F0060EC06FC16BBF8F399639823886E1
:1014B000349888EC30F0E8661DEF0FF038823D9AE2
:1014C0003D903D92E10EF76E260EF66E23EE00F093
:1014D000EEEC65F0DE6ADFEC65F0640EAE6F320EA6
:1014E000AD6F3DB090EF0AF03DB27BEF0AF0AD6713
:1014F000F8D7CFEF08F03D92E40EF76E2E0EF66EA1
:1015000020EED6F0F5EC65F0E40EF76E3E0EF66ECA
:1015100020EEE6F0F5EC65F013EC66F054EF14F015
:101520003D90640EAE6F040EAD6FAD67FED73D907B
:101530003D92E10EF76E340EF66E23EE00F0EEEC07
:1015400065F0DE6ADFEC65F0640EAE6F320EAD6FF3
:101550003DBAB4EF0AF03DB0B8EF0AF03DB2B6EFD5
:101560000AF0AD67F5D71BD63D9AF2D73D9217D654
:101570003D90E50EF76E4E0EF66E20EED6F0F5ECD1
:1015800065F0E50EF76E5E0EF66E20EEE6F0F5EC19
:1015900065F001EE7CF010EEDEF0080E976FEECFF6
:1015A000E6FF972FFCD7310E39B4320EE96F13ECFA
:1015B00066F0976B57B0E7EF0AF057B80AEF0BF0F9
:1015C00034B002EF0BF03DB000EF0BF0F3D75990C1
:1015D000E40EF76EAE0EF66E20EED6F0F5EC65F08A
:1015E000E40EF76E9E0EF66E20EEE6F0F5EC65F07A
:1015F000310E39B4320EF06F13EC66F03DEF0AF0A5
:101600003D90D8D73490070E9715F56F972B13ECB4
:1016100066F0D0D757983D903D92DF0EF76ED60E0C
:10162000F66E23EE00F0EEEC65F0DE6ADFEC65F0BE
:10163000640EAE6F320EAD6F3DB027EF0BF03DB2D2
:1016400024EF0BF0AD67F8D73D92CFEF08F03D9057
:1016500003EE00F0410EEE6E540EEE6E2B0EEE6EAB
:10166000570EEE6E560EEE6E520EEE6E3D0EEE6E96
:1016700020C084F059EC61F07FC0EEFF80C0EEFF27
:1016800081C0EEFF2C0EEE6E21C084F059EC61F0AB
:101690007FC0EEFF80C0EEFF81C0EEFFEE6A3D6AC4
:1016A000DFEC65F0640EAE6F320EAD6F3DB060EFF3
:1016B0000BF03DB25EEF0BF0AD67F8D73D92A8D3CB
:1016C0003D903D903D92E00EF76E3A0EF66E23EEA1
:1016D00000F0EEEC65F0DE6ADFEC65F0640EAE6FF4
:1016E000320EAD6F3DB07CEF0BF03DB27AEF0BF0F8
:1016F000AD67F8D73D928CD3D5EC3AF0640EAE6F5F
:10170000320EAD6F3DB08CEF0BF03DB28AEF0BF0B7
:10171000AD67F8D73D927CD3B6EC3AF0640EAE6F6D
:10172000320EAD6F3DB09CEF0BF03DB29AEF0BF077
:10173000AD67F8D73D926CD33D9018EE22F0E6CF1E
:101740007FF0E6CF80F0E6CF81F0330E7F6307D0E5
:10175000340E806304D0330E816301D028D0330E61
:101760007F6307D0340E806304D0340E816301D0D0
:101770001ED0340E7F6307D0340E806304D0330E46
:10178000816301D014D0360E7F6307D0350E80639D
:1017900004D0370E816301D00AD0350E7F6307D0A5
:1017A000340E806304D0310E816301D00BD13D90A3
:1017B0003D92E20EF76E6C0EF66E23EE00F0EEEC4C
:1017C00065F0DE6ADFEC65F0640EAE6F320EAD6F71
:1017D0003DB0F2EF0BF03DB2F0EF0BF0AD67F8D794
:1017E0003D9216D33D903D92E20EF76E5E0EF66E80
:1017F00023EE00F0EEEC65F0DE6ADFEC65F0640EDF
:10180000AE6F320EAD6F3DB00DEF0CF03DB20BEF91
:101810000CF0AD67F8D73D92FBD23D903D92E20EC1
:10182000F76E520EF66E23EE00F0EEEC65F0DE6A17
:10183000DFEC65F0640EAE6F320EAD6F3DB028EF99
:101840000CF03DB226EF0CF0AD67F8D73D92E0D238
:101850003D903D903D92E20EF76E120EF66E23EE35
:1018600000F0EEEC65F0DE6ADFEC65F0640EAE6F62
:10187000320EAD6F3DB068EF0DF03DB242EF0CF0AF
:10188000AD67F8D73D92FE0EF76EBC0EF66E20EEF9
:10189000D6F0F5EC65F0FE0EF76ECC0EF66E20EE8F
:1018A000E6F0F5EC65F013EC66F0640EAE6F280E12
:1018B000AD6FAD67FED737D43D903D92E10EF76E28
:1018C000E20EF66E23EE00F0EEEC65F0DE6ADFEC81
:1018D00065F0640EAE6F320EAD6F3DB077EF0CF079
:1018E0003DB275EF0CF0AD67F8D73D9291D23D90C7
:1018F0003D92E10EF76ED40EF66E23EE00F0EEECA4
:1019000065F0DE6ADFEC65F0640EAE6F320EAD6F2F
:101910003DB092EF0CF03DB290EF0CF0AD67F8D710
:101920003D9276D23D903D92E10EF76EC60EF66E78
:1019300023EE00F0EEEC65F0DE6ADFEC65F0640E9D
:10194000AE6F320EAD6F3DB0ADEF0CF03DB2ABEF10
:101950000CF0AD67F8D73D925BD23D903D903D9243
:10196000E10EF76EAC0EF66E23EE00F0EEEC65F0D5
:10197000DE6ADFEC65F0640EAE6F320EAD6F3DB027
:1019800068EF0DF03DB2C7EF0CF0AD67F8D73D92B0
:10199000FE0EF76EBC0EF66E20EED6F0F5EC65F09E
:1019A000FE0EF76ECC0EF66E20EEE6F0F5EC65F06E
:1019B00013EC66F0640EAE6F280EAD6FAD67FED708
:1019C00093EF08F03D903D92E20EF76EB00EF66E8A
:1019D00023EE00F0EEEC65F0DE6ADFEC65F0640EFD
:1019E000AE6F320EAD6F3DB0FDEF0CF03DB2FBEFD0
:1019F0000CF0AD67F8D73D920BD23D903D92E20ED0
:101A0000F76EA20EF66E23EE00F0EEEC65F0DE6AE5
:101A1000DFEC65F0640EAE6F320EAD6F3DB018EFC7
:101A20000DF03DB216EF0DF0AD67F8D73D92F0D155
:101A30003D903D92E20EF76E940EF66E23EE00F0AE
:101A4000EEEC65F0DE6ADFEC65F0640EAE6F320E30
:101A5000AD6F3DB033EF0DF03DB231EF0DF0AD673E
:101A6000F8D73D92D5D13D903D903D92E20EF76E74
:101A70007A0EF66E23EE00F0EEEC65F0DE6ADFEC37
:101A800065F0640EAE6F320EAD6F3DB068EF0DF0D5
:101A90003DB24DEF0DF0AD67F8D73D92FE0EF76EFB
:101AA000BC0EF66E20EED6F0F5EC65F0FE0EF76E8D
:101AB000CC0EF66E20EEE6F0F5EC65F013EC66F079
:101AC000640EAE6F280EAD6FAD67FED793EF08F0D2
:101AD0003D903D92E10EF76EA00EF66E23EE00F003
:101AE000EEEC65F0DE6ADFEC65F0640EAE6F320E90
:101AF000AD6F3DB083EF0DF03DB281EF0DF0AD67FE
:101B0000F8D73D9285D13D903D92E00EF76EA60E3E
:101B1000F66E23EE00F0EEEC65F0DE6ADFEC65F0C9
:101B2000640EAE6F320EAD6F3DB09EEF0DF03DB264
:101B30009CEF0DF0AD67F8D73D926AD13D903D9294
:101B4000E00EF76EE40EF66E23EE00F0EEEC65F0BC
:101B5000DE6ADFEC65F0640EAE6F320EAD6F3DB045
:101B6000B9EF0DF03DB2B7EF0DF0AD67F8D73D928C
:101B70004FD13D903D92E00EF76EEE0EF66E23EEE5
:101B800000F0EEEC65F0DE6ADFEC65F0640EAE6F3F
:101B9000320EAD6F3DB0D4EF0DF03DB2D2EF0DF08F
:101BA000AD67F8D73D9234D13D903D92E10EF76E8E
:101BB000720EF66E23EE00F0EEEC65F0DE6ADFECFE
:101BC00065F0640EAE6F320EAD6F3DB006EF0EF0F5
:101BD0003DB2EDEF0DF0AD67F8D73D92FE0EF76E1A
:101BE000FC0EF66E20EED6F0F5EC65F0FE0EF76E0C
:101BF000FC0EF66E20EED6F0F5EC65F013EC66F018
:101C0000640EAE6F280EAD6FAD67FED73D90F90E36
:101C1000F76EBE0EF66E20EED6F0F5EC65F0F90E1E
:101C2000F76ECE0EF66E20EEE6F0F5EC65F013ECF6
:101C300066F03D903D92E20EF76EBE0EF66E23EE1C
:101C400000F0EEEC65F0DE6ADFEC65F0640EAE6F7E
:101C5000640EAD6F3DB034EF0EF03DB232EF0EF0DA
:101C6000AD67F8D73D92D4D03D903D92E20EF76E2D
:101C7000CA0EF66E23EE00F0EEEC65F0DE6ADFECE5
:101C800065F0640EAE6F640EAD6F3DB04FEF0EF0B9
:101C90003DB24DEF0EF0AD67F8D73D92B9D03D9013
:101CA0003D92E20EF76ED60EF66E23EE00F0EEECED
:101CB00065F0DE6ADFEC65F0640EAE6F640EAD6F4A
:101CC0003DB06AEF0EF03DB268EF0EF0AD67F8D7A9
:101CD0003D929ED03D903D92E20EF76EF40EF66E70
:101CE00023EE00F0EEEC65F0DE6ADFEC65F0640EEA
:101CF000AE6FFA0EAD6F3DB091EF0EF03DB28FEFCB
:101D00000EF0AD67F8D7640EAE6FFA0EAD6F3DB052
:101D100091EF0EF03DB28FEF0EF0AD67F8D73D9228
:101D200077D03EEC5DF03D903D92E00EF76E800E78
:101D3000F66E23EE00F0EEEC65F0DE6ADFEC65F0A7
:101D4000640EAE6F640EAD6F3DB0AEEF0EF03DB2FF
:101D5000ACEF0EF0AD67F8D73D925AD009EE00F027
:101D6000EECF5BF0EECF5CF0EECF5DF0EECF5EF04D
:101D7000EECF00F0EECF00F0EECF00F0EECF00F0AF
:101D8000EECF5FF0EECF60F0EECF61F0EECF62F01D
:101D9000636B640EAE6F050EAD6FAD67FED73D9001
:101DA0003D92DF0EF76EB80EF66E23EE00F0EEEC0D
:101DB00065F0DE6ADFEC65F0640EAE6F320EAD6F7B
:101DC0003DB0EBEF0EF03DB2E8EF0EF0AD67F8D7A7
:101DD0003D92CFEF08F03D903D92E00EF76EFA0E87
:101DE000F66E23EE00F0EEEC65F0DE6ADFEC65F0F7
:101DF000640EAE6F640EAD6F3DB006EF0FF03DB2F6
:101E000004EF0FF0AD67F8D73D9202D03D9015D0AA
:101E1000E60EF76E3E0EF66E20EED6F0F5EC65F0AF
:101E2000E60EF76E4E0EF66E20EEE6F0F5EC65F07F
:101E300013EC66F081B21AEF0FF0040E9A6F9AC09D
:101E4000E5F0576A586A596AAFEC61F0809A358CB0
:101E5000320EAB6FAB67FED782AA41EF0FF0F60EE2
:101E6000F76EDE0EF66E20EED6F0F5EC65F0F60EAF
:101E7000F76EEE0EF66E20EEE6F0F5EC65F0358EC0
:101E800011D0F60EF76EBE0EF66E20EED6F0F5EC23
:101E900065F0F60EF76ECE0EF66E20EEE6F0F5EC7F
:101EA00065F0359E808A359C13EC66F0640EAE6F4B
:101EB000140EAD6FAD67FED7FFEC65F009EC66F070
:101EC000808680948082809000D067936795349A52
:101ED00030B0348A34B893EF08F026C0BBF027C086
:101EE000BCF0A66BA76B53EC63F0A68753EC63F0D2
:101EF000809A358C320EAB6FAB67FED7359E82BAB7
:101F0000358E808A359CD5EC3AF0640EAE6F320E79
:101F1000AD6F3DB092EF0FF03DB291EF0FF0AD67B6
:101F2000F8D73D923D90389E389E576A586A3D6A70
:101F30003E6AF66B120E976F01EE8CF011EE9EF07A
:101F4000200EEE6EE66E972FFBD739A41DD0399682
:101F50003982060EC06FC16BBF8FE70EF76E5E0E43
:101F6000F66E20EED6F0F5EC65F0E70EF76E6E0E2D
:101F7000F66E20EEE6F0F5EC65F013EC66F03886D0
:101F800088EC30F0E8665BD0A66BA76B53EC63F08F
:101F9000AFEC61F038B6BBD264A715D0649724C00B
:101FA0009AF09A3B030E9A17000E9A5DD8B4F6D2B7
:101FB000010E9A5DD8B400D3020E9A5DD8B4A5D3B1
:101FC000CF0E2416EBD2FF0EF76E3C0EF66E20EE0F
:101FD000D6F0F5EC65F0F60EF76E4E0EF66E20EECE
:101FE000E6F0F5EC65F035BE13D000EEEEF0200E15
:101FF0004E0EEE6E6F0EEE6E200EEE6E4C0EEE6E10
:10200000690EEE6E6E0EEE6E650EEE6E200EEE6ECC
:1020100038B2348238B2388038B20FD0389000EEFF
:10202000E6F04E0EEE6E6F0EEE6E200EEE6E470E6A
:10203000EE6E530EEE6E4D0EEE6E13EC66F034BA8D
:102040006CEF10F067B585EF12F067B383EF12F015
:1020500081A261EF14F05AB02FEF12F05AB232EFB2
:1020600012F05AB432EF12F05AB632EF12F05AB8F8
:102070002FEF12F05ABA32EF12F035B241EF18F0EA
:1020800038B462EF1EF03BB653EF26F038BA22EFB9
:1020900029F057B046EF12F057B25CEF12F059B08A
:1020A0007BEF12F059B280EF12F034B036EF14F03B
:1020B0006BA203D06B9800006B8824C081F0300EB7
:1020C0008117100E815D54E024C081F0030E81174A
:1020D000010E8163B4D7FBD0349A3D903D92E00E5F
:1020E000F76E200EF66E23EE00F0EEEC65F0DE6A81
:1020F000DFEC65F0640EAE6F320EAD6F3DB0A1EF58
:1021000010F03DB286EF10F0AD67F8D73D92FE0EAD
:10211000F76E7C0EF66E20EED6F0F5EC65F0FE0E56
:10212000F76E8C0EF66E20EEE6F0F5EC65F013EC33
:1021300066F0640EAE6F280EAD6FAD67FED73090BF
:10214000C4D63D90FE0EF76E9C0EF66E20EED6F0D5
:10215000F5EC65F0FE0EF76EAC0EF66E20EEE6F0D6
:10216000F5EC65F013EC66F081A261EF14F0FCD79A
:1021700064A565D76495040E976F8A2B040E8A6157
:102180008A6B19EEA2F0080E8A03F350E126F45090
:10219000E222E6CF7CF0E6CF7DF0E6CF7EF0E6CF20
:1021A0007FF0E6CF80F0E6CF81F0E6CF7AF0E6CFA1
:1021B0007BF0200E7D5D04E07A671FD07B671DD029
:1021C0008A2B972FDED7E50EF76EDE0EF66E20EE29
:1021D000D6F0F5EC65F0E50EF76EEE0EF66E20EE3D
:1021E000E6F0F5EC65F013EC66F0640EAE6F320EBF
:1021F000AD6FAD67FED73DEF0AF003EE00F0410E84
:10220000EE6E540EEE6E2B0EEE6E430EEE6E4F0E15
:10221000EE6E500EEE6E530EEE6E3D0EEE6E310E05
:10222000EE6E2C0EEE6E320EEE6E2C0EEE6E7CC04E
:10223000EEFF7DC0EEFF7EC0EEFF7FC0EEFF80C0F0
:10224000EEFF81C0EEFF000EEE6E3D6A576A586ADF
:10225000DFEC65F0640EAE6FC80EAD6F3DB05DEFA4
:1022600011F03DB236EF11F0AD67F8D73D92E50EB3
:10227000F76E8E0EF66E20EED6F0F5EC65F0E50EFC
:10228000F76EAE0EF66E20EEE6F0F5EC65F07CC073
:10229000E0F07DC0E1F07EC0E2F07FC0E3F080C0FE
:1022A000E4F081C0E5F013EC66F0640EAE6F320E20
:1022B000AD6FAD67FED73DEF0AF064957AC065F06B
:1022C0007BC066F065C0BDF066C0BEF07CD664A180
:1022D000B6D664913EEC5DF03D903D92E00EF76E17
:1022E000800EF66E23EE00F0EEEC65F0DE6ADFECB9
:1022F00065F0640EAE6F640EAD6F3DB087EF11F008
:102300003DB285EF11F0AD67F8D73D9298D6060E35
:10231000976F632B060E6361636B09EE16F0160E62
:102320006303F350E926F450EA26EECF7AF0EECFBD
:102330007BF0EECF7CF0EECF7DF0EECF7EF0EECFF7
:102340007FF0300E286412D07A51286285D07B51FC
:10235000296282D07C512A627FD07D512B627CD051
:102360007E512C6279D07F512D6276D0EECF7AF0FB
:10237000EECF7BF0EECF7CF0EECF7DF0200E7A5DDD
:102380006BE07A515B620AD07B515C6207D07C5172
:102390005D6204D07D515E6201D05ED07AC0C2F928
:1023A0007BC0C3F97CC0C4F97DC0C5F909EE24F037
:1023B000160E6303F350E926F450EA26EECFC6F971
:1023C000EECFC7F9EECFC8F9EECFC9F9EECF7EF068
:1023D000EECF7FF0EECF80F0EECF81F0200E7F5D6C
:1023E000300ED8B47F6F200E805D300ED8B4806F71
:1023F0000FEC61F0845125602FD0C2C95BF0C3C9D6
:102400005CF0C4C95DF0C5C95EF003EE00F0410E9A
:10241000EE6E540EEE6E2B0EEE6E430EEE6EEE6E04
:10242000450EEE6E4C0EEE6EEE6E3D0EEE6EC6C9B5
:10243000EEFFC7C9EEFFC8C9EEFFC9C9EEFFEE6ADD
:102440005A6ADFEC65F0C6C95FF0C7C960F0C8C959
:1024500061F0C9C962F0F3D5972F5BD7F0D55A90D8
:102460005A98EDD55A6AEE0EF76EAE0EF66E20EE65
:10247000D6F0F5EC65F0EE0EF76EBE0EF66E20EEC1
:10248000E6F0F5EC65F013EC66F0D9D5579038908E
:102490003492E40EF76E4E0EF66E20EED6F0F5ECAA
:1024A00065F0E40EF76E6E0EF66E20EEE6F0F5ECDB
:1024B00065F013EC66F0C3D5579238903492E40E71
:1024C000F76E4E0EF66E20EED6F0F5EC65F0E40EEB
:1024D000F76E7E0EF66E20EEE6F0F5EC65F013EC8E
:1024E00066F039963982640EAE6F140EAD6FAD672B
:1024F000FED73DEF0AF05990389034923DEF0AF044
:1025000059923DEF0AF06793C2D76795D6D73896B0
:102510001EC09AF09A3B030E9A17000E9A630ED0D3
:102520003D903D92DF0EF76EEE0EF66E23EE00F05C
:10253000EEEC65F0DE6ADFEC65F01ED0010E9A630A
:102540000ED03D903D92DF0EF76EFA0EF66E23EE42
:1025500000F0EEEC65F0DE6ADFEC65F00DD03D904A
:102560003D92E00EF76E060EF66E23EE00F0EEECF6
:1025700065F0DE6ADFEC65F0640EAE6F320EAD6FB3
:102580003DB0CCEF12F03DB2C9EF12F0AD67F8D715
:1025900003D53D92CCEF0FF03D90FED43D903D929F
:1025A000E10EF76E000EF66E23EE00F0EEEC65F035
:1025B000DE6ADFEC65F007D5040E976F8A6B19EEC3
:1025C000A2F0080E8A03F350E126F450E222E6CF8F
:1025D0007CF0E6CF7DF0E6CF7EF0E6CF7FF0E6CF71
:1025E00080F0E6CF81F0E6CF7AF0E6CF7BF0200EE8
:1025F0007D5D04E07A671FD07B671DD08A2B972F03
:10260000DED7E50EF76EDE0EF66E20EED6F0F5ECB8
:1026100065F0E50EF76EEE0EF66E20EEE6F0F5ECE8
:1026200065F013EC66F0640EAE6F280EAD6FAD670B
:10263000FED73DEF0AF003EE00F0410EEE6E540EB1
:10264000EE6E2B0EEE6E430EEE6E4F0EEE6E500ED5
:10265000EE6E530EEE6E3D0EEE6E310EEE6E2C0EE5
:10266000EE6E320EEE6E2C0EEE6E7CC0EEFF7DC076
:10267000EEFF7EC0EEFF7FC0EEFF80C0EEFF81C0A8
:10268000EEFF000EEE6E3D6A576A586ADFEC65F0A9
:10269000640EAE6FC80EAD6F3DB07BEF13F03DB270
:1026A00054EF13F0AD67F8D73D92E50EF76E8E0E3E
:1026B000F66E20EED6F0F5EC65F0E50EF76EAE0E98
:1026C000F66E20EEE6F0F5EC65F07CC0E0F07DC043
:1026D000E1F07EC0E2F07FC0E3F080C0E4F081C0B2
:1026E000E5F013EC66F0640EAE6F320EAD6FAD67C1
:1026F000FED73DEF0AF064957AC065F07BC066F0C6
:1027000065C0BDF066C0BEF05ED4E50EF76E6E0E1D
:10271000F66E20EED6F0F5EC65F0E50EF76E7E0E67
:10272000F66E20EEE6F0F5EC65F0200E9BC99AF00F
:102730009A631AD0E50EF76EBE0EF66E20EED6F056
:10274000F5EC65F0E50EF76ECE0EF66E20EEE6F0D7
:10275000F5EC65F013EC66F0640EAE6F280EAD6F0D
:10276000AD67FED73DEF0AF003EE00F0410EEE6ECE
:10277000540EEE6E2B0EEE6E430EEE6E4F0EEE6EA0
:10278000500EEE6E530EEE6E3D0EEE6E310EEE6E90
:102790002C0EEE6E320EEE6E2C0EEE6E19EE9AF0E0
:1027A000060E976F200EE75C05E0E6CFEEFF972F51
:1027B000D2EF13F0000EEE6E3D6A576A586ADFECF6
:1027C00065F0640EAE6FC80EAD6F3DB012EF14F041
:1027D0003DB2EDEF13F0AD67F8D73D92E50EF76E21
:1027E0008E0EF66E20EED6F0F5EC65F0E50EF76E87
:1027F000AE0EF66E20EEE6F0F5EC65F0060E976F85
:1028000019EE9AF000EEE0F0E6CFEEFF972FFCD73E
:1028100013EC66F0640EAE6F320EAD6FAD67FED78F
:102820003DEF0AF0E50EF76E8E0EF66E20EED6F056
:10283000F5EC65F0E50EF76E9E0EF66E20EEE6F016
:10284000F5EC65F0060E976F19EE9AF000EEE0F0E9
:10285000E6CFEEFF972FFCD713EC66F0640EAE6F59
:10286000320EAD6FAD67FED7E3EF0FF0CAEC5CF050
:102870001FEF10F0A66BA76B53EC63F0A68753EC29
:1028800063F0BFC081F0030E8117816705D0020E8F
:10289000C06FC16BBF8F0CD0010E816305D0030EDA
:1028A000C06FC16BBF8F04D0060EC06FC16BBF8FEE
:1028B00081A258EF14F0FC0EBF0BAFEC61F065EF96
:1028C0000FF021EC62F0A5EC62F0A66BA76B53EC65
:1028D00063F0A68753EC63F0A78953EC63F0320EE4
:1028E000AB6FAB67FED7FFEC65F009EC66F0E60E68
:1028F000F76E5E0EF66E20EED6F0F5EC65F009ECA4
:1029000066F013EC66F0010EC06FC16BBF8F2EEC4A
:102910005DF03494640EAB6FAB67FED7640EAE6FA0
:10292000FA0EAD6F81B29CEF14F0A0B10AD0AD6782
:10293000F9D7010EBF139ED7AFEC61F0348265EF7B
:102940000FF0AFEC61F001EED2F010EEE6F09E6B0E
:1029500034943496FCEC61F09DC0EEFF9DC0E6FF20
:1029600013EC66F09E2B230E9D5DD8B434842A0EA2
:102970009D5DD8B43486640EAE6F17C0ADF081B2E1
:102980001AEF15F0A0B104D0AD67F9D766EF15F0D6
:10299000FCEC61F09E2B230E9D6306D034B4C5EF92
:1029A00034F034B649D008D02A0E9D63DCEF14F021
:1029B00034B67DD034B4B4D0020E9E6307D034A4B4
:1029C00005D02B0EE8CFD2F1E8CFE6F03494349660
:1029D000110E9E61F4EF14F09DC0EEFF9DC0E6FF66
:1029E00013EC66F0BBEF14F0E7C0E6F0E8C0E7F0E8
:1029F000E9C0E8F0EAC0E9F0EBC0EAF0ECC0EBF0C7
:102A0000EDC0ECF0EEC0EDF0EFC0EEF0F0C0EFF096
:102A1000F1C0F0F0F2C0F1F0F3C0F2F0F4C0F3F066
:102A2000F5C0F4F09DC0EEFF9DC0F5F013EC66F02C
:102A3000BBEF14F065EF0FF0FF0EF76E1C0EF66E95
:102A400020EED6F0F5EC65F009EC66F0100E976F0D
:102A500008EE22F010EEE6F0EECFE6FF972FFCD75F
:102A600013EC66F081B265EF0FF0A0B139EF15F00D
:102A7000F9D7FCEC61F0FF0EF76E2C0EF66E20EE2F
:102A8000D6F0F5EC65F0FF0EF76E4C0EF66E20EE0C
:102A9000E6F0F5EC65F013EC66F081B265EF0FF04F
:102AA000A0B154EF15F0F9D7FCEC61F0C5D7E70EF3
:102AB000F76E4E0EF66E20EEE6F0F5EC65F013ECD8
:102AC00066F081A261EF15F065EF0FF015EC30F0C4
:102AD000E866BAEF15F0040EC06FC16BBF8F39B650
:102AE0000AD0E70EF76E6E0EF66E20EED6F0F5EC1D
:102AF00065F039940AD0E70EF76E7E0EF66E20EE82
:102B0000D6F0F5EC65F03984398213EC66F038863E
:102B100088EC30F0E86602D0B8EF1CF065EF0FF0FB
:102B2000E60EF76ECE0EF66E20EED6F0F5EC65F002
:102B3000E60EF76EDE0EF66E20EEE6F0F5EC65F0D2
:102B400013EC66F0809A358CA66BA76B53EC63F0A0
:102B5000A68953EC63F0A68353EC63F081B2B2EF25
:102B600015F0FCD7A66BA76B53EC63F0808A359CFD
:102B700065EF0FF0E70EF76E0E0EF66E20EED6F054
:102B8000F5EC65F009EC66F013EC66F0809A358C94
:102B9000A66BA76B53EC63F0A68F53EC63F0A6898A
:102BA00053EC63F0A68353EC63F0320EAB6FAB676C
:102BB000FED782AA2AEF16F0358E640EAE6F080E8D
:102BC000AD6FAD67FED79E6B01EED2F011EE78F0DF
:102BD000200EE76430D0040E976FEF50E7622BD0E1
:102BE000EE50E650200EE76201D002D0972FF5D7C5
:102BF00097C09AF010EEE6F0040E976F01EE78F0B1
:102C00000CAEAAEC2DF00CBEEBEC2DF0E86639D042
:102C10000F5009E0976F640EAE6F0A0EAD6FAD678F
:102C2000FED7972FF8D701EED2F09A510508E92682
:102C3000E86AEA2204D001EED2F010EEE6F0200EAF
:102C4000976F0CAEAAEC2DF00CBEEBEC2DF0E86605
:102C500018D02DD0808A359C359EF90EF76E0E0E59
:102C6000F66E20EED6F0F5EC65F0F90EF76E1E0E5E
:102C7000F66E20EEE6F0F5EC65F013EC66F054EF3E
:102C800014F0808A359CF90EF76E9E0EF66E20EEDB
:102C9000D6F0F5EC65F0F90EF76EAE0EF66E20EE9E
:102CA000E6F0F5EC65F013EC66F04CEF14F0A66B73
:102CB000A76B53EC63F0A68953EC63F0A68353EC47
:102CC00063F0A78953EC63F0A68753EC63F0E70E3B
:102CD000F76E1E0EF66E20EED6F0F5EC65F013ECF6
:102CE00066F0A5EC62F0FCEC61F0A06B579C3494AC
:102CF00081B28CEF16F038B4A5EF16F03DB6B1EF07
:102D000016F057BC94EF16F0A0A1F2D7FCEC61F0DE
:102D1000230E9D63EDD74FD0FA0EAB6FAB67FED796
:102D200081B209EF18F0E4D7579C010E7063E0D729
:102D300038943D96E70EF76E1E0EF66E20EED6F036
:102D4000F5EC65F013EC66F0D3D73894F60EF76E19
:102D5000AE0EF66E20EED6F0F5EC65F013EC66F0F4
:102D6000C7D73D96E8EC17F0030E1E140208D8A44E
:102D7000BFD7D5EC33F03BA0BBD73D903D92640E5E
:102D8000AE6F140EAD6F3D903D92DF0EF76EBE0E2E
:102D9000F66E23EE00F0EEEC65F0DE6ADFEC65F037
:102DA0003DB0D7EF16F03DB2D9EF16F0F9D73D9010
:102DB0009FD73D929DD73484E70EF76E2E0EF66EA8
:102DC00020EED6F0F5EC65F009EC66F013EC66F059
:102DD0002EEC5DF001EED2F010EEE6F09E6B640E8C
:102DE000AE6F17C0ADF081B209EF18F038B4B2EF92
:102DF00017F03DB6BEEF17F057BCA1EF17F0A0B12A
:102E000005EF17F0AD67EFD742D0FCEC61F0230E71
:102E10009D6309D034A43BD001EE50F0200EEF6248
:102E200053D0349442D034942A0E9D5D35E09E2BCD
:102E3000110E9E6107D09DC0EEFF9DC0E6FF13EC12
:102E400066F0CDD7E7C0E6F0E8C0E7F0E9C0E8F00B
:102E5000EAC0E9F0EBC0EAF0ECC0EBF0EDC0ECF05A
:102E6000EEC0EDF0EFC0EEF0F0C0EFF0F1C0F0F02A
:102E7000F2C0F1F0F3C0F2F0F4C0F3F0F5C0F4F0FA
:102E80009DC0EEFF9DC0F5F013EC66F0A8D701EEF3
:102E9000D2F0200EEF6233D02EEC5DF009EC66F03C
:102EA0008FEC34F0FCEC61F012D7E70EF76E8E0E6B
:102EB000F66E20EED6F0F5EC65F013EC66F0AAECB9
:102EC00034F0FCEC61F003D72EEC5DF0100E8B6F4C
:102ED0009E6B11EED2F001EE50F0200EEF5C05E09B
:102EE000EECFE6FF9E2B8B2FF8D7100E8B6F01EEE7
:102EF000D2F010EEE6F0EECFE6FF8B2FFCD7A66BFC
:102F0000A76B53EC63F0A68F53EC63F0A78B53ECE5
:102F100063F0040EC06FC16BBF8F24AC06D0A68DCA
:102F200053EC63F0A78353EC63F0E70EF76E3E0EAD
:102F3000F66E20EED6F0F5EC65F013EC66F029EFB6
:102F40001BF0579C010E70634AD738943D96E70EEC
:102F5000F76E1E0EF66E20EED6F0F5EC65F013EC73
:102F600066F03DD73894F60EF76EAE0EF66E20EE94
:102F7000D6F0F5EC65F013EC66F031D73D96E8EC51
:102F800017F0030E1E140208D8A429D7D5EC33F08D
:102F90003BA025D73D903D92640EAE6F140EAD6FF1
:102FA0003D903D92DF0EF76EBE0EF66E23EE00F002
:102FB000EEEC65F0DE6ADFEC65F03DB0E4EF17F0B3
:102FC0003DB2E6EF17F0ECD63D9009D73D9207D71A
:102FD00000EEDBF00B0E976F200EEE6E972FECEFEE
:102FE00017F001EE8CF010EEDBF00A0E976FEECFCB
:102FF000E6FF972FF7EF17F013EC66F0100E976FC0
:1030000001EE8CF011EE9EF0EECFE6FF972FFCD78D
:10301000120021EC62F0A06BA5EC62F0808A359C76
:10302000A66BA76B53EC63F0F70EF76E1E0EF66EF1
:1030300020EED6F0F5EC65F0F70EF76E2E0EF66E7C
:1030400020EEE6F0F5EC65F05AEC33F013EC66F0A8
:10305000640EAE6F140EAD6FAD67FED7C00E3516A1
:1030600065EF0FF0808A359C3C0EAB6FAB67FED7E7
:10307000809A358C280EAB6FAB67FED79F2FF2D7A7
:103080001200640EAE6F140EAD6F35B403D0AD6791
:10309000FCD70FD0A66BA76B53EC63F0A78B53EC58
:1030A00063F081962EEC2FF08186A66BA76B53EC14
:1030B00063F0F60EF76E8E0EF66E20EED6F0F5EC9F
:1030C00065F0F60EF76E8E0EF66E20EEE6F0F5EC7D
:1030D00065F013EC66F0F2EC2FF0640EAE6F1E0E8E
:1030E000AD6F36B202D0AD67FCD70CC081F0030ED5
:1030F00081178167A3D037B006D001EE8CF0200E87
:10310000EE6EEE6E0AD010EEE6F001EE8CF0100ED0
:10311000976FE6CFEEFF972FFCD7F6EC2EF0A66B5D
:10312000A76B53EC63F0A78953EC63F0A68753ECCD
:1031300063F0140E6C6F1AC06DF03A903A923A86B2
:103140003A94C56B808680948092808016A44ED07D
:1031500016C081F0030E8117816718D0140E6C6FB2
:103160001AC06DF03A903A923A863A94C56B8086CE
:103170008094809280803AA4FED7640EAE6F060ED3
:10318000AD6FAD67FED77CEC2EF030D0010E8163C1
:1031900012D055EC33F02BEC2EF0140E6C6F1AC0DD
:1031A0006DF03A903A923A863A94C56B8086809454
:1031B000809280801BD0020E8163D0D7140E6C6F7A
:1031C0001AC06DF03A903A923A863A94C56B80866E
:1031D0008094809280803AA4FED7640EAE6F060E73
:1031E000AD6FAD67FED77CEC2EF000D081A208EF6A
:1031F00019F035A6FDEF18F0F9D73A6A8086809469
:1032000080828090FA0EAB6FAB67FED765EF0FF050
:10321000AFEC61F03A6A80868094808280904EECB8
:1032200033F0809A358C3596FA0EAB6FAB67FED7CC
:1032300009EC66F013EC66F057EF16F0010E8163AF
:10324000E8D0A66BA76B53EC63F0A68F53EC63F04A
:10325000A78B53EC63F0A68D53EC63F0A78353EC7C
:1032600063F021EC62F0A5EC62F0809A358C359623
:10327000E70EF76E0E0EF66E20EED6F0F5EC65F06A
:103280002EEC5DF009EC66F013EC66F0640EAE6FA8
:10329000050EAD6FAD67FED7050EC06FC16BBF8F5A
:1032A00001EED2F010EEE6F09E6B640EAE6F640E8F
:1032B000AD6FA0B103D0AD67FCD7A3D0AFEC61F088
:1032C000FCEC61F0230E9D6301D0DAD79DC0EEFFC8
:1032D0009DC0E6FF13EC66F09E2B11509E6149D015
:1032E000640EAE6F12C0ADF0640EB06F1350AF6FCE
:1032F000A0B109D010509E6103D0AF67F9D781D03B
:10330000AD67F6D736D0FCEC61F0230E9D6301D09B
:10331000B7D79E2B110E9E6107D09DC0EEFF9DC0BA
:10332000E6FF13EC66F0D9D7E7C0E6F0E8C0E7F0B7
:10333000E9C0E8F0EAC0E9F0EBC0EAF0ECC0EBF07D
:10334000EDC0ECF0EEC0EDF0EFC0EEF0F0C0EFF04D
:10335000F1C0F0F0F2C0F1F0F3C0F2F0F4C0F3F01D
:10336000F5C0F4F09DC0EEFF9DC0F5F013EC66F0E3
:10337000B4D7A66BA76B53EC63F0A68F53EC63F046
:10338000A78B53EC63F0040EC06FC16BBF8F24ACEE
:10339000D0EF19F0A68D53EC63F0A78353EC63F0E4
:1033A0000CA657D110509E6554D1100E976F01EEA8
:1033B000D2F011EE8CF0EECFE6FF972FFCD789EC20
:1033C00033F03CB846D1808A359CFE0EF76E3C0E39
:1033D000F66E20EED6F0F5EC65F0FE0EF76E4C0EB4
:1033E000F66E20EEE6F0F5EC65F013EC66F0640E98
:1033F000AE6F140EAD6FAD67FED7C00E351665EF1C
:103400000FF0A66BA76B53EC63F0808A359C65EFD9
:103410000FF0020E81636FD601EE50F0200EEF62C6
:1034200013D0F60EF76EFE0EF66E20EED6F0F5EC2B
:1034300065F0F70EF76E0E0EF66E20EEE6F0F5EC88
:1034400065F013EC66F057D60E503BE1A66BA76B08
:1034500053EC63F0A68F53EC63F0A78B53EC63F04F
:1034600024AC0CD0809A358CA68D53EC63F0A783E6
:1034700053EC63F0040EC06FC16BBF8FE70EF76EA5
:103480003E0EF66E20EED6F0F5EC65F009EC66F037
:103490002EEC5DF0100E8B6F11EED2F001EE50F0BD
:1034A000EECFE6FF8B2FFCD7100E8B6F01EED2F024
:1034B00010EEE6F0EECFE6FF8B2FFCD713EC66F0B4
:1034C000C8D001EE50F037B006D001EE8CF0200EDF
:1034D000EE6EEE6E0AD010EEE6F001EE8CF0100EFD
:1034E000976FE6CFEEFF972FFCD7F6EC2EF0A66B8A
:1034F000A76B53EC63F0A78953EC63F0A68753ECFA
:1035000063F0140E6C6F1AC06DF03A903A923A86DE
:103510003A94C56B808680948092808016A44DD0AA
:1035200016C081F0030E8117816718D0140E6C6FDE
:103530001AC06DF03A903A923A863A94C56B8086FA
:103540008094809280803AA4FED7640EAE6F060EFF
:10355000AD6FAD67FED77CEC2EF02FD0010E8163EE
:1035600012D055EC33F02BEC2EF0140E6C6F1AC009
:103570006DF03A903A923A863A94C56B8086809480
:10358000809280801AD0020E8163E8D5140E6C6F91
:103590001AC06DF03A903A923A863A94C56B80869A
:1035A0008094809280803AA4FED7640EAE6F060E9F
:1035B000AD6FAD67FED7B9EC2EF0A66BA76B53ECE1
:1035C00063F0A68F53EC63F0A78B53EC63F024AC4D
:1035D0000CD0809A358CA68D53EC63F0A78353EC06
:1035E00063F0040EC06FC16BBF8F81A208EF19F0AA
:1035F00024BC03D035A61EEF1BF00E50C563F5D7D3
:103600003A6A80868094808280902EEC5DF0100E65
:103610008B6F11EED2F001EE50F0EECFE6FF8B2F64
:10362000FCD7100E8B6F01EED2F010EEE6F0EECF6D
:10363000E6FF8B2FFCD713EC66F00BD03A6A80863E
:10364000809480828090FA0EAB6FAB67FED765EFF7
:103650000FF00CA406D015EC30F0E8661FD039B698
:103660000BD0E70EF76E6E0EF66E20EED6F0F5EC90
:1036700065F0399639940AD0E70EF76E7E0EF66E35
:1036800020EED6F0F5EC65F03984398213EC66F063
:10369000388688EC30F0E86601D02AD0FE0EF76E4E
:1036A0005C0EF66E20EED6F0F5EC65F0FE0EF76ED1
:1036B0006C0EF66E20EEE6F0F5EC65F013EC66F0BD
:1036C000809A358CA68F53EC63F0A78B53EC63F094
:1036D000030EC06FC16BBF8F640EAE6F140EAD6F63
:1036E000AD67FED7808A359CC00E351665EF0FF0AA
:1036F000EEEC28F0E60EF76E9E0EF66E20EED6F09B
:10370000F5EC65F0310E39B4320EE56F13EC66F06E
:10371000B2EC62F021EC62F00CEC5CF01E0EBA6FC1
:10372000A0B118EC5CF0A0B5E5D0A0AB03D0AF51D0
:10373000D8B4E0D057B0C0EF1BF057B4C2EF1BF0C5
:1037400057BAC4EF1BF057BCC6EF1BF058B0CBEF15
:103750001BF058B2CDEF1BF03DB2D2EF1BF03DB0E5
:10376000F0EF1BF03EB0D4EF1BF03EB2E2EF1BF0E7
:1037700035BC03D035A67AEF1CF0BA67D1D7A7D0F5
:103780005790A5D05794CCD7579ACAD7579C010EBB
:103790007063C6D79CD058909AD0589224BCAFEC96
:1037A00061F0BED73D9293D03E90FC0EF76EEE0EC8
:1037B000F66E20EED6F0F5EC65F0ABEC1CF013ECF9
:1037C00066F0AAD03E92FD0EF76E0E0EF66E20EE5B
:1037D000D6F0F5EC65F0ABEC1CF013EC66F09CD089
:1037E0003D90AFEC61F0809A358CA66BA76B53ECE3
:1037F00063F0A78B53EC63F0A68D53EC63F0A783C3
:1038000053EC63F0E60EF76EAE0EF66E20EED6F0D9
:10381000F5EC65F0310E39B4320EE56F13EC66F05D
:1038200021EC62F0A0B118EC5CF0A0B563D0A0ABC5
:1038300003D0AF51D8B45ED057B035EF1CF057BCB1
:1038400037EF1CF058B03CEF1CF03DB03EEF1CF0E1
:103850003DB240EF1CF03EB042EF1CF03EB250EFE4
:103860001CF03DB45EEF1CF0DDD7579030D0579C74
:10387000010E7063D7D72BD0589029D03D90D2D766
:103880003D9225D03E90FC0EF76EEE0EF66E20EEC9
:10389000D6F0F5EC65F0ABEC1CF013EC66F03CD028
:1038A0003E92FD0EF76E0E0EF66E20EED6F0F5ECA3
:1038B00065F0ABEC1CF013EC66F02ED03D94030EDB
:1038C0001E140208D8A4AED7D5EC33F0ABD7F70E50
:1038D000F76E5E0EF66E20EED6F0F5EC65F0F70EA4
:1038E000F76E6E0EF66E20EEE6F0F5EC65F013EC7A
:1038F00066F012D0F70EF76E3E0EF66E20EED6F0A2
:10390000F5EC65F0F70EF76E4E0EF66E20EEE6F073
:10391000F5EC65F013EC66F0AFEC61F0A66BA76B0D
:1039200053EC63F0808A359C3D903D92DF0EF76E3C
:10393000BE0EF66E23EE00F0EEEC65F0DE6ADFEC14
:1039400065F0640EAE6F140EAD6FAD67FED7C00E9E
:10395000351665EF0FF009EC66F0100E976F11EE5B
:10396000D2F000EEE6F0E6CFEEFF972FFCD7120084
:10397000A66BA76B53EC63F0A78153EC63F0A687AB
:1039800053EC63F024AC03D0A68553EC63F003EE54
:1039900000F0410EEE6E540EEE6E440EEE6E9EC0C2
:1039A00097F011EED2F0E6CFEEFF972FD3EF1CF099
:1039B0003B0EEE6E000EEE6E3D6A3E6A576A586A26
:1039C000DFEC65F0E60EF76E9E0EF66E20EED6F09A
:1039D000F5EC65F0310E39B4320EE8CFE5F013ECBA
:1039E00066F03C0EBA6F57B013EF1DF057BC19EFDD
:1039F0001DF058B022EF1DF058B232EF1DF03DB26D
:103A000037EF1DF03DB05DEF1DF03EB03DEF1DF016
:103A10003EB24DEF1DF081B233EF1EF0BA67E3D72F
:103A2000AFEC61F00DD15790AFEC61F0020EBF1317
:103A300007D1579C010E7063D6D7AFEC61F0010E31
:103A4000BF13FED05890AFEC61F0020EBF13E40E2E
:103A5000F76EAE0EF66E20EEE6F0F5EC65F013ECC8
:103A600066F013D1589224BCAFEC61F0BCD73D9204
:103A7000AFEC61F0020EBF13E3D03E90AFEC61F00B
:103A8000FD0EF76E2E0EF66E20EED6F0F5EC65F01C
:103A900013EC66F0000EBF13D3D03E92AFEC61F092
:103AA000FD0EF76E4E0EF66E20EED6F0F5EC65F0DC
:103AB00013EC66F0000EBF13C3D03D90AFEC61F085
:103AC000A66BA76B53EC63F0A78153EC63F0A6855C
:103AD00053EC63F0A68F53EC63F04EEC33F0640EBE
:103AE000AB6FAB67FED7E60EF76EAE0EF66E20EE4E
:103AF000D6F0F5EC65F0310E39B4320EE8CFE5F0D2
:103B000013EC66F081B233EF1EF035B658D057B0E3
:103B10009DEF1DF057BCA1EF1DF058B0A8EF1DF0B0
:103B20003DB2B6EF1DF03EB0BAEF1DF03EB2C8EFA9
:103B30001DF03DB4D6EF1DF0E5D75790020EBF1330
:103B40007FD0579C010E7063DDD7010EBF1378D074
:103B50005890020EBF13E40EF76EAE0EF66E20EE16
:103B6000E6F0F5EC65F013EC66F08FD03D92020EB6
:103B7000BF1366D03E90FD0EF76E2E0EF66E20EE51
:103B8000D6F0F5EC65F013EC66F0000EBF1358D0DC
:103B90003E92FD0EF76E4E0EF66E20EED6F0F5EC70
:103BA00065F013EC66F0000EBF134AD03D94030E8F
:103BB0001E140208D8A4A6D7D5EC33F0A3D7809A58
:103BC000358CF60EF76E6E0EF66E20EED6F0F5EC36
:103BD00065F0F60EF76E7E0EF66E20EEE6F0F5EC72
:103BE00065F013EC66F0640EAE6F280EAD6F020E3A
:103BF000C06FC16BBF8FAD67FED7AFEC61F0808A3D
:103C0000359CC00E3516E60EF76EAE0EF66E20EE43
:103C1000D6F0F5EC65F0310E39B4320EE8CFE5F0B0
:103C20009EC097F009EC66F011EED2F000EEE6F0DF
:103C3000E6CFEEFF972F18EF1EF013EC66F062D779
:103C4000F70EF76E5E0EF66E20EED6F0F5EC65F030
:103C5000F70EF76E6E0EF66E20EEE6F0F5EC65F000
:103C600013EC66F012D0F70EF76E1E0EF66E20EE15
:103C7000D6F0F5EC65F0F70EF76E2E0EF66E20EE30
:103C8000E6F0F5EC65F013EC66F05AEC33F03D909D
:103C90003D92DF0EF76EBE0EF66E23EE00F0EEECF8
:103CA00065F0DE6ADFEC65F0640EAE6F140EAD6F8A
:103CB000AD67FED73D903D923E6A579A579C8B6BFD
:103CC0003AEF14F0E60EF76E6E0EF66E20EED6F0BA
:103CD000F5EC65F0E60EF76EEE0EF66E20EEE6F011
:103CE000F5EC65F013EC66F0C56B3B923D963E6AD1
:103CF0005790579C5890640EAE6FFA0EAD6F57B048
:103D000097EF1EF057BC99EF1EF058B09EEF1EF0D3
:103D10003EB0A0EF1EF03EB2A0EF1EF03DB6BFEFEA
:103D20001EF038B4D6EF1EF0AD67E9D70AD0579031
:103D300008D0579C010E7063E2D703D0589001D091
:103D40003E6A3D903D923D903D92DF0EF76EBE0E75
:103D5000F66E23EE00F0EEEC65F0DE6ADFEC65F067
:103D6000640EAE6F140EAD6F3DB0BCEF1EF03DB2F1
:103D7000BCEF1EF0AD67F8D7389465EF0FF03D96B5
:103D80003BB2BDD73B8209EC66F001EE8CF0200E11
:103D9000EF5CB5E010EEE6F0100E976FEECFE6FFA9
:103DA000972FCEEF1EF013EC66F0A9D73894C52BF1
:103DB000010EC565A4D71EC081F0030E811781676F
:103DC00087EF20F034D0F70EF76EDE0EF66E20EEA1
:103DD000D6F0F5EC65F0F70EF76EEE0EF66E20EE0F
:103DE000E6F0F5EC65F013EC66F03B903B923D900D
:103DF0003D92DF0EF76EBE0EF66E23EE00F0EEEC97
:103E000065F0DE6ADFEC65F0640EAE6F140EAD6F28
:103E10003DB010EF1FF03DB210EF1FF0AD67F8D7C7
:103E2000AD67FED73D903D923D96C4EF0FF01EA4C6
:103E30000CD089EC33F03CB208D0500EEA6303D0CA
:103E40001EBE03D0C0D716A6BED73D903D923E6A97
:103E50005790579C5890F6EC2EF0A66BA76B53EC3E
:103E600063F0A78953EC63F0A68753EC63F016B4B4
:103E70000ED0140E6C6F1AC06DF03A903A923A86DA
:103E80003A94C56B808680948092808034D016C02E
:103E900081F0030E8117816718D0140E6C6F1AC061
:103EA0006DF03A903A923A863A94C56B8086809447
:103EB000809280803AA4FED7640EAE6F060EAD6F7E
:103EC000AD67FED77CEC2EF016D0010E816312D0C8
:103ED00055EC33F02BEC2EF0140E6C6F1AC06DF015
:103EE0003A903A923A863A94C56B80868094809252
:103EF000808001D0D2D781B285EF1FF0640EAB6F06
:103F0000AB67FED781A29FEF1FF057B08FEF1FF076
:103F100057BC93EF1FF058B091EF1FF0ECD75790BC
:103F200006D0589004D0579C010E7063E4D73894A3
:103F30003A6A808680948082809065EF0FF03A6ABA
:103F400080868094808280904EEC33F0FA0EAB6FC6
:103F5000AB67FED7E60EF76EAE0EF66E20EED6F02D
:103F6000F5EC65F013EC66F0A66BA76B53EC63F011
:103F7000A78153EC63F0A68553EC63F0A68F53EC56
:103F800063F038BE0DD03D903D92DF0EF76EC40E4B
:103F9000F66E23EE00F0EEEC65F0DE6ADFEC65F025
:103FA00081B2E8EF1FF03DB03D9057BC31EF20F0FB
:103FB00035B6F0EF1FF03DB4DFEF1FF0F1D73D94C1
:103FC000030E1E140208D8A4EBD7D5EC33F0E8D7C3
:103FD000FA0EAB6FAB67FED781B24BEF20F0E0D7A4
:103FE000809A358CF60EF76E6E0EF66E20EED6F0D9
:103FF000F5EC65F0F60EF76E7E0EF66E20EEE6F04E
:10400000F5EC65F013EC66F0640EAE6F280EAD6F44
:10401000020EC06FC16BBF8FAD67FED7AFEC61F012
:10402000808A359CC00E3516E60EF76EAE0EF66E23
:1040300020EED6F0F5EC65F0310E39B4320EE8CF53
:10404000E5F009EC66F001EE8CF010EEE6F0100EF3
:10405000976FEECFE6FF972F29EF20F013EC66F075
:104060009FD7579C010E70639BD73894F70EF76E5D
:104070005E0EF66E20EED6F0F5EC65F0F70EF76EFC
:104080006E0EF66E20EEE6F0F5EC65F013EC66F0E1
:10409000010EBF1312D0F70EF76E1E0EF66E20EE55
:1040A000D6F0F5EC65F0F70EF76E2E0EF66E20EEFC
:1040B000E6F0F5EC65F013EC66F05AEC33F0320EF6
:1040C000AB6FAB67FED73D903D923D903D92DF0ECA
:1040D000F76EBE0EF66E23EE00F0EEEC65F0DE6AD3
:1040E000DFEC65F0640EAE6F140EAD6F3DB07EEF89
:1040F00020F03DB27EEF20F0AD67F8D7640EAE6FD2
:10410000140EAD6FAD67FED738943AEF14F0010E80
:104110008163DAD11EA417D089EC33F03BA003D021
:104120003CB00BD050D6500EEA6303D01EBE05D073
:104130004AD616A648D625EF1FF001EE60F0200EF5
:10414000EF6201D0BCD0100E976F01EE60F011EE5F
:10415000D2F0EECFE6FF972FFCD7A66BA76B53EC00
:1041600063F0A68F53EC63F0A78B53EC63F0809A57
:10417000358C320EAB6FAB67FED782AAA9EF21F068
:10418000358E640EAE6F0A0EAD6FAD67FED721ECB3
:1041900062F038BE0ED03D903D92DF0EF76EC40E39
:1041A000F66E23EE00F0EEEC65F0DE6ADFEC65F013
:1041B000388EF70EF76E8E0EF66E20EED6F0F5EC1A
:1041C00065F013EC66F009EC66F0640EAE6F050E58
:1041D000AD6F3DB03D90AD67FCD7389401EED2F0A5
:1041E00010EEE6F0100E976F0CAEAAEC2DF00CBEA0
:1041F000EBEC2DF0E8664AD03DB03D9057B01BEF98
:1042000021F057BC1DEF21F058B022EF21F03DB254
:1042100024EF21F0A66BA76B53EC63F0A68753EC59
:1042200063F0A78D53EC63F0A68D53EC63F0A78386
:1042300053EC63F0B8D0579009D0579C010E7063CF
:10424000B2D004D0589002D03D9200D0F70EF76E55
:104250005E0EF66E20EED6F0F5EC65F0F70EF76E1A
:104260006E0EF66E20EEE6F0F5EC65F013EC66F0FF
:10427000A66BA76B53EC63F0808A359C640EAE6F1F
:10428000140EAD6FAD67FED765EF0FF0F90EF76E48
:104290009E0EF66E20EED6F0F5EC65F0F90EF76E98
:1042A000AE0EF66E20EEE6F0F5EC65F013EC66F07F
:1042B000808A359CA66BA76B53EC63F05FD0A66B2E
:1042C000A76B53EC63F0A68753EC63F0A78D53EC18
:1042D00063F0A68D53EC63F0A78353EC63F0809AF0
:1042E000358C640EAB6FAB67FED782AAA9EF21F0C5
:1042F000358E3D903D92E10EF76EFA0EF66E23EE8E
:1043000000F0EEEC65F0DE6ADFEC65F0640EAE6F97
:104310000A0EAD6F3DB03D90AD67FCD73C9E349426
:1043200038BE41D0388E3D903D92DF0EF76EC40E00
:10433000F66E23EE00F0EEEC65F0DE6ADFEC65F081
:10434000640EAE6F0A0EAD6F3DB03D90AD67FCD709
:104350002AD0808A359C359EF60EF76EBE0EF66E1C
:1043600020EED6F0F5EC65F0F60EF76ECE0EF66E9A
:1043700020EEE6F0F5EC65F013EC66F03D903D9232
:10438000DF0EF76EBE0EF66E23EE00F0EEEC65F07B
:10439000DE6ADFEC65F0640EAE6F140EAD6FAD67D4
:1043A000FED765EF0FF021EC62F0A5EC62F0A06B98
:1043B000020EC06FC16BBF8FE60EF76EAE0EF66ECB
:1043C00020EED6F0F5EC65F009EC66F001EE8CF02D
:1043D000200EEF5C09E010EEE6F0100E976FEECFC6
:1043E000E6FF972FEFEF21F013EC66F0A0B10CD0B1
:1043F0003DB03D9057B010EF22F057BC14EF22F0C3
:1044000058B012EF22F0F2D73CAED5EC3AF03C8E29
:10441000FCEC61F0230E9D63E9D71EACE7D735D0E5
:10442000579006D0589004D0579C010E7063DED789
:10443000F70EF76E5E0EF66E20EED6F0F5EC65F038
:10444000F70EF76E6E0EF66E20EEE6F0F5EC65F008
:1044500013EC66F0A66BA76B53EC63F0808A359C77
:104460003D903D92DF0EF76EBE0EF66E23EE00F02D
:10447000EEEC65F0DE6ADFEC65F0640EAE6F140EF4
:10448000AD6FAD67FED765EF0FF0F70EF76E9E0EBE
:10449000F66E20EED6F0F5EC65F0F70EF76EAE0E88
:1044A000F66E20EEE6F0F5EC65F013EC66F0A66B28
:1044B000A76B53EC63F0808A359C640EAE6F140ECC
:1044C000AD6FAD67FED739D6020E8163CCEF22F017
:1044D000100E976F11EE8CF001EE9EF0E6CFEEFF1E
:1044E000972FFCD7D5EC33F03BA0ADD43CA420D023
:1044F0003B903B923D903D92DF0EF76EBE0EF66E06
:1045000023EE00F0EEEC65F0DE6ADFEC65F03DB026
:104510008EEF22F03DB28EEF22F0F9D73D903D9222
:104520003D963B86640EB96F320EB86FC4EF0FF044
:10453000F70EF76EDE0EF66E20EED6F0F5EC65F0B7
:10454000F70EF76EEE0EF66E20EEE6F0F5EC65F087
:1045500013EC66F03B903B923D903D92DF0EF76E80
:10456000BE0EF66E23EE00F0EEEC65F0DE6ADFECD8
:1045700065F0640EAE6F140EAD6F3DB0C5EF22F066
:104580003DB2C5EF22F0AD67F8D7AD67FED73D90DD
:104590003D923D96C4EF0FF01EC081F0030E8117CF
:1045A000030E816365EF0FF0100E976F11EE8CF024
:1045B00001EE9EF0E6CFEEFF972FFCD723EC34F010
:1045C0003CA6B6D73B903B923D903D92DF0EF76EF6
:1045D000BE0EF66E23EE00F0EEEC65F0DE6ADFEC68
:1045E00065F03DB0F8EF22F03DB2F8EF22F0F9D7D8
:1045F0003D903D923D963B86640EB96F320EB86F8A
:10460000C4EF0FF015EC30F0E86602D039B60AD0EE
:10461000E70EF76E6E0EF66E20EED6F0F5EC65F056
:1046200039960AD0E70EF76E7E0EF66E20EED6F0C3
:10463000F5EC65F039823984E60EF76E7E0EF66E83
:1046400020EED6F0F5EC65F013EC66F0388688ECD9
:1046500030F0E86665EF0FF0EEEC28F0E60EF76E4E
:104660009E0EF66E20EED6F0F5EC65F0310E39B404
:10467000320EE56F13EC66F0640EAE6FFA0EAD6F9E
:104680003DB076EF23F057B055EF23F057BC57EF0E
:1046900023F058B05CEF23F03EB05EEF23F03EB263
:1046A0006AEF23F0AD67ECD7B2D25790B0D2579CE7
:1046B000010E7063E5D7ABD25890A9D23E90FD0EA3
:1046C000F76EFC0EF66E20EED6F0F5EC65F013EC0E
:1046D00066F09DD23E92FD0EF76EEC0EF66E20EE69
:1046E000D6F0F5EC65F013EC66F091D221EC62F0B7
:1046F000A5EC62F0A06BA66BA76B53EC63F0A787E9
:1047000053EC63F0A78D53EC63F0E60EF76EBE0E2C
:10471000F66E20EED6F0F5EC65F009EC66F02EECC6
:104720005DF013EC66F0050EC06FC16BBF8F9E6B22
:10473000A0B11CD03DB03D9057B0ADEF23F057BCB9
:10474000AFEF23F058B0B4EF23F03DB4A9EF23F05E
:10475000EFD73D9423EC34F0EBD7579058D2579CC9
:10476000010E7063E5D753D265EF0FF0AFEC61F047
:10477000FCEC61F0230E9D5DD0E000EEE6F011EE62
:10478000D2F09DC0EEFF9DC0E6FF13EC66F09E2BBD
:10479000640EAE6F17C0ADF0A0B111D03DB03D902A
:1047A00057B019EF24F057BC1BEF24F058B020EF9E
:1047B00024F03DB415EF24F0AD67EED743D0FCEC08
:1047C00061F0230E9D6301D0A8D79E2B110E9E6130
:1047D00007D09DC0EEFF9DC0E6FF13EC66F0D8D772
:1047E000E7C0E6F0E8C0E7F0E9C0E8F0EAC0E9F0C9
:1047F000EBC0EAF0ECC0EBF0EDC0ECF0EEC0EDF099
:10480000EFC0EEF0F0C0EFF0F1C0F0F0F2C0F1F068
:10481000F3C0F2F0F4C0F3F0F5C0F4F09DC0EEFF89
:104820009DC0F5F013EC66F0B3D73D9423EC34F063
:10483000B3D75790ECD1579C010E7063ADD7E7D139
:1048400065EF0FF015EC30F0E86601D0CBD0809A20
:10485000358C640EAB6FAB67FED782AAA9EF21F04F
:10486000358EA66BA76B53EC63F0A68F53EC63F009
:10487000A78D53EC63F0A68D53EC63F0A78353EC44
:1048800063F0640EAE6F080EAD6FAD67FED79E6B22
:1048900001EED2F011EE78F0200EE76430D0040E75
:1048A000976FEF50E7622BD0EE50E650200EE76294
:1048B00001D002D0972FF5D797C09AF010EEE6F00E
:1048C000040E976F01EE78F00CAEAAEC2DF00CBE42
:1048D000EBEC2DF0E8665DD00F5009E0976F640EA9
:1048E000AE6F0A0EAD6FAD67FED7972FF8D701EE0A
:1048F000D2F09A510508E926E86AEA2204D001EECE
:10490000D2F010EEE6F0200E976F0CAEAAEC2DF070
:104910000CBEEBEC2DF0E8663CD0A66BA76B53EC1D
:1049200063F0A68753EC63F0A78D53EC63F0A68D7C
:1049300053EC63F0A78353EC63F0D3EF21F0808A4C
:10494000359C359EF90EF76E0E0EF66E20EED6F003
:10495000F5EC65F0F90EF76E1E0EF66E20EEE6F041
:10496000F5EC65F013EC66F03D903D92DF0EF76ECE
:10497000BE0EF66E23EE00F0EEEC65F0DE6ADFECC4
:1049800065F0640EAE6F140EAD6FAD67FED765EFC8
:104990000FF0808A359CF90EF76E9E0EF66E20EEB3
:1049A000D6F0F5EC65F0F90EF76EAE0EF66E20EE71
:1049B000E6F0F5EC65F013EC66F03D903D92DF0E0D
:1049C000F76EBE0EF66E23EE00F0EEEC65F0DE6ADA
:1049D000DFEC65F0640EAE6F140EAD6FAD67FED701
:1049E00065EF0FF0FD0EF76EAC0EF66E20EED6F012
:1049F000F5EC65F009EC66F09EC097F001EED2F0A0
:104A000010EEE6F0EECFE6FF972FFCD713EC66F042
:104A10003D903D92E30EF76E2A0EF66E23EE00F007
:104A2000EEEC65F0DE6ADFEC65F0640EAE6F320E20
:104A3000AD6F3DB029EF25F03DB22CEF26F057BC0D
:104A400025EF25F0AD67F5D7E2D0579C010E7063D6
:104A5000F0D703EE00F0410EEE6E540EEE6E440EF3
:104A6000EE6E9EC097F011EED2F0E6CFEEFF972FDC
:104A700035EF25F03B0EEE6E000EEE6E3D6A3E6A9F
:104A8000576A586ADFEC65F0FD0EF76EDC0EF66EC5
:104A900020EED6F0F5EC65F013EC66F03C0EBA6F44
:104AA00057B06EEF25F057BC70EF25F058B075EF9A
:104AB00025F058B277EF25F03DB279EF25F03DB003
:104AC0009BEF25F03EB07BEF25F03EB287EF25F05F
:104AD0003DB493EF25F0BA67E3D799D0579097D0BC
:104AE000579C010E7063DCD792D0589090D05892AA
:104AF000D7D73D928CD03E90FD0EF76EFC0EF66E31
:104B000020EED6F0F5EC65F013EC66F080D03E9226
:104B1000FD0EF76EEC0EF66E20EED6F0F5EC65F0BD
:104B200013EC66F074D03D94030E1E140208D8B442
:104B300023EC34F0B5D73D903D903D92E30EF76EF7
:104B4000420EF66E23EE00F0EEEC65F0DE6ADFEC6E
:104B500065F0FE0EF76E0C0EF66E20EED6F0F5EC5C
:104B600065F0A5EC62F0FCEC61F0A06B13EC66F074
:104B7000A0B113D057B0D3EF25F057BCDFEF25F02D
:104B800058B0D5EF25F03DB0D7EF25F03DB2D9EFC5
:104B900025F03DB4DBEF25F0EBD7FCEC61F0230E04
:104BA0009D63E6D715D0579032D0589030D03D90C5
:104BB000DFD73D9251D03D9423EC34F0D9D7579CA8
:104BC000010E706301D023D0579C020E7063D0D7C2
:104BD0001EAC1DD03D903D92E30EF76E360EF66E84
:104BE00023EE00F0EEEC65F0DE6ADFEC65F0640EBB
:104BF000AE6F320EAD6F3DB004EF26F03DB22CEF3C
:104C000026F0AD67F8D703D0388E76EF23F0FD0E8F
:104C1000F76EBC0EF66E20EED6F0F5EC65F0FD0EEC
:104C2000F76ECC0EF66E20EEE6F0F5EC65F03D90FA
:104C30003D92DF0EF76EBE0EF66E23EE00F0EEEC48
:104C400065F0DE6ADFEC65F0640EAE6F140EAD6FDA
:104C5000AD67FED765EF0FF0FE0EF76E1C0EF66E19
:104C600020EED6F0F5EC65F0FE0EF76E2C0EF66E2B
:104C700020EEE6F0F5EC65F013EC66F03D903D9229
:104C8000DF0EF76EBE0EF66E23EE00F0EEEC65F072
:104C9000DE6ADFEC65F0640EAE6F140EAD6FAD67CB
:104CA000FED765EF0FF0B8671FEF10F0400E976F5B
:104CB00014EEC0F0E76606D0E650972FFBD73B9680
:104CC0001FEF10F03B94E7B23B84E76A975140082E
:104CD000A26F9E6B15EE08F00A0EA203F350E126B8
:104CE000F450E222E7CF3CF02EEC5DF001EED2F082
:104CF00015EE00F00A0EA203F350E126F450E22272
:104D0000080ECB6F200E806FE7380F0B300F816FCE
:104D10003F0E816180C081F0080ECB6305D03B0E51
:104D2000816302D02B0E816F81C0EEFF200E815D6A
:104D300012E09E2BE6500F0B9A6F300F816F3F0EE3
:104D4000816180C081F081C0EEFF200E815F03E0B1
:104D50009E2BCB2FD9D71EC081F0030E8117020ED8
:104D6000816302EF23F03BB402D01EB6BAD015EC3B
:104D700030F0E86602D039B60AD0E70EF76E6E0E54
:104D8000F66E20EED6F0F5EC65F039960AD0E70E17
:104D9000F76E7E0EF66E20EED6F0F5EC65F03982F9
:104DA0003984E60EF76E7E0EF66E20EED6F0F5EC48
:104DB00065F013EC66F0388688EC30F0E86665EF55
:104DC0000FF0EEEC28F0E60EF76E9E0EF66E20EE7B
:104DD000D6F0F5EC65F0310E39B4320EE56F13EC18
:104DE00066F0640EAE6FFA0EAD6F3DB02EEF27F099
:104DF00057B00AEF27F057BC0CEF27F058B011EF6F
:104E000027F03EB013EF27F03EB220EF27F0AD675A
:104E1000ECD722D0579020D0579C010E7063E5D775
:104E20001BD0589019D03E90FD0EF76E6E0EF66EA8
:104E300020EED6F0F5EC65F013EC66F02CEF27F0E1
:104E40003E92FD0EF76E8E0EF66E20EED6F0F5EC6D
:104E500065F013EC66F000D018EF22F0388E3BA41A
:104E60009DEF20F01DEE00F0080EA203F350E126A6
:104E7000F450E2222EEC5DF09E6B01EED2F0080EB3
:104E8000CB6F200E806FE7380F0B300F816F3F0E16
:104E9000816180C081F081C0EEFF200E816512D05B
:104EA0009E2BE6500F0B9A6F300F816F3F0E816182
:104EB00080C081F081C0EEFF200E816503D09E2B63
:104EC000CB2FE1D71DEE00F0080EA203F350E12630
:104ED000F450E222080E976FE668972FFDD7ADEFEA
:104EE00020F0E70EF76E0E0EF66E20EED6F0F5EC23
:104EF00065F009EC66F013EC66F0809A358CA66BD1
:104F0000A76B53EC63F0A68F53EC63F0A68953ECC8
:104F100063F0A68353EC63F0320EAB6FAB67FED742
:104F200082AAD1EF28F0358E640EAE6F080EAD6FF9
:104F3000AD67FED79E6B01EED2F02B0EEF6202D072
:104F400001EED3F011EE70F0200EE76435D0080EBC
:104F5000976FEF50E76230D0EE50E650200EE762D8
:104F600001D002D0972FF5D797C09AF010EEE6F057
:104F7000040E976F01EE78F00CAEAAEC2DF00CBE8B
:104F8000EBEC2DF0E866F1D00F5009E0976F640E5E
:104F9000AE6F0A0EAD6FAD67FED7972FF8D701EE53
:104FA000D2F02B0EEF6202D001EED3F09A51090835
:104FB000E926E86AEA224AD001EED2F02B0EEF622F
:104FC00002D001EED3F011EE78F0200EE76435D078
:104FD000040E976FEF50E76230D0EE50E650200E8F
:104FE000E76201D002D0972FF5D797C09AF010EE64
:104FF000E6F0040E976F01EE78F00CAEAAEC2DF0FF
:105000000CBEEBEC2DF0E866B0D00F5009E0976FC6
:10501000640EAE6F0A0EAD6FAD67FED7972FF8D74F
:1050200001EED2F02B0EEF6202D001EED3F09A51D6
:105030000508E926E86AEA2209D001EED2F02B0E33
:10504000EF6202D001EED3F010EEE6F0200E976F83
:105050000CAEAAEC2DF00CBEEBEC2DF0E86685D082
:10506000A66BA76B53EC63F0A78953EC63F0A6879C
:1050700053EC63F0F6EC2EF016B40ED0140E6C6FF9
:105080001AC06DF03A903A923A863A94C56B80868F
:105090008094809280802BD016A012D055EC33F0F3
:1050A0002BEC2EF0140E6C6F1AC06DF03A903A9201
:1050B0003A863A94C56B808680948092808017D01F
:1050C000140E6C6F1AC06DF03A903A923A863A9488
:1050D000C56B80868094809280803AA4FED7640E4F
:1050E000AE6F060EAD6FAD67FED77CEC2EF0640E92
:1050F000B06FFA0EAF6F81B285EF28F0640EAB6F20
:10510000AB67FED781A2ACEF28F0AF67F4D7808AF7
:10511000359CA66BA76B53EC63F0F70EF76EBE0ED3
:10512000F66E20EED6F0F5EC65F0F70EF76ECE0ECB
:10513000F66E20EEE6F0F5EC65F013EC66F03A6AF8
:105140008086809480828090640EAE6F140EAD6F66
:10515000AB67FED765EF0FF03A6A80868094808255
:1051600080904EEC33F057EF16F0808A359CF90EA4
:10517000F76E9E0EF66E20EED6F0F5EC65F0F90EA9
:10518000F76EAE0EF66E20EEE6F0F5EC65F013EC81
:1051900066F0640EAE6F140EAD6FAD67FED765EFAF
:1051A0000FF0808A359C359EF90EF76E0E0EF66E66
:1051B00020EED6F0F5EC65F0F90EF76E1E0EF66EE9
:1051C00020EEE6F0F5EC65F013EC66F0640EAE6FE1
:1051D000140EAD6FAD67FED765EF0FF009EC66F00A
:1051E0009E6B11EED2F003EE00F0410EEE6E540E07
:1051F000EE6E440EEE6E200E976FE750200804E02E
:10520000E6CFEEFF972FF9D73B0EEE6E000EEE6E57
:1052100000EEE6F011EED2F0100E976FE750200886
:1052200004E0E6CFEEFF972FF9D713EC66F03D9040
:105230003D923E6A57905794579A579C5890DFEC8E
:1052400065F01200140E976F00EE43F0426AEF66AD
:1052500007D0422AEE50972FFAD7389A65EF0FF011
:10526000EF6A200E976F08EE32F0200EEE6E972F49
:10527000FCD73F9E42C084F059EC61F03D903D92D6
:1052800003EE00F0410EEE6E540EEE6E2B0EEE6E3F
:10529000430EEE6E4D0EEE6E470EEE6E520EEE6E3D
:1052A0003D0EEE6E300E7F637FC0EEFF806380C0E8
:1052B000EEFF81C0EEFF000EEE6EDFEC65F0640ED7
:1052C000AE6FFA0EAD6F3DB07EEF29F03DB26BEFE1
:1052D00029F0AD67F8D73D92F90EF76EDE0EF66E47
:1052E00020EEE6F0F5EC65F013EC66F0640EAE6FC0
:1052F0001E0EAD6FAD67FED765EF0FF03D902EA08F
:10530000EED018EE52F0430EE6626CD0620EE6620A
:10531000A5D2120E976F01EEB0F0200EEE6E972F11
:10532000FCD7000EE7620BD0120E976F18EE32F02A
:1053300001EEB0F0E6CFEEFF972FFCD70BD0100EAA
:10534000976F01EEB0F0000EE75C04E0E6CFEEFFF1
:10535000972FF9D75BEC2DF03BA09BD23CA414D047
:105360001E50030B020828E13B8614EEC0F0A25148
:10537000E126E86AE222E768640EB96F140EB86F9E
:1053800020EC2DF065EF0FF0FA0EF76E3E0EF66E84
:1053900020EEE6F0F5EC65F000EED6F011EEB0F0A0
:1053A000100E976FE6CFEEFF972FFCD713EC66F049
:1053B00020EC2DF065EF0FF0FE0EF76EDC0EF66EB2
:1053C00020EED6F0F5EC65F0FE0EF76EEC0EF66E04
:1053D00020EEE6F0F5EC65F013EC66F020EC2DF035
:1053E00065EF0FF02EA27BD0120E976F08EE00F043
:1053F00011EEB0F0200EEE6EE66E972FFBD718EE92
:1054000052F0530EE6626BD0630EE66227D2000EB6
:10541000E75CD8B423D2100E976F08EE00F02E0E82
:10542000E75C07E0000EE75C04E0E6CFEEFF972FB5
:10543000F6D7000EE7620BD0120E976F18EE32F01F
:1054400001EEB0F0E6CFEEFF972FFCD711D02E0E75
:10545000E66204D2000EE75CEFE0100E976F01EEFB
:10546000B0F0000EE75C04E0E6CFEEFF972FF9D72F
:105470003C6A5BEC2DF03BA00CD23CA485D71E50BF
:10548000030B020899E13B8614EEC0F0A251E1261D
:10549000E86AE222020EE76E1DEE00F0080EA2039B
:1054A000F350E126F450E222080ECB6F08EE00F034
:1054B000200EEF64EF68EE38F00B816F200EEF6482
:1054C000EF680F0EEE148111E66ECB2FF1D7640E4C
:1054D000B96F140EB86F20EC2DF065EF0FF02EB4FD
:1054E0001CD0FC0EF76E8E0EF66E20EED6F0F5ECAC
:1054F00065F0FC0EF76E9E0EF66E20EEE6F0F5EC13
:1055000065F013EC66F020EC2DF0640EAE6F140E17
:10551000AD6FAD67FED765EF0FF001EE2EF0200EF8
:10552000EF5C19E0100E976F01EE2EF018EE32F0DE
:105530002B0EE76202D018EE33F0EE50E6620BD08D
:10554000972FFBD7100E976F01EEB0F0200EEE6E86
:10555000972FFCD712D02EA810D0100E976F01EE07
:105560001CF018EE32F02B0EE76202D018EE33F08A
:10557000EE50E66285D1972FFBD7080E976F01EEAC
:105580000CF018EE52F0200EEF6202D0EE5005D073
:10559000EE50E6625AD1972FF6D7100E976F01EEB4
:1055A000B0F0200EEE6E972FFCD72E0EE66256D18D
:1055B000410EE6629DD0640EE66299D0640EE6620A
:1055C00095D02E0EE66291D0100E976F01EEB0F0DE
:1055D0002E0EE75C04E0E6CFEEFF972FF9D72E0EF4
:1055E000E6623CD13C6A590EE76202D03C8004D0AE
:1055F0004E0EE76233D13C90E6502E0EE6622ED17D
:10560000590EE76202D03C8204D04E0EE76226D1EA
:105610003C92E6502E0EE66221D1590EE76202D08E
:105620003C8404D04E0EE76219D13C94E6502E0E15
:10563000E66214D1590EE76202D03C8604D04E0EC9
:10564000E7620CD13C96E6502E0EE66207D1590E69
:10565000E76202D03C8804D04E0EE762FFD03C984F
:105660005BEC2DF03BA00BD015EE08F00A0EA20368
:10567000F350E126F450E2223CC0E7FF21D096EC43
:105680002DF03BA0F4D015EE00F00A0EA203F3506B
:10569000E126F450E222080ECB6F01EEB0F0200EAE
:1056A000EF64EF68EE38F00B816F200EEF64EF6867
:1056B0000F0EEE148111E66ECB2FF1D73CC0E6FF42
:1056C00005EE00F00A0EA203F350E926F450EA2298
:1056D000010EAA6E200EA96EF350A926F450AA223C
:1056E0000A0ECB6FC6EC65F0E9D0E106E106E106F3
:1056F000E106430EE66243D06C0EE6623FD0720EC6
:10570000E6623BD02E0EE66237D0100E976F01EEA8
:10571000B0F0000EE75C07E02E0EE75C04E0E6CF99
:10572000EEFF972FF6D75BEC2DF03BA0B2D015EE35
:1057300000F00A0EA203F350E126F450E222080E14
:10574000CB6FFF0EE66ECB2FFCD7E66AE66805EE60
:1057500000F00A0EA203F350E926F450EA22010EEB
:10576000AA6E200EA96EF350A926F450AA220A0EA2
:10577000CB6FC6EC65F0A2D0E106E106E106E106DA
:10578000460EE6626BD06C0EE66268D06D0EE66285
:1057900065D02E0EE66262D0100E976F01EEB0F06B
:1057A0002E0EE75C0AE02F0EE76458D03A0EE76051
:1057B00055D0E6CFEEFF972FF3D72E0EE6624ED0F0
:1057C0003C6A590EE76202D03C6804D04E0EE76294
:1057D00045D03C6AE6502E0EE66240D02F0EE764BC
:1057E0003DD03A0EE7603AD0E6CF9AF00F0E9A1706
:1057F000100E976F11EEB0F001EE50F0E6CFEEFF15
:10580000972FFCD7FC0E0C16020E3C660C129AC0A9
:105810000EF0030EAA6E9E0E100ECB6F05EE00F07A
:10582000C6EC65F0030EAA6E020E00EE0EF0010E3D
:10583000CB6FC6EC65F0030EAA6E000E00EE0CF006
:10584000010ECB6FC6EC65F039D0F90EF76EEE0E97
:10585000F66E20EEE6F0F5EC65F023D0F90EF76E6B
:10586000FE0EF66E20EEE6F0F5EC65F01AD0FA0EBC
:10587000F76E0E0EF66E20EEE6F0F5EC65F011D048
:10588000FA0EF76E1E0EF66E20EEE6F0F5EC65F001
:1058900008D0FA0EF76E2E0EF66E20EEE6F0F5EC5E
:1058A00065F03F8E00EED6F011EEB0F0100E976F5F
:1058B000E6CFEEFF972FFCD713EC66F020EC2DF02F
:1058C0002EA665EF0FF03D903D9203EE00F0410EE5
:1058D000EE6E540EEE6E2B0EEE6E430EEE6E4D0E11
:1058E000EE6E470EEE6E530EEE6E3D0EEE6E220E17
:1058F000EE6E200E976F18EE32F0200EE75C04E09B
:10590000E6CFEEFF972FF9D7220EEE6EEE6ADFECB0
:1059100065F0640EAE6F320EAD6F3DB295EF2CF0B8
:105920003FB297EF2CF0AD67F8D73D926FD03F9222
:1059300003EE00F0530EEE6E4D0EEE6E530EEE6E55
:10594000200EEE6E530EEE6E650EEE6E740EEE6E63
:10595000750EEE6E700EEE6E200EEE6E2F0EEE6E6B
:10596000400E976F18EE52F0000EE75C04E0E6CFB1
:10597000EEFF972FF9D72F0EEE6E200EEE6E770EFC
:10598000EE6E610EEE6E730EEE6E200EEE6E3FAE9C
:105990000DD0660EEE6E610EEE6E690EEE6E6C0E42
:1059A000EE6E650EEE6E640EEE6E12D0730EEE6E3F
:1059B000750EEE6E630EEE6EEE6E650EEE6E730E8F
:1059C000EE6EEE6E660EEE6E750EEE6E6C0EEE6E9A
:1059D0001A0EEE6EEE6A3D903D923F94DFEC65F05C
:1059E000640EAE6F320EAD6F3DB2FFEF2CF03DB0E6
:1059F00003EF2DF03FB401EF2DF0AD67F5D73D92E9
:105A000005D03F94F1D73D9065EF0FF0FB0EF76E98
:105A1000CE0EF66E20EED6F0F5EC65F0FB0EF76ECE
:105A2000DE0EF66E20EEE6F0F5EC65F013EC66F0B7
:105A3000640EAE6F140EAD6FAD67FED765EF0FF05D
:105A4000640EB06F140EAF6F42C084F059EC61F079
:105A50003D903D9203EE00F0410EEE6E540EEE6E60
:105A60002B0EEE6E430EEE6E4D0EEE6E470EEE6E8C
:105A7000440EEE6E3D0EEE6E300E7F637FC0EEFF85
:105A8000806380C0EEFF81C0EEFF000EEE6EDFECA3
:105A900065F0640EAE6FFA0EAD6F3DB057EF2DF0AE
:105AA0003DB255EF2DF0AD67F8D73D9201D03D9056
:105AB000AF67FED71200A26B3B9015EE00F00A0E06
:105AC000A203F350E126F450E22201EEB0F0FF0E03
:105AD000E76026D0080ECB6FE7380F0B300F806FD2
:105AE000080ECB6305D03B0E806302D02B0E806F77
:105AF000E6500F0B300F816F200E9A6F3F0E8061C2
:105B00009AC080F081619AC081F0EE50806308D025
:105B1000EE50816305D0CB2FDFD73C843B80120051
:105B2000A22B400EA263C9D73B901200A26B15EEC8
:105B300000F00A0EA203F350E126F450E222FF0E19
:105B4000E76202D03B801200A22B3F0EA265EFD786
:105B50003B901200640EAB6FAB67FED7EECF9DF0AB
:105B6000200E9D5DD8B436D005EC5DF0EFEC61F011
:105B7000640EAB6FAB67FED7AFEC61F0110E9E61A8
:105B800003D09DC0E6FF20D0E7C0E6F0E8C0E7F014
:105B9000E9C0E8F0EAC0E9F0EBC0EAF0ECC0EBF0F5
:105BA000EDC0ECF0EEC0EDF0EFC0EEF0F0C0EFF0C5
:105BB000F1C0F0F0F2C0F1F0F3C0F2F0F4C0F3F095
:105BC000F5C0F4F09DC0F5F013EC66F0974F02D0ED
:105BD0009E2BC0D7000C640EAE6F050EAD6FAD6787
:105BE000FED7EECF9DF0200E9D5D33E0EFEC5CF034
:105BF0000B0E9F612FD032EC18F0110E9E6103D076
:105C00009DC0E6FF20D0E7C0E6F0E8C0E7F0E9C0BD
:105C1000E8F0EAC0E9F0EBC0EAF0ECC0EBF0EDC070
:105C2000ECF0EEC0EDF0EFC0EEF0F0C0EFF0F1C040
:105C3000F0F0F2C0F1F0F3C0F2F0F4C0F3F0F5C010
:105C4000F4F09DC0F5F013EC66F0974F02D09E2B58
:105C5000C2D7000CFF0CC80EAB6FAB67FED7640E4B
:105C6000AB6FE8EC61F0AB67FED7AFEC61F03C0ED8
:105C7000AB6FAB67FED7110ECE6F000ECF6FD0ECBF
:105C800062F0300ECE6F180ECF6FD5EC62F0960E2C
:105C9000AB6FAB67FED7300ECE6F160ECF6FD5EC65
:105CA00062F03C0EAB6FAB67FED7110ECE6F480EA5
:105CB000CF6FD0EC62F081B0FED7E9EC62F004EE79
:105CC00000F0EECFCEF0DFEC62F081B0FED7E9EC71
:105CD00062F081B0FED7E9EC62F0CB2FF2D7110E63
:105CE000CE6F000ECF6FD0EC62F0F5EC61F0FA0EE3
:105CF000AB6FAB67FED71200110ECE6F000ECF6FE9
:105D0000D0EC62F0300ECE6F180ECF6FD5EC62F093
:105D1000FA0EAB6FAB67FED7300ECE6F160ECF6F9D
:105D2000D5EC62F0960EAB6FAB67FED7110ECE6F5F
:105D3000480ECF6FD0EC62F081B0FED7E9EC62F094
:105D400004EE00F0EECFCEF0DFEC62F081B0FED7D3
:105D5000E9EC62F081B0FED7E9EC62F0CB2FF2D72C
:105D6000110ECE6F000ECF6FD0EC62F0F5EC61F04B
:105D70001200110ECE6F000ECF6FD0EC62F0500EFD
:105D8000CE6F180ECF6FD5EC62F0FA0EAB6FAB672B
:105D9000FED7500ECE6F160ECF6FD5EC62F0960E7A
:105DA000AB6FAB67FED7110ECE6F480ECF6FD0EC46
:105DB00062F081B0FED7E9EC62F004EE00F0EECFC5
:105DC000CEF0DFEC62F081B0FED7E9EC62F081B09A
:105DD000FED7E9EC62F0CB2FF2D7110ECE6F000E9A
:105DE000CF6FD0EC62F0F5EC61F01200CB6B04EEFB
:105DF00000F0800EEE6E000EEE6E020EEE6E000EE5
:105E0000EE6E11EE8CF0200EE76205D0500EEE6EB5
:105E1000010ECB270AD0100E976F200EE75C05E02D
:105E2000CB2BE6CFEEFF972FF8D7CBC003F4020EB3
:105E3000CB27CBC001F4020ECB27CBC097F004EEEA
:105E400000F0C86BEE50C827972F22EF2FF0C81F25
:105E5000010EC827C8C0EEFFCB2B1200376A100E08
:105E6000976F01EEC2F0200EEE6E972FFCD708EE72
:105E700052F0500E976FEE6A972F3BEF2FF0E9EC40
:105E800062F0E4EC62F03E0ECE6F160ECF6FDAECED
:105E900062F0110ECE6F420ECF6FD0EC62F0640E46
:105EA000B06F140EAF6FAF51D8B49AD081B0FBD79A
:105EB000E9EC62F0CEC09AF0E4EC62F09AA3F3D77A
:105EC000AF51D8B48DD081B0FBD7E9EC62F0CFC030
:105ED0009AF0E4EC62F09AAFF3D73E0ECE6F360E36
:105EE000CF6FDAEC62F0110ECE6F410ECF6FD0ECB7
:105EF00062F0C86BCB6B08EE52F0AF5171E081B02D
:105F0000FCD7E9EC62F0E4EC62F0CEC0EEFFCE51DB
:105F1000C827CB2BAF5164E081B0FCD7E9EC62F02D
:105F2000E4EC62F0CEC0EEFFCEC097F0CE51C827B1
:105F3000CB27CB2B97510FE0AF5152E081B0FCD76C
:105F4000E9EC62F0E4EC62F0CEC0EEFFCE51C8277F
:105F5000972F9CEF2FF0AF5143E081B0FCD7E9ECD5
:105F600062F0E4EC62F0CEC0EEFFCE51C827CB2B3E
:105F7000110ECE6F000ECF6FD0EC62F0C8672BD041
:105F800018EE52F0800EE66226D0E6CF97F0020EB1
:105F9000E76214D0E650E6CFCBF0500EE7601DD09C
:105FA000CB5119E0100ECB6501D0CB6F01EEC2F0E2
:105FB000E6CFEEFFCB2FFCD737801200040EE7624E
:105FC00001D00BD0E650E6CFCBF0E650974F03D090
:105FD000CB2FFBD7DCD737841200378237801200F3
:105FE000FAD7120037A016D037B20BD0100E976F29
:105FF00011EEC2F000EEE6F0E6CFEEFF972FFCD7F1
:1060000011D0E60EF76EEE0EF66E20EEE6F0F5EC31
:1060100065F008D0E60EF76EFE0EF66E20EEE6F0A6
:10602000F5EC65F013EC66F0120004EE40F0200E83
:10603000976F8B6BFF0EEF5C58E0EF380F0B7A6FAA
:10604000EE500F0B7B6FEF380F0B7C6FEE500F0B8A
:106050007D6FEF380F0B7E6FEE500F0B7F6FEF38B9
:106060000F0B806FEE500F0B816F0F0E815D3DE0C7
:106070000A0E7A6303D0FA0E7A6F05D00B0E7A639C
:1060800002D0FB0E7A6F300E7A277B277C277D2784
:106090007E277F27802711EED2F07A51E66225D045
:1060A0003F0E7B5D30E07B51E6621FD03F0E7C5D92
:1060B0002AE07C51E66219D03F0E7D5D24E07D51DF
:1060C000E66213D03F0E7E5D1EE07E51E6620DD08B
:1060D0003F0E7F5D18D07F51E66207D03F0E805D96
:1060E00012D08051E66201D00ED08B2B040E8B03B0
:1060F000F35004EE40F0E926E86AEA22972F1AEFFF
:1061000030F03996FF0C3996010E81633986000C08
:1061100039B607D039B202D038B2AED239923994FA
:1061200002D0398400D03892399239905790640E59
:10613000AE6F140EAD6F57B0A0EF30F0AD67FBD768
:106140005790389239B4838C39A4839C3D6A576A3E
:10615000586A596A39803D903D92E00EF76E9A0E6A
:10616000F66E23EE00F0EEEC65F0DE6ADFEC65F033
:10617000640EAE6F320EAD6F3DB0C7EF30F03DB282
:10618000C5EF30F0AD67F8D73AD03D9238D03D90AA
:10619000640EB06FFA0EAF6F57B0FEEF31F057B22A
:1061A00016EF32F057B667EF32F059B0A6EF32F083
:1061B00059B2A9EF32F059B40FEF33F059B611EFDD
:1061C00033F059B825EF33F059BA39EF33F03DB217
:1061D00012EF31F0AF67E0D7E50EF76E0E0EF66EF8
:1061E00020EED6F0F5EC65F0E50EF76E1E0EF66EBD
:1061F00020EEE6F0F5EC65F013EC66F040D2F90E17
:10620000F76E5E0EF66E20EED6F0F5EC65F0F90E48
:10621000F76E6E0EF66E20EEE6F0F5EC65F013EC20
:1062200066F02DD23D923DB812D00A0E405CD8B433
:10623000A3D00B0E405C58E00C0E405C42E00D0E0B
:10624000405C2BE0100E405CD8B4B2D000D0F80E09
:10625000F76E8E0EF66E20EED6F0F5EC65F0F80EC9
:10626000F76E9E0EF66E20EEE6F0F5EC65F010EEA1
:10627000EEF0826B40C083F075EC61F0350E3DB8F6
:106280007F6F300E7F637FC0E6FF806380C0E6FFD4
:1062900081C0E6FF13EC66F0F2D1F90EF76E3E0E08
:1062A000F66E20EED6F0F5EC65F0F90EF76E4E0EB8
:1062B000F66E20EEE6F0F5EC65F013EC66F000000B
:1062C000DED1F80EF76E6E0EF66E20EED6F0F5EC1F
:1062D00065F0F80EF76E7E0EF66E20EEE6F0F5EC49
:1062E00065F013EC66F0CBD111EE40F039B411EE4D
:1062F00048F0200EE75CD8B46ED003EE00F0410EFB
:10630000EE6E540EEE6E2B0EEE6E430EEE6E500ED3
:10631000EE6E490EEE6E4E0EEE6E3D0EEE6E080EF9
:10632000976F200EE75C05E0E6CFEEFF972F91EF29
:1063300031F0000EEE6E3D903D92DFEC65F0640EA4
:10634000AE6F320EAD6F3DB0ACEF31F03DB2AEEF9F
:1063500031F0AD67F8D7A1D73D901ED73D923DB83B
:1063600076D70A0E405C08E00C0E405CD8B4A9D782
:10637000100E405C1DE06BD73D92E40EF76EAE0E42
:10638000F66E20EED6F0F5EC65F0E40EF76E9E0E9C
:10639000F66E20EEE6F0F5EC65F0310E39B4320E13
:1063A000F06F39A4399C39B4399E13EC66F067D18B
:1063B000F80EF76E5E0EF66E20EED6F0F5EC65F098
:1063C000F90EF76E2E0EF66E20EEE6F0F5EC65F0A7
:1063D00013EC66F054D1F80EF76E0E0EF66E20EE4A
:1063E000D6F0F5EC65F0F80EF76E1E0EF66E20EEA8
:1063F000E6F0F5EC65F013EC66F041D15790E40E51
:10640000F76E4E0EF66E20EED6F0F5EC65F0E40E6B
:10641000F76E6E0EF66E20EEE6F0F5EC65F0310EDE
:1064200039B4320EDC6F13EC66F029D157923D90EF
:106430003D923D983D903D92E10EF76E820EF66ED4
:1064400023EE00F0EEEC65F0DE6ADFEC65F0640E42
:10645000AE6F320EAD6F3DB045EF32F03DB237EF6B
:1064600032F03DBC47EF32F0AD67F5D7C8D63DA856
:1064700093D63D983D920F0E4062C1D6640EAE6F2A
:10648000050EAD6FAD67FED7D5D73D9085D63D9C47
:10649000000E6F6301D080D6010E6F6301D024D748
:1064A000020E6F6301D00DD7F90EF76E7E0EF66EF9
:1064B00020EED6F0F5EC65F0F90EF76E8E0EF66E66
:1064C00020EEE6F0F5EC65F013EC66F0D8D05796C8
:1064D0003D903D923D903D92E00EF76EBE0EF66E01
:1064E00023EE00F0EEEC65F0DE6ADFEC65F0640EA2
:1064F000AE6F320EAD6F3DB086EF32F03DB284EF3D
:1065000032F0AD67F8D77BD63D9279D63D903D927B
:106510003D903D92DF0EF76ECA0EF66E23EE00F050
:10652000EEEC65F0DE6ADFEC65F0640EAE6F320E05
:10653000AD6F3DB0A4EF32F03DB2A2EF32F0AD67E7
:10654000F8D75DD63D925BD63D9026D659903892CD
:1065500023D65992388238A68FD038961E389A6F33
:10656000030E9A17000E9A630ED03D903D92DF0EF7
:10657000F76EEE0EF66E23EE00F0EEEC65F0DE6ADE
:10658000DFEC65F01ED0010E9A630ED03D903D9277
:10659000DF0EF76EFA0EF66E23EE00F0EEEC65F00D
:1065A000DE6ADFEC65F00DD03D903D92E00EF76EB7
:1065B000060EF66E23EE00F0EEEC65F0DE6ADFEC20
:1065C00065F0640EAE6F320EAD6F3DB0F1EF32F09C
:1065D0003DB2EEEF32F0AD67F8D74ED03D923DA818
:1065E0004BD03D903D903D92E00EF76ED60EF66E8C
:1065F00023EE00F0EEEC65F0DE6ADFEC65F0640E91
:10660000AE6F320EAD6F3DB00DEF33F03DB20BEF1C
:1066100033F0AD67F8D73D922FD03D902DD05994EF
:10662000BBD55996E40EF76ECE0EF66E20EED6F080
:10663000F5EC65F0E40EF76E8E0EF66E20EEE6F0E9
:10664000F5EC65F013EC66F01AD05998E40EF76E8D
:10665000EE0EF66E20EED6F0F5EC65F0E40EF76E79
:106660008E0EF66E20EEE6F0F5EC65F013EC66F0BB
:1066700006D0599A388200D0000C3D92C0D5060E43
:10668000C06FC16BBF8F640EAE6F320EAD6FAD6762
:10669000FED7AFEC61F034923490EE0C000E18622D
:1066A00001D01200010E1862120080868084808260
:1066B00080901200000E186201D01200010E1862C4
:1066C00004D08086809480828090020E18620FD061
:1066D0008086808480828090640EAE6F19C0ADF099
:1066E000AD67FED780868094808280901200030E72
:1066F000186212008096809480928090640EAE6F33
:1067000019C0ADF0AD67FED78086809480828090FE
:106710001200A26B3B90E00E3C1611EE8CF0200EA6
:10672000E76201D0120015EE00F00A0EA203F3504A
:10673000E126F450E22201EE8CF0FF0EE7602FD04C
:10674000080ECB6FE7380F0B300F806F080ECB634E
:1067500005D03B0E806302D02B0E806FE6500F0BEE
:10676000300F816F200E9A6F3F0E80619AC080F0CB
:1067700081619AC081F0EE50806311D0EE50816348
:106780000ED0CB2FDFD7E7B03C80E7B23C82E7B436
:106790003C84E7B63C86E7B83C883B801200A22BDD
:1067A000400EA263C0D73B901200A26B3B90F00E4C
:1067B0003C1611EE9EF0200EE76201D0120015EE9D
:1067C00000F00A0EA203F350E126F450E22201EE9B
:1067D0009EF0FF0EE76031D0080ECB6FE7380F0B4D
:1067E000300F806F080ECB6305D03B0E806302D064
:1067F0002B0E806FE6500F0B300F816F200E9A6FBB
:106800003F0E80619AC080F081619AC081F0EE50A5
:10681000806313D0EE50816310D0CB2FDFD73B8045
:10682000E7A412003C843B8614EEC0F0A251E1269E
:10683000E86AE222010EE76E1200A22B400EA2636C
:10684000BED73B901200A26B3B90F00E3C1611EEAF
:106850009EF0200EE76201D0120015EE00F00A0E45
:10686000A203F350E126F450E22201EE9EF0FF0E67
:10687000E76031D0080ECB6FE7380F0B300F806F19
:10688000080ECB6305D03B0E806302D02B0E806FC9
:10689000E6500F0B300F816F200E9A6F3F0E806114
:1068A0009AC080F081619AC081F0EE50806313D06D
:1068B000EE50816310D0CB2FDFD7E7A612003C86C5
:1068C0003B803B8614EEC0F0A251E126E86AE2224A
:1068D000010EE76E1200A22B400EA263BED73B90C2
:1068E00012003990020EAB6FAB67FED7839C020E8D
:1068F000AB6FAB67FED783AE398C83BE399C120079
:106900003990020EAB6FAB67FED7838C020EAB6F74
:10691000AB67FED783AE398E83BE399E1200C80E98
:10692000AB6FAB67FED7050EEFEC61F0640EAB6F9B
:10693000AB67FED7AFEC61F0640EAB6FAB67FED711
:10694000050EEFEC61F0640EAB6FAB67FED7AFECFA
:1069500061F01200C80EAB6FAB67FED7050EEFEC0F
:1069600061F0FA0EAB6FAB67FED7AFEC61F0640E6F
:10697000AB6FAB67FED7050EEFEC61F0FA0EAB6FB5
:10698000AB67FED7AFEC61F0120038903492E60EA0
:10699000F76E1E0EF66E20EED6F0F5EC65F009EC03
:1069A00066F013EC66F02EEC5DF09E6B716B8FEC75
:1069B00034F001EED2F010EEE6F081B265EF0FF0A8
:1069C000A0B1E4EF34F0F9D7FCEC61F0230E9D5D4B
:1069D00075E09E2B200E9E659DC0EEFF2A0E9A6FDD
:1069E000100E9E659AC0E6FF13EC66F0DDEF34F002
:1069F00001EED2F0300EEE6253D0300EEE6250D087
:106A0000310EEE624DD0310EEE624AD0320EEE62A1
:106A100047D0320EEE6244D0330EEE6241D0330ED8
:106A2000EE623ED001EE00F0300EEE6EEE6EEE6ED7
:106A3000EE6E01EE0CF0310EEE6E320EEE6E330E97
:106A4000EE6E340EEE6E350EEE6E360EEE6E370EC8
:106A5000EE6E380EEE6E01EE14F0310EEE6E320E6A
:106A6000EE6E330EEE6E340EEE6E350EEE6E360EAC
:106A7000EE6E370EEE6E380EEE6E01EE04F0340E52
:106A8000EE6E320EEE6E330EEE6E380EEE6E360E8B
:106A9000EE6E370EEE6E380EEE6E330EEE6E22D0C8
:106AA000E60EF76E2E0EF66E20EED6F0F5EC65F0E3
:106AB00009EC66F013EC66F054EF14F0040E9E63DC
:106AC0000DD001EED2F011EE00F0040E976FEE50F3
:106AD000E662E6D7972F67EF35F010D0080E9E6379
:106AE000DFD786D78FEC34F0716B640EAE6F0F0E6C
:106AF000AD6FAD67FED781B2ECEF5BF0000E716356
:106B000013D0E70EF76E9E0EF66E20EED6F0F5EC83
:106B100065F0E70EF76EAE0EF66E20EEE6F0F5ECE1
:106B200065F013EC66F05AD0010E716313D0E70ED6
:106B3000F76EBE0EF66E20EED6F0F5EC65F0E70EC1
:106B4000F76ECE0EF66E20EEE6F0F5EC65F013EC87
:106B500066F044D0020E716313D0E70EF76EDE0EBE
:106B6000F66E20EED6F0F5EC65F0E70EF76EEE0E61
:106B7000F66E20EEE6F0F5EC65F013EC66F02ED044
:106B8000030E716313D0E70EF76EFE0EF66E20EE65
:106B9000D6F0F5EC65F0E80EF76E0E0EF66E20EE10
:106BA000E6F0F5EC65F013EC66F018D0040E7163B6
:106BB00013D0E80EF76E1E0EF66E20EED6F0F5EC52
:106BC00065F0E80EF76E2E0EF66E20EEE6F0F5ECB0
:106BD00065F013EC66F002D0716B90D781B2ECEFE8
:106BE0005BF0A0B1F5EF35F0F9D7FCEC61F0230EC6
:106BF0009D631BD0000E716302D063EF57F0010E4E
:106C0000716302D0D4EF49F0020E716302D02DEF10
:106C100044F0030E716302D098EF39F0040E7163F3
:106C200002D01DEF36F0716B69D72A0E9D6366D7CF
:106C3000712B050E7161716B61D78FEC34F0640EAE
:106C4000AE6F0F0EAD6FAD67FED781B2ECEF5BF0AC
:106C5000FA0EF76E4E0EF66E20EED6F0F5EC65F0FD
:106C6000FA0EF76E5E0EF66E20EEE6F0F5EC65F0CD
:106C700013EC66F081B272EF35F0A0B141EF36F05F
:106C8000F9D7FCEC61F0230E9D63C6EF38F0FA0EE5
:106C9000F76E8E0EF66E20EED6F0F5EC65F0FA0E7D
:106CA000F76E9E0EF66E20EEE6F0F5EC65F013EC56
:106CB00066F02EEC5DF09E6B81B21FEF36F0A0B156
:106CC00081EF36F0F9D70F0E9A6F100E9E619AC0C1
:106CD0009EF09E5111EED2F09DC0E3FF00EEEEF06B
:106CE000070E9A6F9EC097F0080E9E619AC097F0AB
:106CF0002A0E9A6F97519AC0EBFF13EC66F09E2B09
:106D0000DBD7FCEC61F0230E9D63DDD7080E9E639C
:106D10000AD001EE14F011EED2F0EE50E66203D08C
:106D20009E2FFBD71CD0FA0EF76EAE0EF66E20EE3D
:106D3000D6F0F5EC65F0FA0EF76EBE0EF66E20EEAC
:106D4000E6F0F5EC65F013EC66F0AAEC34F0640EB6
:106D5000AE6F140EAD6FAD67FED772EF35F0FB0E60
:106D6000F76E0E0EF66E20EED6F0F5EC65F02EB452
:106D700009D0FB0EF76E1E0EF66E20EEE6F0F5EC77
:106D800065F008D0FB0EF76E2E0EF66E20EEE6F0E4
:106D9000F5EC65F013EC66F081B21FEF36F0A0B1B0
:106DA000D3EF36F0F9D7FCEC61F02A0E9D6302D0E8
:106DB0002E74D5D7230E9D63EFD7FB0EF76E4E0EC4
:106DC000F66E20EED6F0F5EC65F02EB609D0FB0E8F
:106DD000F76E5E0EF66E20EEE6F0F5EC65F008D08C
:106DE000FB0EF76E6E0EF66E20EEE6F0F5EC65F03B
:106DF00013EC66F081B21FEF36F0A0B101EF37F06F
:106E0000F9D7FCEC61F02A0E9D6302D02E76D5D71F
:106E1000230E9D63EFD7FB0EF76E7E0EF66E20EE0F
:106E2000D6F0F5EC65F02EB809D0FB0EF76E8E0E9D
:106E3000F66E20EEE6F0F5EC65F008D0FB0EF76E8E
:106E40009E0EF66E20EEE6F0F5EC65F013EC66F0C3
:106E500081B21FEF36F0A0B12FEF37F0F9D7FCEC7D
:106E600061F02A0E9D6302D02E78D5D7230E9D6344
:106E7000EFD7FB0EF76EEE0EF66E20EED6F0F5ECC9
:106E800065F0100E976F00EEE6F011EE1CF0E6CF05
:106E9000EEFF972FFCD713EC66F09E6B81B280EF6C
:106EA00037F0A0B155EF37F0F9D7FCEC61F02A0EBE
:106EB0009D6306D009EC66F013EC66F09E6BEED78E
:106EC000230E9D630BD0100E976F10EEE6F001EECF
:106ED0001CF0E6CFEEFF972FFCD71ED09E6704D0A4
:106EE00009EC66F010EEE6F0100E9E619E690F0E42
:106EF0009E179E519DC0E3FF13EC66F09E2BCED7EC
:106F0000100E976F10EEE6F001EE1CF0E6CFEEFFEC
:106F1000972FFCD71FEF36F0FB0EF76EFE0EF66EC6
:106F200020EED6F0F5EC65F009EC66F0080E976FF0
:106F300000EEE6F011EE0CF0E6CFEEFF972FFCD757
:106F400013EC66F09E6B81B2CCEF37F0A0B1AAEFE4
:106F500037F0F9D7FCEC61F02A0E9D6308D009ECFC
:106F600066F010EEE6F013EC66F09E6BECD7230EA5
:106F70009D5D1DE09E6704D009EC66F010EEE6F022
:106F8000080E9E619E690F0E9E179E519DC0E3FFE5
:106F90009E2B13EC66F0D7D7080E976F10EEE6F035
:106FA00001EE0CF0E6CFEEFF972FFCD748D6080E87
:106FB000976F10EEE6F001EE0CF0E6CFEEFF972FA4
:106FC000FCD7FC0EF76E0E0EF66E20EED6F0F5EC4A
:106FD00065F009EC66F013EC66F09E6B81B21FEF72
:106FE00036F0A0B1F5EF37F0F9D7FCEC61F02A0EDE
:106FF0009D6325D6FC0EF76E1E0EF66E20EED6F0C3
:10700000F5EC65F0FC0EF76E2E0EF66E20EEE6F057
:10701000F5EC65F013EC66F02EEC5DF09E6B81B242
:107020001FEF36F0A0B134EF38F0F9D70F0E9A6F9A
:10703000100E9E619AC09EF09E5111EED2F09DC03E
:10704000E3FF00EEEEF0070E9A6F9EC097F0080E79
:107050009E619AC097F02A0E9A6F97519AC0EBFFE3
:1070600013EC66F09E2BDBD7FCEC61F0230E9D63E6
:10707000DDD7080E9E631BD011EED2F0330EE66210
:1070800016D0380EE66213D0370EE66210D0360EF8
:10709000E6620DD0380EE6620AD0330EE66207D003
:1070A000320EE66204D0340EE66201D01CD0FC0E33
:1070B000F76E3E0EF66E20EED6F0F5EC65F0FC0EA7
:1070C000F76E4E0EF66E20EEE6F0F5EC65F013EC82
:1070D00066F0AAEC34F0640EAE6F140EAD6FAD67BF
:1070E000FED772EF35F09E6BFC0EF76E5E0EF66EFD
:1070F00020EED6F0F5EC65F0100E976F00EEE6F09E
:1071000011EE2EF0E6CFEEFF972FFCD713EC66F0D2
:1071100081B2BAEF38F0A0B18FEF38F0F9D7FCECBC
:1071200061F02A0E9D6306D009EC66F013EC66F060
:107130009E6BEED7230E9D630BD0100E976F10EE53
:10714000E6F001EE2EF0E6CFEEFF972FFCD777D5D5
:107150009E6704D009EC66F010EEE6F0100E9E611A
:107160009E690F0E9E179E519DC0E3FF13EC66F0C3
:107170009E2BCED7100E976F10EEE6F001EE2EF09C
:10718000E6CFEEFF972FFCD71FEF36F0FA0EF76E23
:107190006E0EF66E20EED6F0F5EC65F0FA0EF76E98
:1071A0007E0EF66E20EEE6F0F5EC65F013EC66F080
:1071B00081B21FEF36F0A0B1DFEF38F0F9D7FCEC69
:1071C00061F0230E9D6344D5FA0EF76ECE0EF66E77
:1071D00020EED6F0F5EC65F009EC66F013EC66F005
:1071E0002EEC5DF09E6B81B21FEF36F0A0B10FEF79
:1071F00039F0F9D70F0E9A6F100E9E619AC09EF06B
:107200002A0E9A6F9E5111EED2F000EEE6F09DC06C
:10721000E3FF9AC0EBFF13EC66F09E2BE4D7FCEC87
:1072200061F0230E9D63E6D7080E9E637CD5080EA1
:10723000976F11EE14F001EED2F0E650EE6273D5C6
:10724000972FFBD7FA0EF76EDE0EF66E20EED6F015
:10725000F5EC65F009EC66F02EEC5DF013EC66F0F1
:107260009E6B81B21FEF36F0A0B138EF39F0F9D73D
:10727000FCEC61F0230E9D632BD02F0E11EED2F0AB
:10728000E7643BD03A0EE76038D0080E976F01EE06
:1072900014F0E6CFEEFF972FFCD7FA0EF76EEE0E46
:1072A000F66E20EED6F0F5EC65F0FA0EF76EFE0EF7
:1072B000F66E20EEE6F0F5EC65F013EC66F0640E89
:1072C000AE6F140EAD6FAD67FED78FEC34F0B7D450
:1072D000070E9A6F080E9E619AC09EF02A0E9A6F52
:1072E0009E5111EED2F000EEE6F09DC0E3FF9AC091
:1072F000EBFF13EC66F09E2BB4D7AAEC34F0FB0E38
:10730000F76EAE0EF66E20EED6F0F5EC65F0FB0EE5
:10731000F76EBE0EF66E20EEE6F0F5EC65F013ECBF
:1073200066F0640EAE6F140EAD6FAD67FED787D4F6
:107330008FEC34F0640EAE6F0F0EAD6FAD67FED7FD
:1073400081B2ECEF5BF0F20EF76E3E0EF66E20EEC1
:10735000D6F0F5EC65F0F20EF76E4E0EF66E20EEFE
:10736000E6F0F5EC65F013EC66F081B272EF35F003
:10737000A0B1BCEF39F0F9D7FCEC61F0230E9D63AE
:1073800072EF3BF0F20EF76E5E0EF66E20EED6F068
:10739000F5EC65F0F20EF76E6E0EF66E20EEE6F08E
:1073A000F5EC65F033EC3BF080C0F3F081C0F4F015
:1073B000F4EC3AF080C0E3F081C0E4F013EC66F046
:1073C0009E6B640EB06F060EAF6F81B28FEF3AF016
:1073D000A0B107EF3AF0AF67F8D7200EE36FE46F84
:1073E00013EC66F0640EB06F020EAF6F81B28FEFD8
:1073F0003AF0A0B107EF3AF0AF67F8D7F4EC3AF003
:1074000080C0E3F081C0E4F013EC66F0DAD7FCEC66
:1074100061F0230E9D5D25E02A0E9D6303D0300EA2
:10742000226EC6D7310E9D5D10E0320E9D5D0DE0DF
:10743000330E9D5D0AE0370E9D5D0DE0380E9D5DBB
:107440000AE0390E9D5D07E0B3D7000E2264B0D785
:10745000F00E2226ADD7600E2260AAD7100E22268B
:10746000A7D7F4EC3AF080C0E3F081C0E4F033EC4D
:107470003BF080C0F3F081C0F4F013EC66F0640ED2
:10748000B06F060EAF6F81B28FEF3AF0A0B165EF2B
:107490003AF0AF67F8D7200EF36FF46F13EC66F095
:1074A000640EB06F020EAF6F81B28FEF3AF0A0B1F1
:1074B00065EF3AF0AF67F8D733EC3BF080C0F3F0FC
:1074C00081C0F4F013EC66F0DAD7FCEC61F0230E27
:1074D0009D5D25E02A0E9D6303D0000E236EC7D765
:1074E000310E9D5D10E0320E9D5D0DE0330E9D5D11
:1074F0000AE0370E9D5D0DE0380E9D5D0AE0390E05
:107500009D5D07E0B4D70C0E235CB1E0040E23268A
:10751000AED7F40E235CABE0FC0E2326A8D733ECE9
:107520003BF080C0F3F081C0F4F013EC66F0B6ECF1
:107530003AF0640EAE6F320EAD6F3DB0A6EF3AF08A
:107540003DB2A5EF3AF0AD67F8D73D92D5EC3AF0F1
:10755000640EAE6F320EAD6F3DB0B5EF3AF03DB296
:10756000B4EF3AF0AD67F8D73D92E4D603EE00F001
:10757000410EEE6E540EEE6E2B0EEE6E560EEE6E4D
:10758000470EEE6E520EEE6E3D0EEE6E22C084F091
:1075900059EC61F07FC0EEFF80C0EEFF81C0EEFFCE
:1075A000EE6A3D6ADFEC65F0120003EE00F0410E7A
:1075B000EE6E540EEE6E2B0EEE6E560EEE6E470E07
:1075C000EE6E540EEE6E3D0EEE6E23C084F059EC5E
:1075D00061F07FC0EEFF80C0EEFF81C0EEFFEE6A7B
:1075E0003D6ADFEC65F01200100E226005D02B0E14
:1075F000806F360E816F1200200E226005D02B0E98
:10760000806F340E816F1200300E226005D02B0E79
:10761000806F320E816F1200400E226005D0200E66
:10762000806F300E816F1200500E226005D02D0E3B
:10763000806F320E816F1200600E226005D02D0E19
:10764000806F340E816F1200700E226005D02D0EF7
:10765000806F360E816F1200300E226E200E806F0A
:10766000300E816F12000C0E236205D02B0E806F3E
:10767000360E816F1200080E236205D02B0E806F2C
:10768000340E816F1200040E236205D02B0E806F22
:10769000320E816F1200000E236205D0200E806F23
:1076A000300E816F1200FC0E236205D02D0E806F0C
:1076B000320E816F1200F80E236205D02D0E806FFE
:1076C000340E816F1200F40E236205D02D0E806FF0
:1076D000360E816F1200000E236E200E806F300E6A
:1076E000816F1200F20EF76E7E0EF66E20EED6F06F
:1076F000F5EC65F0F20EF76E8E0EF66E20EEE6F00B
:10770000F5EC65F013EC66F081B29AEF39F0A0B1B8
:107710008BEF3BF0F9D7FCEC61F0230E9D63C6EFD5
:107720003CF0F20EF76E9E0EF66E20EED6F0F5EC03
:1077300065F0F20EF76EAE0EF66E20EEE6F0F5ECAA
:1077400065F020C084F059EC61F0200EE36FE46F27
:10775000300E806380C0E4F081C0E5F021C084F089
:1077600059EC61F0200EF36FF46F300E806380C02F
:10777000F4F081C0F5F013EC66F0640EB06F060E05
:10778000AF6F81B2F9EF3BF0A0B1EBEF3BF0AF6729
:10779000F8D7200EE36FE46FE56F13EC66F0640E2C
:1077A000B06F020EAF6F81B2F9EF3BF0A0B1EBEF1B
:1077B0003BF0AF67F8D720C084F059EC61F0200EA1
:1077C000E36FE46F300E806380C0E4F081C0E5F0C9
:1077D00013EC66F0D2D7FCEC61F0230E9D6301D070
:1077E00018D02A0E9D63ADD7202A0F0E2060206A84
:1077F000A8D720C084F059EC61F0200EE36FE46F4D
:10780000300E806380C0E4F081C0E5F013EC66F0D8
:1078100067D020C084F059EC61F0200EE36FE46F74
:10782000300E806380C0E4F081C0E5F021C084F0B8
:1078300059EC61F0200EF36FF46F300E806380C05E
:10784000F4F081C0F5F013EC66F0640EB06F060E34
:10785000AF6F81B261EF3CF0A0B153EF3CF0AF6786
:10786000F8D7200EF36FF46FF56F13EC66F0640E2B
:10787000B06F020EAF6F81B261EF3CF0A0B153EF79
:107880003CF0AF67F8D721C084F059EC61F0200ECE
:10789000F36FF46F300E806380C0F4F081C0F5F0B8
:1078A00013EC66F0D2D7FCEC61F0230E9D6301D09F
:1078B00008D02A0E9D63BAD7212A0F0E2160216AB3
:1078C000B5D721C084F059EC61F0200EF36FF46F4E
:1078D000300E806380C0F4F081C0F5F013EC66F0E8
:1078E00003EE00F0410EEE6E540EEE6E2B0EEE6EB9
:1078F000570EEE6E560EEE6E520EEE6E3D0EEE6EA4
:1079000020C084F059EC61F07FC0EEFF80C0EEFF34
:1079100081C0EEFF2C0EEE6E21C084F059EC61F0B8
:107920007FC0EEFF80C0EEFF81C0EEFFEE6A3D6AD1
:10793000DFEC65F0640EAE6F320EAD6F3DB0C3EF9D
:107940003CF03DB2A6EF3CF0AD67F8D73D92F20EA9
:10795000F76EBE0EF66E20EED6F0F5EC65F0F20E88
:10796000F76ECE0EF66E20EEE6F0F5EC65F013EC59
:1079700066F0640EAE6F320EAD6FAD67FED7050ECA
:10798000206E216ACED63D903488D4D4F20EF76EA4
:10799000DE0EF66E20EED6F0F5EC65F0F20EF76E28
:1079A000EE0EF66E20EEE6F0F5EC65F013EC66F008
:1079B00081B29AEF39F0A0B1DFEF3CF0F9D7FCECDF
:1079C00061F0230E9D63C7EF3DF0F20EF76EFE0EE1
:1079D000F66E20EED6F0F5EC65F070EC3DF013ECB1
:1079E00066F0640EB06F060EAF6F81B221EF3DF00E
:1079F000A0B114EF3DF0AF67F8D7F30EF76E7E0E2F
:107A0000F66E20EEE6F0F5EC65F013EC66F0640E31
:107A1000B06F020EAF6F81B221EF3DF0A0B114EF55
:107A20003DF0AF67F8D7D9D7FCEC61F02A0E9D6323
:107A300005D01F2A070E1F601F6ACFD7230E9D6334
:107A4000D0D770EC3DF013EC66F003EE00F0410E81
:107A5000EE6E540EEE6E2B0EEE6E570EEE6E4D0E5B
:107A6000EE6E420EEE6E530EEE6E3D0EEE6E1FC0CB
:107A700084F059EC61F07FC0EEFF80C0EEFF81C062
:107A8000EEFFEE6A3D6ADFEC65F0640EAE6F320E1B
:107A9000AD6F3DB06DEF3DF03DB251EF3DF0AD67E4
:107AA000F8D73D92F30EF76E8E0EF66E20EED6F0FE
:107AB000F5EC65F0F30EF76E9E0EF66E20EEE6F036
:107AC000F5EC65F013EC66F0640EAE6F320EAD6F40
:107AD000AD67FED7050E1F6E78D73D9034882AD447
:107AE000000E1F6209D0F30EF76E0E0EF66E20EE3A
:107AF000E6F0F5EC65F01200010E1F6209D0F30EFE
:107B0000F76E1E0EF66E20EEE6F0F5EC65F0120054
:107B1000020E1F6209D0F30EF76E2E0EF66E20EEE7
:107B2000E6F0F5EC65F01200030E1F6209D0F30ECB
:107B3000F76E3E0EF66E20EEE6F0F5EC65F0120004
:107B4000040E1F6209D0F30EF76E4E0EF66E20EE95
:107B5000E6F0F5EC65F01200050E1F6209D0F30E99
:107B6000F76E5E0EF66E20EEE6F0F5EC65F01200B4
:107B7000060E1F6209D0F30EF76E6E0EF66E20EE43
:107B8000E6F0F5EC65F01200050E1F6EA9D7F30EB6
:107B9000F76EAE0EF66E20EED6F0F5EC65F0F30E55
:107BA000F76EBE0EF66E20EEE6F0F5EC65F013EC27
:107BB00066F081B29AEF39F0A0B1E0EF3DF0F9D76D
:107BC000FCEC61F0230E9D6325EF3EF08FEC34F06A
:107BD000F30EF76ECE0EF66E20EED6F0F5EC65F0F5
:107BE00009EC66F013EC66F001EED2F010EEE6F070
:107BF0009E6B81B298EF39F0A0B100EF3EF0F9D75B
:107C0000FCEC61F0230E9D6312D0040E9E6350EFD6
:107C100035F001EED2F011EE00F0EECFE6FFEECF40
:107C2000E6FFEECFE6FFEECFE6FF9AEF39F09E2BB0
:107C3000200E9E659DC0EEFF2A0E9A6F100E9E6567
:107C40009AC0E6FF13EC66F0D4D7F30EF76EDE0EA3
:107C5000F66E20EED6F0F5EC65F0F30EF76EEE0E54
:107C6000F66E20EEE6F0F5EC65F013EC66F081B20E
:107C70009AEF39F0A0B13EEF3EF0F9D7FCEC61F09D
:107C8000230E9D63F6EF3EF08FEC34F0F80EF76EA6
:107C90002E0EF66E20EED6F0F5EC65F0F80EF76ECF
:107CA0003E0EF66E20EEE6F0F5EC65F03998310EFA
:107CB00039B8320EE56F9E6B080E976F00EEEEF04E
:107CC00011EE40F039B811EE48F0E6CFEEFF972FF5
:107CD000FCD713EC66F0640EB06F060EAF6F81B286
:107CE000F4EF3EF0A0B1A0EF3EF0AF67F8D710EE92
:107CF000EEF0200EE66EE66EE66EE66EE66EE66E80
:107D0000E66EE66E13EC66F0640EB06F020EAF6FB7
:107D100081B2F4EF3EF0A0B1A0EF3EF0AF67F8D72C
:107D2000080E976F00EEEEF011EE40F039B811EE4C
:107D300048F0E6CFEEFF972FFCD713EC66F0CBD7D9
:107D4000FCEC61F0230E9D5D44E02A0E9D630DD096
:107D5000080E976F11EE40F039B811EE48F0200E82
:107D6000E66E972FFCD79E6BA7D79E670BD0080EA9
:107D7000976F11EE40F039B811EE48F0200EE66E24
:107D8000972FFCD7080E9E610AD011EE40F039B84B
:107D900011EE48F09E519DC0E3FF9E2B8DD7F80E4B
:107DA000F76E4E0EF66E20EEE6F0F5EC65F013EC95
:107DB00066F081B2F4EF3EF0A0B1E0EF3EF0F9D70B
:107DC000F80EF76E3E0EF66E20EEE6F0F5EC65F07E
:107DD000BFD730A202D09AEF39F03978310E39B8D6
:107DE000320EE56F9E6B68D79AEF39F0F40EF76E9E
:107DF0001E0EF66E20EED6F0F5EC65F0F40EF76E82
:107E00002E0EF66E20EEE6F0F5EC65F013EC66F063
:107E100081B29AEF39F0A0B10FEF3FF0F9D7FCEC47
:107E200061F0230E9D638CEF3FF08FEC34F0E30E96
:107E3000F76E5E0EF66E20EED6F0F5EC65F009EC0E
:107E400066F013EC66F02EEC5DF09E6B01EED2F066
:107E500010EEE6F081B29AEF39F0A0B131EF3FF0C9
:107E6000F9D7FCEC61F0230E9D5D0EE09E2B200EF9
:107E70009E659DC0EEFF2A0E9A6F100E9E659AC0F9
:107E8000E6FF13EC66F0E6D701EED2F0330EEE62B9
:107E900035D0380EEE6232D0370EEE622FD0360E6D
:107EA000EE622CD0380EEE6229D0330EEE6226D070
:107EB000320EEE6223D0340EEE6220D0E30EF76E67
:107EC0007E0EF66E20EED6F0F5EC65F0E30EF76E62
:107ED0008E0EF66E20EEE6F0F5EC65F013EC66F033
:107EE000FF0ED16FD26F00EED1F0020ECB6F030EFA
:107EF000AA6EFE0EA96EC6EC65F0FF00E60EF76EE8
:107F00002E0EF66E20EED6F0F5EC65F009EC66F07C
:107F100013EC66F054EF14F0F40EF76E3E0EF66EAE
:107F200020EED6F0F5EC65F0F40EF76E4E0EF66E20
:107F300020EEE6F0F5EC65F013EC66F081B29AEF16
:107F400039F0A0B1A5EF3FF0F9D7FCEC61F0230EBA
:107F50009D63BBEF43F0F40EF76E7E0EF66E20EEDF
:107F6000D6F0F5EC65F009EC66F03F963D903D9259
:107F7000E00EF76E740EF66E23EE00F0EEEC65F098
:107F8000DE6ADFEC65F0640EAE6F320EAD6F3DB0B1
:107F9000E6EF3FF0AD67FBD7F40EF76E8E0EF66E90
:107FA00020EED6F0F5EC65F0F40EF76E9E0EF66E50
:107FB00020EEE6F0F5EC65F013EC66F0640EAE6FC3
:107FC000140EAD6FAD67FED772EF35F0100E976FE0
:107FD00018EE12F000EEE6F0E6CFEEFF972FFCD79A
:107FE00013EC66F081B29AEF39F0A0B1F9EF3FF0EF
:107FF000F9D7FCEC61F02A0E9D6302D0E5EF40F06A
:10800000F50EF76E2E0EF66E20EED6F0F5EC65F05E
:10801000F50EF76E3E0EF66E20EEE6F0F5EC65F02E
:1080200013EC66F09E6B81B29AEF39F0A0B138EF95
:1080300040F0F9D70F0E9A6F100E9E619AC09EF015
:108040009E5111EED2F09DC0E3FF00EEEEF0070E60
:108050009A6F9EC097F0080E9E619AC097F02A0E04
:108060009A6F97519AC0EBFF13EC66F09E2BDBD70B
:10807000FCEC61F0230E9D63DDD7080E9E6389D072
:1080800001EE04F011EED2F0EE50E66282D09E2FA7
:10809000FBD7F50EF76E4E0EF66E20EED6F0F5EC31
:1080A00065F0F50EF76E5E0EF66E20EEE6F0F5EC7E
:1080B00065F013EC66F02EEC5DF013EC66F09E6B51
:1080C00081B29AEF39F0A0B167EF40F0F9D7FCEC3C
:1080D00061F0230E9D632CD02F0E11EED2F0E764D9
:1080E0003CD03A0EE76039D0080E976F01EE04F0ED
:1080F000E6CFEEFF972FFCD7F50EF76E6E0EF66EFD
:1081000020EED6F0F5EC65F0F50EF76E7E0EF66E0D
:1081100020EEE6F0F5EC65F013EC66F0640EAE6F61
:10812000140EAD6FAD67FED78FEC34F09AEF39F0D7
:10813000070E9A6F080E9E619AC09EF02A0E9A6FE3
:108140009E5111EED2F000EEEEF09DC0E3FF9AC01A
:10815000EBFF13EC66F09E2BB3D7AAEC34F0F50ED0
:10816000F76EAE0EF66E20EED6F0F5EC65F0F50E7D
:10817000F76EBE0EF66E20EEE6F0F5EC65F013EC51
:1081800066F0640EAE6F140EAD6FAD67FED79AEF5A
:1081900039F0F50EF76E8E0EF66E20EED6F0F5EC99
:1081A00065F0F50EF76E9E0EF66E20EEE6F0F5EC3D
:1081B00065F013EC66F0AAEC34F0640EAE6F140EAA
:1081C000AD6FAD67FED772EF35F0F40EF76EAE0E01
:1081D000F66E20EED6F0F5EC65F0F40EF76EBE0EFE
:1081E000F66E20EEE6F0F5EC65F013EC66F02EECA2
:1081F0005DF09E6B81B29AEF39F0A0B11FEF41F0B4
:10820000F9D70F0E9A6F100E9E619AC09EF09E5184
:1082100011EED2F09DC0E3FF00EEEEF0070E9A6F74
:108220009EC097F0080E9E619AC097F02A0E9A6F32
:1082300097519AC0EBFF13EC66F09E2BDBD7FCEC5A
:1082400061F0230E9D63DDD7080E9E630AD001EE18
:1082500004F011EED2F0EE50E66203D09E2FFBD771
:108260001CD0F50EF76E8E0EF66E20EED6F0F5EC05
:1082700065F0F50EF76E9E0EF66E20EEE6F0F5EC6C
:1082800065F013EC66F0AAEC34F0640EAE6F140ED9
:10829000AD6FAD67FED772EF35F0F40EF76ECE0E10
:1082A000F66E20EED6F0F5EC65F009EC66F013EC16
:1082B00066F02EEC5DF09E6B81B29AEF39F0A0B1C2
:1082C00076EF41F0F9D70F0E9A6F100E9E619AC0AB
:1082D0009EF09E5111EED2F09DC0E3FF00EEE6F05D
:1082E0009DC0EBFF13EC66F09E2BE6D7FCEC61F033
:1082F0002A0E9D6301D0D9D7230E9D63E4D70F0EBC
:108300009E6301D003D00E0E9E6340D03D903D92FF
:10831000E00EF76E6A0EF66E23EE00F0EEEC65F0FE
:10832000DE6ADFEC65F0640EAE6F640EAD6F3DB0DB
:10833000DAEF41F03DB2A2EF41F03FB8DCEF41F09F
:10834000AD67F5D73D92F40EF76E5E0EF66E20EE39
:10835000D6F0F5EC65F0F40EF76E6E0EF66E20EECC
:10836000E6F0F5EC65F013EC66F0A66BA76B53EC4A
:1083700063F0A68753EC63F0020EC06FC16BBF8F32
:1083800081A2C0EF41F0AFEC61F0FF00F40EF76E98
:10839000DE0EF66E20EED6F0F5EC65F0F40EF76E1C
:1083A000EE0EF66E20EEE6F0F5EC65F013EC66F0FE
:1083B00054EF14F03D90BBD73F983D9E640EAE6FD6
:1083C000640EAD6F3DBE03D0AD67FCD7BCD73D9EFC
:1083D000150EC963F7D7F40EF76EFE0EF66E20EE9B
:1083E000D6F0F5EC65F013EC66F0860EF76ED00E65
:1083F000F66E100E986F5FEC43F0100E986F55EC10
:1084000043F0860EF76EE00EF66E100E986F5FEC7E
:1084100043F0100E986F55EC43F0860EF76EF00E99
:10842000F66E100E986F5FEC43F0100E986F55ECDF
:1084300043F0870EF76E000EF66E100E986F5FEC2D
:1084400043F0100E986F55EC43F0870EF76E100E48
:10845000F66E100E986F5FEC43F0100E986F55ECAF
:1084600043F0030E976F870EF76E200EF66E100E18
:10847000986F5FEC43F0100E986F55EC43F0972F18
:10848000F2D7870EF76E300EF66E100E986F5FEC17
:1084900043F0100E986F55EC43F0870EF76E400EC8
:1084A000F66E100E986F5FEC43F0100E986F55EC5F
:1084B00043F0870EF76E500EF66E100E986F5FEC5D
:1084C00043F0100E986F55EC43F0350E976F870E02
:1084D000F76E600EF66E100E986F5FEC43F0100EA4
:1084E000986F55EC43F0972FF2D7870EF76E700E0A
:1084F000F66E040E986F5FEC43F0040E986F55EC27
:1085000043F0640EAE6F050EAD6FAD67FED7870EFC
:10851000F76E740EF66E010E986F5FEC43F0010E6D
:10852000986F55EC43F0640EAE6F0A0EAD6FAD67F9
:10853000FED78280576A640EAE6F050EAD6FAD67D1
:10854000FED78290640EAE6F140EAD6FAD67FED78E
:108550003D903D92E00EF76E9A0EF66E23EE00F01F
:10856000EEEC65F0DE6ADFEC65F0640EAE6F640E73
:10857000AD6F57B6C5EF42F057B0C5EF42F03DB012
:1085800003D0AD67F6D7DFD63D903D903D92E00E2B
:10859000F76E120EF66E23EE00F0EEEC65F0DE6A7A
:1085A000DFEC65F0640EAE6F140EAD6F3DB0DFEF23
:1085B00042F03DB2A3EF41F0AD67F8D7C4D63D908D
:1085C0003D92E00EF76E2E0EF66E23EE00F0EEEC0E
:1085D00065F0DE6ADFEC65F0640EAE6F320EAD6FF3
:1085E0003DB0FAEF42F03DB2F8EF42F0AD67F8D798
:1085F0003D92A9D6640EAE6F140EAD6FAD67FED777
:1086000003EE00F0410EEE6E540EEE6E2B0EEE6E8B
:10861000570EEE6E490EEE6E4D0EEE6E450EEE6E80
:10862000490EEE6E3D0EEE6E100E976F11EED2F00B
:10863000200EE76404D0E6CFEEFF972FF9D70D0E9A
:10864000EE6EEE6ADFEC65F0640EAE6F640EAD6F39
:108650003DB230EF43F03DB032EF43F0AD67F8D7B5
:108660003D9271D6F50EF76E0E0EF66E20EED6F038
:10867000F5EC65F0F50EF76E1E0EF66E20EEE6F0E8
:10868000F5EC65F013EC66F0A66BA76B53EC63F0AA
:10869000A68753EC63F0020EC06FC16BBF8F81A23F
:1086A0004FEF43F0AFEC61F0FF0003EE00F0EECFD0
:1086B000ADFF00009EA8FED7982FF9D71200F86AE8
:1086C00003EE00F00900F5CFEEFF982FFBD7120064
:1086D0000201FE454550524F4D2020202032382FB8
:1086E00030312F30302031323A3038002056657228
:1086F00073696F6E20763161303620202020202073
:1087000020433A5C544D505C746D705C3430305F83
:108710006D3131622E35345C6F757400202020205D
:108720002020202020202020202020202020202049
:10873000207E81F7EB18000000908258AD2A0102DC
:1087400000CDAB12000100005E010900BAD34D75E7
:10875000FE4A6F92F11A1A1A1A1A1A1A1A1A1A1AC1
:108760001A1A1A1A1A1A1A1A1A1A1A1A1A1A1A1A69
:108770001A1A1A910400F50EF76ECE0EF66E20EE60
:10878000D6F0F5EC65F0F50EF76EDE0EF66E20EE27
:10879000E6F0F5EC65F013EC66F081B29AEF39F093
:1087A000A0B1D4EF43F0F9D7FCEC61F0230E9D6348
:1087B0009AEF39F0F50EF76EEE0EF66E20EED6F06B
:1087C000F5EC65F030C081F030B009D0F50EF76EF1
:1087D000FE0EF66E20EEE6F0F5EC65F008D0F60E33
:1087E000F76E0E0EF66E20EEE6F0F5EC65F013EC8B
:1087F00066F0640EAE6F060EAD6F81B29AEF39F07F
:10880000A0B11CEF44F0AD67F8D7F60EF76E1E0E60
:10881000F66E20EEE6F0F5EC65F013EC66F0640E13
:10882000AE6F020EAD6F81B29AEF39F0A0B11CEFBE
:1088300044F0AD67F8D7C8D7FCEC61F02A0E9D6311
:1088400002D03070C1D7230E9D63BED781A19AEFAD
:1088500039F030A034889AEF39F0640EAE6F0F0E05
:10886000AD6FAD67FED781B2ECEF5BF0EF0EF76E48
:108870004E0EF66E20EED6F0F5EC65F0EF0EF76ECC
:108880005E0EF66E20EEE6F0F5EC65F013EC66F0A9
:1088900081B272EF35F0A0B14FEF44F0F9D7FCECA4
:1088A00061F0230E9D63EEEF44F0EF0EF76E6E0E57
:1088B000F66E20EED6F0F5EC65F0A2EC49F013EC84
:1088C00066F0640EAE6F060EAD6F81B22DEF44F010
:1088D000A0B184EF44F0AD67F8D7EF0EF76EAE0E9F
:1088E000F66E20EEE6F0F5EC65F013EC66F0640E43
:1088F000AE6F020EAD6F81B22DEF44F0A0B184EFE8
:1089000044F0AD67F8D7D9D7FCEC61F02A0E9D632F
:108910000CD00CC081F0FC0E0C16030E8117812BBD
:108920008161816B81510C12C8D7230E9D63C5D71D
:10893000EF0EF76EBE0EF66E20EED6F0F5EC65F09B
:108940000CB409D0EF0EF76EDE0EF66E20EEE6F0F8
:10895000F5EC65F008D0EF0EF76ECE0EF66E20EE59
:10896000E6F0F5EC65F013EC66F081B22DEF44F023
:10897000A0B1BCEF44F0F9D7FCEC61F0230E9D5D93
:1089800002E00C74D5D7EF0EF76EEE0EF66E20EE09
:10899000D6F0F5EC65F00CB609D0F00EF76E0E0EC1
:1089A000F66E20EEE6F0F5EC65F008D0EF0EF76E0F
:1089B000FE0EF66E20EEE6F0F5EC65F013EC66F0D8
:1089C00081B22DEF44F0A0B1E7EF44F0F9D7FCEC11
:1089D00061F0230E9D5D02E00C76D5D7F00EF76EA8
:1089E0001E0EF66E20EED6F0F5EC65F0F00EF76E8A
:1089F0002E0EF66E20EEE6F0F5EC65F013EC66F068
:108A000081B22DEF44F0A0B107EF45F0F9D7FCECAF
:108A100061F0230E9D63D0EF45F0F00EF76E3E0E31
:108A2000F66E20EED6F0F5EC65F0F00EF76E4E0E19
:108A3000F66E20EEE6F0F5EC65F013EC66F0640EF1
:108A4000B06F060EAF6F81B22DEF44F0A0B142EFD0
:108A500045F0AF67F8D7200EF56F13EC66F0640EA3
:108A6000B06F020EAF6F81B22DEF44F0A0B142EFB4
:108A700045F0AF67F8D70E500F0B300FF56F13ECC2
:108A800066F0DDD7FCEC61F02A0E9D6304D00E6A1F
:108A9000300EF56FD4D7230E9D6301D008D00F0E92
:108AA0009D150E6E9DC0F5F013EC66F0C8D7F00E64
:108AB000F76E5E0EF66E20EED6F0F5EC65F009EC82
:108AC00066F001EE50F011EED2F0100E8B6FEECF8B
:108AD000E6FF8B2FFCD79E6B01EED2F010EEE6F096
:108AE000100E8B6FEECFE6FF8B2FFCD713EC66F0EA
:108AF00081B2C4EF45F0A0B17FEF45F0F9D7FCECAF
:108B000061F02A0E9D630AD0100E8B6F01EED2F039
:108B1000200EEE6E8B2FFCD79E6BDED7230E9D634F
:108B200001D027D09E6708D0100E8B6F01EED2F0D7
:108B3000200EEE6E8B2FFCD7100E9E6115D0010E0D
:108B40009E630BD0300E9D6308D0300E01EED2F044
:108B5000EF6203D09E6B2B0E9D6F9E5111EED2F0F3
:108B60009DC0E3FF9E2BB8D7AAEC34F0100E9E6F89
:108B7000B3D7100E8B6F01EED2F011EE50F0EECFA6
:108B8000E6FF8B2FFCD70CD0100E8B6F01EED2F0CE
:108B900011EE50F0EECFE6FF8B2FFCD72DEF44F017
:108BA000F00EF76E6E0EF66E20EED6F0F5EC65F078
:108BB000F00EF76E7E0EF66E20EEE6F0F5EC65F048
:108BC00013EC66F081B22DEF44F0A0B1E9EF45F06F
:108BD000F9D7FCEC61F0230E9D638DEF48F0F00EA9
:108BE000F76E8E0EF66E20EED6F0F5EC65F0F00E18
:108BF000F76E9E0EF66E20EEE6F0F5EC65F09E6BDD
:108C000010C084F059EC61F080C0F4F081C0F5F040
:108C100013EC66F0640EB06F060EAF6F81B22DEFED
:108C200044F0A0B12EEF46F0AF67F8D7200EF46FF6
:108C3000F56F13EC66F0640EB06F020EAF6F81B289
:108C40002DEF44F0A0B12EEF46F0AF67F8D780C00B
:108C5000F4F081C0F5F013EC66F0DCD7FCEC61F0C9
:108C60002A0E9D6304D0010E106E9E6BC9D7230E91
:108C70009D5D25E09E6708D0200EF46FF56F300EE5
:108C80007F6F806F816F9E6B030E9E6112D080C0DC
:108C90007FF081C080F09DC081F00FEC61F0000E8C
:108CA000846507D0210E846104D084C010F09E2B0F
:108CB000A7D7AAEC34F0010E106E9E6BA1D7F00E70
:108CC000F76EAE0EF66E20EED6F0F5EC65F0F00E17
:108CD000F76EBE0EF66E20EEE6F0F5EC65F09E6BDC
:108CE00011C084F059EC61F080C0F4F081C0F5F05F
:108CF00013EC66F0640EB06F060EAF6F81B22DEF0D
:108D000044F0A0B19EEF46F0AF67F8D7200EF46FA5
:108D1000F56F13EC66F0640EB06F020EAF6F81B2A8
:108D20002DEF44F0A0B19EEF46F0AF67F8D780C0BA
:108D3000F4F081C0F5F013EC66F0DCD7FCEC61F0E8
:108D40002A0E9D6304D0010E116E9E6BC9D7230EAF
:108D50009D5D25E09E6708D0200EF46FF56F300E04
:108D60007F6F806F816F9E6B030E9E6112D080C0FB
:108D70007FF081C080F09DC081F00FEC61F0000EAB
:108D8000846507D0210E846104D084C011F09E2B2D
:108D9000A7D7AAEC34F0010E116E9E6BA1D7F00E8E
:108DA000F76ECE0EF66E20EED6F0F5EC65F0F00E16
:108DB000F76EDE0EF66E20EEE6F0F5EC65F012C012
:108DC00084F059EC61F080C0E8F02E0EE96F81C0AC
:108DD000EAF013EC66F0640EB06F060EAF6F81B26E
:108DE0002DEF44F0A0B112EF47F0AF67F8D7200E97
:108DF000E86FE96FEA6F13EC66F0640EB06F020E75
:108E0000AF6F81B22DEF44F0A0B112EF47F0AF6722
:108E1000F8D780C0E8F02E0EE96F81C0EAF013ECBD
:108E200066F0D9D7FCEC61F0230E9D5D13E02A0EAD
:108E30009D6303D0050E126EC2D712C084F0050EDA
:108E40008427370E846103D084C012F0B8D70A0E8D
:108E5000126EB5D7F00EF76EEE0EF66E20EED6F06F
:108E6000F5EC65F0F00EF76EFE0EF66E20EEE6F015
:108E7000F5EC65F013C084F059EC61F07FC0F4F0BC
:108E800080C0F5F013EC66F0640EB06F060EAF6FA5
:108E900081B22DEF44F0A0B168EF47F0AF67F8D78B
:108EA000200EF46FF56F13EC66F0640EB06F020ED7
:108EB000AF6F81B22DEF44F0A0B168EF47F0AF671C
:108EC000F8D77FC0F4F080C0F5F013EC66F0DCD783
:108ED000FCEC61F0230E9D5D16E02A0E9D6303D02D
:108EE0000A0E136EC7D713C084F00A0E8427FB0E38
:108EF000846106D0090E846503D084C013F0BAD70C
:108F00000A0E136EB7D7F10EF76E0E0EF66E20EE48
:108F1000D6F0F5EC65F00CBE09D0F10EF76E1E0E22
:108F2000F66E20EEE6F0F5EC65F008D0F10EF76E87
:108F30002E0EF66E20EEE6F0F5EC65F013EC66F022
:108F400081B22DEF44F0A0B1A7EF47F0F9D7FCECC8
:108F500061F02A0E9D6302D00C7ED5D7230E9D634F
:108F6000EFD7F10EF76E3E0EF66E20EED6F0F5EC72
:108F700065F0F10EF76E4E0EF66E20EEE6F0F5ECB3
:108F800065F09E6B080E976F11EE70F000EEEEF03C
:108F9000E6CFEEFF972FFCD713EC66F081B2FDEF22
:108FA00047F0A0B1D5EF47F0F9D7FCEC61F02A0EFD
:108FB0009D6325D0080E976F01EE70F0200EEE6EC7
:108FC000972FFCD79E6BDED79E6708D0080E976F51
:108FD00001EE70F0200EEE6E972FFCD79E2B090E3F
:108FE0009E6106D09E5111EE6FF09DC0E3FFCAD77F
:108FF000AAEC34F0080E9E6FC5D72DEF44F0230E77
:109000009D63E2D7F10EF76E5E0EF66E20EED6F09F
:10901000F5EC65F0F10EF76E6E0EF66E20EEE6F0F2
:10902000F5EC65F09E6B040E976F11EE78F000EE94
:10903000F2F0E6CFEEFF972FFCD713EC66F081B28B
:109040004EEF48F0A0B126EF48F0F9D7FCEC61F004
:109050002A0E9D6325D0040E976F01EE78F0200E46
:10906000EE6E972FFCD79E6BDED79E6708D0040E5E
:10907000976F01EE78F0200EEE6E972FFCD79E2BA7
:10908000050E9E6106D09E5111EE77F09DC0E3FF64
:10909000CAD7AAEC34F0040E9E6FC5D72DEF44F06A
:1090A000230E9D63E2D7F10EF76E7E0EF66E20EE74
:1090B000D6F0F5EC65F0F10EF76E8E0EF66E20EE42
:1090C000E6F0F5EC65F09E6B0F50300FF56F13EC8A
:1090D00066F081B286EF48F0A0B170EF48F0F9D7A2
:1090E000FCEC61F02A0E9D6313D00F6A9E6BECD7E7
:1090F0009E2B020E9E6105D09D51F56F0F0B0F6EDA
:10910000E3D7AAEC34F09E6B0F6ADED72DEF44F064
:10911000230E9D63EDD72DEF44F0F10EF76E9E0EFA
:10912000F66E20EED6F0F5EC65F0F10EF76EAE0EB1
:10913000F66E20EEE6F0F5EC65F013EC66F081B229
:109140002DEF44F0A0B1A6EF48F0F9D7FCEC61F0A8
:10915000230E9D632DEF44F09E6BF10EF76EBE0E55
:10916000F66E20EED6F0F5EC65F0F10EF76ECE0E51
:10917000F66E20EEE6F0F5EC65F0000E146207D016
:10918000320E7F6F350E806F300E816F20D0010E52
:10919000146207D0330E7F6F370E806F350E816FEC
:1091A00016D0020E146207D0340E7F6F300E806F1F
:1091B000300E816F0CD0030E146207D0350E7F6F16
:1091C000300E806F300E816F02D0146AD6D77FC008
:1091D000EEF080C0EFF081C0F0F013EC66F0640EAA
:1091E000B06F060EAF6F81B22DEF44F0A0B116EF55
:1091F00049F0AF67F8D7200EEE6FEF6FF06F13EC0A
:1092000066F0640EB06F020EAF6F81B22DEF44F0C6
:10921000A0B116EF49F0AF67F8D77FC0EEF080C07D
:10922000EFF081C0F0F013EC66F0D9D7FCEC61F000
:109230002A0E9D6308D0142A040E1460146A8EEC62
:1092400063F08E6F9AD7230E9D6397D79E6BF10EB6
:10925000F76EDE0EF66E20EED6F0F5EC65F0F10E50
:10926000F76EEE0EF66E20EEE6F0F5EC65F0000E11
:10927000156207D0320E7F6F350E806F300E816F12
:1092800020D0010E156207D0330E7F6F370E806F2E
:10929000350E816F16D0020E156207D0340E7F6F27
:1092A000300E806F300E816F0CD0030E156207D028
:1092B000350E7F6F300E806F300E816F02D0156AD1
:1092C000D6D77FC0EEF080C0EFF081C0F0F013EC95
:1092D00066F0640EB06F060EAF6F81B22DEF44F0F2
:1092E000A0B190EF49F0AF67F8D7200EEE6FEF6FA7
:1092F000F06F13EC66F0640EB06F020EAF6F81B2C8
:109300002DEF44F0A0B190EF49F0AF67F8D77FC0E0
:10931000EEF080C0EFF081C0F0F013EC66F0D9D72A
:10932000FCEC61F02A0E9D6308D0152A040E15602E
:10933000156A9DEC63F08F6F9AD7230E9D6397D7C4
:109340002DEF44F00C50030B816F000E816309D0A8
:10935000EF0EF76E7E0EF66E20EEE6F0F5EC65F0A1
:109360001200010E816309D0EF0EF76E8E0EF66EBD
:1093700020EEE6F0F5EC65F01200020E816309D0F4
:10938000EF0EF76E9E0EF66E20EEE6F0F5EC65F051
:109390001200FC0E0C16EF0EF76E7E0EF66E20EE2F
:1093A000E6F0F5EC65F01200640EAE6F0F0EAD6FD7
:1093B000AD67FED781B2ECEF5BF0E90EF76EBE0E43
:1093C000F66E20EED6F0F5EC65F0E90EF76ECE0EF7
:1093D000F66E20EEE6F0F5EC65F013EC66F081B287
:1093E00072EF35F0A0B1F6EF49F0F9D7FCEC61F07F
:1093F000230E9D635BEF4AF0E90EF76EDE0EF66E0C
:1094000020EED6F0F5EC65F016B609D0E90EF76E51
:10941000FE0EF66E20EEE6F0F5EC65F008D0E90EF3
:10942000F76EEE0EF66E20EEE6F0F5EC65F013EC5E
:1094300066F0640EB06F060EAF6F81B2D4EF49F0E4
:10944000A0B151EF4AF0AF67F8D7EA0EF76E0E0EF3
:10945000F66E20EEE6F0F5EC65F013EC66F0640EC7
:10946000B06F020EAF6F81B2D4EF49F0A0B151EFEF
:109470004AF0AF67F8D716B609D0E90EF76EFE0EC0
:10948000F66E20EEE6F0F5EC65F008D0E90EF76E2A
:10949000EE0EF66E20EEE6F0F5EC65F013EC66F0FD
:1094A000C8D7FCEC61F02A0E9D6302D01676ACD7CB
:1094B000230E9D63BED7EA0EF76E1E0EF66E20EEEB
:1094C000D6F0F5EC65F0EA0EF76E2E0EF66E20EE95
:1094D000E6F0F5EC65F013EC66F081B2D4EF49F0FC
:1094E000A0B174EF4AF0F9D7FCEC61F0230E9D6354
:1094F00027EF4BF0EA0EF76E2E0EF66E20EED6F04A
:10950000F5EC65F025EC57F013EC66F0640EAE6FE9
:10951000060EAD6F81B2D4EF49F0A0B1A9EF4AF0C9
:10952000AD67F8D7EA0EF76E7E0EF66E20EEE6F027
:10953000F5EC65F013EC66F0640EAE6F020EAD6FE5
:1095400081B2D4EF49F0A0B1A9EF4AF0AD67F8D7E6
:10955000D9D7FCEC61F02A0E9D6307D0FC0E1E16D5
:10956000812B030E81151E12CDD7230E9D63CAD702
:1095700025EC57F013EC66F0EA0EF76E8E0EF66EE1
:1095800020EED6F0F5EC65F009EC66F001EE60F047
:1095900011EED2F0100E8B6FEECFE6FF8B2FFCD7C3
:1095A0009E6B01EED2F010EEE6F0100E8B6FEECF58
:1095B000E6FF8B2FFCD713EC66F081B21BEF4BF06C
:1095C000A0B1E4EF4AF0F9D7FCEC61F02A0E9D63FC
:1095D0000AD0100E8B6F01EED2F0200EEE6E8B2FA4
:1095E000FCD79E6BDED7230E9D6301D019D09E67FA
:1095F00008D0100E8B6F01EED2F0200EEE6E8B2F86
:10960000FCD79E2B110E9E6106D09E5111EED1F01B
:109610009DC0E3FFC6D7AAEC34F0100E9E6FC1D7F1
:10962000100E8B6F01EED2F011EE60F0EECFE6FF80
:109630008B2FFCD70CD0100E8B6F01EED2F011EEF9
:1096400060F0EECFE6FF8B2FFCD7D4EF49F0EA0EA7
:10965000F76E9E0EF66E20EED6F0F5EC65F0EA0E93
:10966000F76EAE0EF66E20EEE6F0F5EC65F013EC5C
:1096700066F081B2D4EF49F0A0B140EF4BF0F9D7DA
:10968000FCEC61F0230E9D6374EF4BF0EA0EF76E75
:10969000BE0EF66E20EED6F0F5EC65F01EAC09D0ED
:1096A000EA0EF76ECE0EF66E20EEE6F0F5EC65F003
:1096B00008D0EA0EF76EDE0EF66E20EEE6F0F5EC60
:1096C00065F013EC66F081B2D4EF49F0A0B16AEF17
:1096D0004BF0F9D7FCEC61F02A0E9D6302D01E7CA2
:1096E000D5D7230E9D63DAD7EA0EF76EEE0EF66E2F
:1096F00020EED6F0F5EC65F0EA0EF76EFE0EF66E93
:1097000020EEE6F0F5EC65F013EC66F081B2D4EFF4
:1097100049F0A0B18DEF4BF0F9D7FCEC61F0230ECE
:109720009D6351EF4CF0EB0EF76E4E0EF66E20EE91
:10973000D6F0F5EC65F01EB609D0EB0EF76E5E0EB6
:10974000F66E20EEE6F0F5EC65F008D0EB0EF76E65
:109750006E0EF66E20EEE6F0F5EC65F013EC66F0BA
:10976000640EB06F060EAF6F81B2D4EF49F0A0B1B6
:10977000E8EF4BF0AF67F8D7EB0EF76E7E0EF66EA4
:1097800020EEE6F0F5EC65F013EC66F0640EB06FD9
:10979000020EAF6F81B2D4EF49F0A0B1E8EF4BF009
:1097A000AF67F8D71EB609D0EB0EF76E5E0EF66EF9
:1097B00020EEE6F0F5EC65F008D0EB0EF76E6E0EDD
:1097C000F66E20EEE6F0F5EC65F013EC66F0C8D727
:1097D000FCEC61F02A0E9D6302D01E76ACD7230EFE
:1097E0009D63A9D7EB0EF76E8E0EF66E20EED6F0C7
:1097F000F5EC65F02EB009D0EB0EF76E9E0EF66E0E
:1098000020EEE6F0F5EC65F008D0EB0EF76EAE0E4C
:10981000F66E20EEE6F0F5EC65F013EC66F0640E03
:10982000B06F060EAF6F81B2D4EF49F0A0B147EF31
:109830004CF0AF67F8D7EB0EF76EBE0EF66E20EE6B
:10984000E6F0F5EC65F013EC66F0640EB06F020E16
:10985000AF6F81B2D4EF49F0A0B147EF4CF0AF67E2
:10986000F8D72EB009D0EB0EF76E9E0EF66E20EEF6
:10987000E6F0F5EC65F008D0EB0EF76EAE0EF66E86
:1098800020EEE6F0F5EC65F013EC66F0C8D7FCECE2
:1098900061F02A0E9D6302D02E70ACD7230E9D631B
:1098A000A9D7EB0EF76ECE0EF66E20EED6F0F5ECE5
:1098B00065F0EB0EF76EDE0EF66E20EEE6F0F5ECE0
:1098C00065F013EC66F081B2D4EF49F0A0B16AEF15
:1098D0004CF0F9D7FCEC61F0230E9D63D1EF4CF016
:1098E000EB0EF76EEE0EF66E20EED6F0F5EC65F0B0
:1098F0001EB409D0EC0EF76E1E0EF66E20EEE6F0EA
:10990000F5EC65F008D0EC0EF76E0E0EF66E20EE5C
:10991000E6F0F5EC65F013EC66F0640EB06F060E41
:10992000AF6F81B2CFEF4CF0A0B1C5EF4CF0AF6795
:10993000F8D7EB0EF76EFE0EF66E20EEE6F0F5ECC5
:1099400065F013EC66F0640EB06F020EAF6F81B27B
:10995000CFEF4CF0A0B1C5EF4CF0AF67F8D71EB415
:1099600009D0EC0EF76E1E0EF66E20EEE6F0F5EC6A
:1099700065F008D0EC0EF76E0E0EF66E20EEE6F0F7
:10998000F5EC65F013EC66F0C8D7FCEC61F0230E43
:109990009D5D26E02A0E9D63C0D71E74A9D7D4EF23
:1099A00049F0EC0EF76E2E0EF66E20EED6F0F5ECCA
:1099B00065F0EC0EF76E3E0EF66E20EEE6F0F5EC7E
:1099C00065F013EC66F081B2D4EF49F0A0B1EAEF94
:1099D0004CF0F9D7FCEC61F0230E9D63DAEF4FF009
:1099E000EC0EF76E4E0EF66E20EED6F0F5EC65F04E
:1099F000EC0EF76E5E0EF66E20EEE6F0F5EC65F01E
:109A000013EC66F081B2D4EF49F0A0B109EF4DF04C
:109A1000F9D7FCEC61F0230E9D5D05E02A0E9D63F5
:109A2000F1D7ACEF4FF0A26B2EEC5DF0EC0EF76EC1
:109A30006E0EF66E20EEE6F0F5EC65F015EE00F039
:109A400001EED2F00A0EA203F350E126F450E22216
:109A5000FF0EE76205D0780EE8CFD2F13C6A22D043
:109A6000080ECB6F200E806FE7380F0B300F816F21
:109A70003F0E816180C081F03B0E816302D02B0ECE
:109A8000816F81C0EEFFE6500F0B9A6F300F816F30
:109A90003F0E816180C081F081C0EEFFCB2FE4D703
:109AA000E6CF3CF0100ECB6F11EED2F000EED6F008
:109AB000E6CFEEFFCB2FFCD74E0E3CB0590EF16F28
:109AC0004E0E3CB2590EF26F4E0E3CB4590EF36F6F
:109AD0004E0E3CB6590EF46F4E0E3CB8590EF56F53
:109AE000826BA2C083F0832B75EC61F080C0E7F03D
:109AF00081C0E8F013EC66F081B27EEF4FF0A0B1C8
:109B000083EF4DF0F9D7FCEC61F0230E9D5D1EE074
:109B10002A0E9D5D20E0370E9D5D18E0380E9D5D9C
:109B200015E0390E9D5D12E0310E9D5D07E0320EAD
:109B30009D5D04E0330E9D5D01E0DED7A2073F0E80
:109B4000CB6F400EA261CBC0A2F06ED7A22B400E0D
:109B5000A261A26B69D79E6B640EB06F060EAF6FE9
:109B600081B27EEF4FF0A0B1DBEF4DF0AF67F8D7D9
:109B700010EED6F0100ECB6F200EE66ECB2FFDD779
:109B800013EC66F0640EB06F020EAF6F81B27EEF21
:109B90004FF0A0B1DBEF4DF0AF67F8D711EED2F088
:109BA00000EED6F0100ECB6FE6CFEEFFCB2FFCD73A
:109BB00013EC66F0D1D7FCEC61F0230E9D5DD8B4B8
:109BC00050D02A0E9D6312D02EEC5DF0780EE8CFB7
:109BD000D2F1100ECB6F11EED2F000EED6F0E6CF40
:109BE000EEFFCB2FFCD713EC66F0B5D79E6702D003
:109BF0002EEC5DF00F0E9E6120D0010E9E630AD008
:109C0000300E9D6307D011EED2F0E76203D09E6B59
:109C10002B0E9D6F11EED2F09E519DC0E3FF00EE22
:109C2000D6F011EED2F0100ECB6FE6CFEEFFCB2FB9
:109C3000FCD713EC66F09E2B8FD7AAEC34F02EECF9
:109C40005DF0780EE8CFD2F100EED6F011EED2F052
:109C5000100ECB6FE6CFEEFFCB2FFCD713EC66F0E8
:109C60007AD711EED2F000EED6F0100ECB6FE6CF21
:109C7000EEFFCB2FFCD713EC66F0640EB06F060E30
:109C8000AF6F81B27EEF4FF0A0B160EF4EF0AF67E3
:109C9000F8D7200EF16F13EC66F0640EB06F020E71
:109CA000AF6F81B27EEF4FF0A0B160EF4EF0AF67C3
:109CB000F8D74E0E3CB0590EF16F13EC66F0DDD7BD
:109CC000FCEC61F02A0E9D6308D03C704E0E3CB057
:109CD000590EF16F13EC66F0D0D7230E9D63CDD7EC
:109CE0004E0E3CB0590EF16F640EB06F060EAF6FA2
:109CF00081B27EEF4FF0A0B197EF4EF0AF67F8D78B
:109D0000200EF26F13EC66F0640EB06F020EAF6FB0
:109D100081B27EEF4FF0A0B197EF4EF0AF67F8D76A
:109D20004E0E3CB2590EF26F13EC66F0DDD7FCEC30
:109D300061F02A0E9D6308D03C724E0E3CB2590E63
:109D4000F26F13EC66F0D0D7230E9D63CDD74E0E85
:109D50003CB2590EF26F640EB06F060EAF6F81B257
:109D60007EEF4FF0A0B1CEEF4EF0AF67F8D7200EE8
:109D7000F36F13EC66F0640EB06F020EAF6F81B23A
:109D80007EEF4FF0A0B1CEEF4EF0AF67F8D74E0E9A
:109D90003CB4590EF36F13EC66F0DDD7FCEC61F0C8
:109DA0002A0E9D6308D03C744E0E3CB4590EF36FDE
:109DB00013EC66F0D0D7230E9D63CDD74E0E3CB486
:109DC000590EF36F640EB06F060EAF6F81B27EEF67
:109DD0004FF0A0B105EF4FF0AF67F8D7200EF46F4A
:109DE00013EC66F0640EB06F020EAF6F81B27EEFBF
:109DF0004FF0A0B105EF4FF0AF67F8D74E0E3CB66D
:109E0000590EF46F13EC66F0DDD7FCEC61F02A0E0E
:109E10009D6308D03C764E0E3CB6590EF46F13ECA1
:109E200066F0D0D7230E9D63CDD74E0E3CB6590EAB
:109E3000F46F640EB06F060EAF6F81B27EEF4FF01D
:109E4000A0B13CEF4FF0AF67F8D7200EF56F13ECE1
:109E500066F0640EB06F020EAF6F81B27EEF4FF00E
:109E6000A0B13CEF4FF0AF67F8D74E0E3CB8590E9B
:109E7000F56F13EC66F0DDD7FCEC61F02A0E9D6304
:109E800008D03C784E0E3CB8590EF56F13EC66F0D6
:109E9000D0D7230E9D63CDD74E0E3CB8590EF56F2B
:109EA00005EE00F011EED2F00A0EA203F350E926FF
:109EB000F450EA22780EE7620BD0FF0EEE6EEE6EE3
:109EC000EE6EEE6EEE6EEE6EEE6EEE6EEE6A3ED6FE
:109ED000080ECB6F11EED2F0200EE764E768E6388B
:109EE000F00B816F200EE764E7680F0EE614811116
:109EF000EE6ECB2FF1D73CC0EEFF28D605EE00F07A
:109F000011EED2F00A0EA203F350E926F450EA2231
:109F1000780EE7620CD0FF0EEE6EEE6EEE6EEE6E19
:109F2000EE6EEE6EEE6EEE6EEE6AD4EF49F0080E57
:109F3000CB6F200EE764E768E638F00B816F200EE8
:109F4000E764E7680F0EE6148111EE6ECB2FF1D7B0
:109F50003CC0EEFFD4EF49F0A26B15EE00F00A0E04
:109F6000A203F350E126F450E222FF0EE75CD8B4DE
:109F700014EF4DF0A22B3F0EA265EFD7EC0EF76E5B
:109F80007E0EF66E20EED6F0F5EC65F0EC0EF76E78
:109F90008E0EF66E20EEE6F0F5EC65F013EC66F052
:109FA000AAEC34F0640EAE6F140EAD6FAD67FED741
:109FB00013EF4DF0EC0EF76E9E0EF66E20EED6F01F
:109FC000F5EC65F0EC0EF76EAE0EF66E20EEE6F0F8
:109FD000F5EC65F013EC66F081B2D4EF49F0A0B176
:109FE000F3EF4FF0F9D7FCEC61F0230E9D6343EFE4
:109FF00050F0EC0EF76EBE0EF66E20EED6F0F5ECDD
:10A0000065F024BC09D0EC0EF76ECE0EF66E20EE95
:10A01000E6F0F5EC65F008D0EC0EF76EDE0EF66EAD
:10A0200020EEE6F0F5EC65F013EC66F0640EAE6F32
:10A03000060EAD6F81B2DDEF49F0A0B139EF50F0FF
:10A04000AD67F8D7EC0EF76EEE0EF66E20EEE6F08A
:10A05000F5EC65F013EC66F0640EAE6F020EAD6FBA
:10A0600081B2DDEF49F0A0B139EF50F0AD67F8D71C
:10A07000C8D7FCEC61F02A0E9D6302D0247CC1D7C6
:10A08000230E9D63D3D7EC0EF76EFE0EF66E20EE18
:10A09000D6F0F5EC65F0ED0EF76E0E0EF66E20EED6
:10A0A000E6F0F5EC65F013EC66F081B2D4EF49F020
:10A0B000A0B15CEF50F0F9D7FCEC61F0230E9D638A
:10A0C000C2D0ED0EF76E1E0EF66E20EED6F0F5EC59
:10A0D00065F01E389A6F030E9A17000E9A630AD025
:10A0E0009A6BED0EF76E2E0EF66E20EEE6F0F5ECA6
:10A0F00065F017D0010E9A6309D0ED0EF76E3E0E93
:10A10000F66E20EEE6F0F5EC65F00BD0020E9A63E9
:10A11000E7D7ED0EF76E4E0EF66E20EEE6F0F5EC9C
:10A1200065F013EC66F0640EB06F060EAF6F81B28F
:10A13000DDEF49F0A0B1B0EF50F0AF67F8D709EC10
:10A1400066F013EC66F0640EB06F020EAF6F81B272
:10A15000DDEF49F0A0B1B0EF50F0AF67F8D7B9D755
:10A16000FCEC61F02A0E9D630AD09A2B030E9A61D3
:10A170009A6BCF0E1E169A391E123886AAD7230E56
:10A180009D63D1D7ED0EF76E5E0EF66E20EED6F023
:10A19000F5EC65F01EAE09D0ED0EF76E6E0EF66EA4
:10A1A00020EEE6F0F5EC65F008D0ED0EF76E7E0ED1
:10A1B000F66E20EEE6F0F5EC65F013EC66F0640E5A
:10A1C000B06F060EAF6F81B2D4EF49F0A0B117EFB8
:10A1D00051F0AF67F8D7ED0EF76E8E0EF66E20EEEB
:10A1E000E6F0F5EC65F013EC66F0640EB06F020E6D
:10A1F000AF6F81B2D4EF49F0A0B117EF51F0AF6764
:10A20000F8D71EAE09D0ED0EF76E6E0EF66E20EE8C
:10A21000E6F0F5EC65F008D0ED0EF76E7E0EF66E0A
:10A2200020EEE6F0F5EC65F013EC66F0C8D7FCEC38
:10A2300061F02A0E9D6302D01E7EACD7230E9D6373
:10A24000BED7DDEF49F0ED0EF76E9E0EF66E20EEF6
:10A25000D6F0F5EC65F0ED0EF76EAE0EF66E20EE74
:10A26000E6F0F5EC65F013EC66F081B2D4EF49F05E
:10A27000A0B13CEF51F0F9D7FCEC61F0230E9D63E7
:10A28000DDEF49F0ED0EF76EBE0EF66E20EED6F065
:10A29000F5EC65F02438816F030E811781670CD0CF
:10A2A000CF0E2416816BED0EF76ECE0EF66E20EEFD
:10A2B000E6F0F5EC65F017D0010E816309D0ED0EE4
:10A2C000F76EDE0EF66E20EEE6F0F5EC65F00BD0E4
:10A2D000020E8163E5D7EE0EF76E0E0EF66E20EEDF
:10A2E000E6F0F5EC65F013EC66F081B2D4EF49F0DE
:10A2F000A0B17CEF51F0F9D7FCEC61F02A0E9D6320
:10A300000AD06487812B030E8161816BCF0E2416E6
:10A3100081392412BFD7230E9D63E7D7000E815DDC
:10A32000D8B425D2010E815DD8B489D0020E8163E4
:10A330001ED2EE0EF76E1E0EF66E20EED6F0F5EC87
:10A3400065F0EE0EF76E2E0EF66E20EEE6F0F5ECF2
:10A3500065F09E6B9AC9F0F09BC9F1F09CC9F2F0D0
:10A360009DC9F3F09EC9F4F09FC9F5F013EC66F0B7
:10A37000640EB06F060EAF6F81B2D4EF49F0A0B19A
:10A38000E8EF51F0AF67F8D7200EF06FF16FF26F82
:10A39000F36FF46FF56F13EC66F0640EB06F020E9E
:10A3A000AF6F81B2D4EF49F0A0B1E8EF51F0AF67E1
:10A3B000F8D79AC9F0F09BC9F1F09CC9F2F09DC999
:10A3C000F3F09EC9F4F09FC9F5F013EC66F0D0D716
:10A3D000FCEC61F02A0E9D6310D09E6B200EE8CF3E
:10A3E0009AF9E8CF9BF9E8CF9CF9E8CF9DF9E8CF3F
:10A3F0009EF9E8CF9FF96487ADD7230E9D5DD8B451
:10A40000B8D19E670DD0200EE8CF9AF9E8CF9BF91E
:10A41000E8CF9CF9E8CF9DF9E8CF9EF9E8CF9FF906
:10A42000060E9E6108D009EE9AF09E519DC0EBFF8A
:10A430009E2B64878FD7AAEC34F09E6B8BD7ED0EE2
:10A44000F76EEE0EF66E20EED6F0F5EC65F0ED0E42
:10A45000F76EFE0EF66E20EEE6F0F5EC65F09E6B04
:10A46000A26B310EA225D66F19EEA2F0080EA20340
:10A47000F350E126F450E222E6CFE0F0E6CFE1F03F
:10A48000E6CFE2F0E6CFE3F0E6CFE4F0E6CFE5F0AA
:10A49000E6CF83F0E6CF82F075EC61F07DC0F1F09D
:10A4A0007EC0F2F07FC0F3F080C0F4F081C0F5F020
:10A4B00013EC66F081B2D4EF49F0A0B161EF52F035
:10A4C000F9D7FCEC61F02A0E9D6305D0A22B040E97
:10A4D000A2614FD1C6D7230E9D63ECD79E6BA26BB2
:10A4E000310EA225D66F19EEA2F0080EA203F3508A
:10A4F000E126F450E222E6CFE0F0E6CFE1F0E6CF4D
:10A50000E2F0E6CFE3F0E6CFE4F0E6CFE5F0E6CF29
:10A5100083F0E6CF82F075EC61F07DC0F1F07EC093
:10A52000F2F07FC0F3F080C0F4F081C0F5F013ECDE
:10A5300066F0640EB06F060EAF6F81B2D4EF49F0D3
:10A54000A0B1D1EF52F0AF67F8D7200EE06FE16F06
:10A55000E26FE36FE46FE56F13EC66F0640EB06FCB
:10A56000020EAF6F81B2D4EF49F0A0B1D1EF52F03B
:10A57000AF67F8D719EEA2F0080EA203F350E12658
:10A58000F450E222E6CFE0F0E6CFE1F0E6CFE2F0F1
:10A59000E6CFE3F0E6CFE4F0E6CFE5F013EC66F0CB
:10A5A000C8D7FCEC61F02A0E9D6311D09E6B19EEAA
:10A5B000A2F0080EA203F350E126F450E222200E8E
:10A5C000E66EE66EE66EE66EE66EE66E89D7230E02
:10A5D0009D5D25E09E670FD019EEA2F0080EA20344
:10A5E000F350E126F450E222200EE66EE66EE66EAF
:10A5F000E66EE66EE66E060E9E610DD019EEA2F0D6
:10A60000080EA203F350E126F450E2229E519DC0B1
:10A61000E3FF9E2B65D7AAEC34F09E6B61D719EE51
:10A62000A2F0080EA203F350E126F450E222E6CF96
:10A63000E0F0E6CFE1F0E6CFE2F0E6CFE3F0E6CF00
:10A64000E4F0E6CFE5F013EC66F019EEA8F0080EA2
:10A65000A203F350E126F450E222E6CF83F0E5CFE7
:10A6600082F075EC61F07DC0F1F07EC0F2F07FC049
:10A67000F3F080C0F4F081C0F5F013EC66F09E6B4F
:10A68000640EB06F060EAF6F81B2D4EF49F0A0B187
:10A6900073EF53F0AF67F8D7200EF16FF26FF36FDF
:10A6A000F46FF56F13EC66F0640EB06F020EAF6FCF
:10A6B00081B2D4EF49F0A0B173EF53F0AF67F8D790
:10A6C000E6CF83F0E5CF82F075EC61F07DC0F1F06C
:10A6D0007EC0F2F07FC0F3F080C0F4F081C0F5F0EE
:10A6E00013EC66F0CDD7FCEC61F02A0E9D6303D02D
:10A6F000E66AE56AAAD7230E9D5DD8B432D09E677C
:10A7000008D0E66AE56A300E7D6F7E6F7F6F806FDE
:10A71000816F7EC07DF07FC07EF080C07FF081C001
:10A7200080F09DC081F07DC075F07EC076F07FC066
:10A7300077F080C078F081C079F01EEC61F083C0C2
:10A74000E6FF82C0E5FF9E2B7DC0F1F07EC0F2F0F7
:10A750007FC0F3F080C0F4F081C0F5F013EC66F038
:10A760008FD7A22B040EA26104D09E6BB9D6CF0E58
:10A770002416EE0EF76E4E0EF66E20EED6F0F5ECC9
:10A7800065F0EE0EF76E5E0EF66E20EEE6F0F5EC7E
:10A7900065F09E6B28C0F0F029C0F1F02AC0F2F0FD
:10A7A0002BC0F3F02CC0F4F02DC0F5F013EC66F0E4
:10A7B000640EB06F060EAF6F81B2D4EF49F0A0B156
:10A7C00008EF54F0AF67F8D7200EF06FF16FF26F1B
:10A7D000F36FF46FF56F13EC66F0640EB06F020E5A
:10A7E000AF6F81B2D4EF49F0A0B108EF54F0AF677A
:10A7F000F8D728C0F0F029C0F1F02AC0F2F02BC041
:10A80000F3F02CC0F4F02DC0F5F013EC66F0D0D7C7
:10A81000FCEC61F02A0E9D630AD09E6B300E286E10
:10A82000200E296E2A6E2B6E2C6E2D6EB3D7230E42
:10A830009D5D1DE09E670DD0200EE8CF28F0E8CF8B
:10A8400029F0E8CF2AF0E8CF2BF0E8CF2CF0E8CFC2
:10A850002DF0060E9E6107D010EE28F09E519DC08F
:10A86000E3FF9E2B97D7AAEC34F09E6B93D7200E74
:10A87000286202D0300E286EEE0EF76E3E0EF66E97
:10A8800020EED6F0F5EC65F024C081F0030E8117C0
:10A89000000E81630BD0FC0E2416EE0EF76E6E0ECA
:10A8A000F66E20EEE6F0F5EC65F017D0010E816350
:10A8B00009D0EE0EF76E7E0EF66E20EEE6F0F5ECA9
:10A8C00065F00BD0020E8163E6D7EE0EF76E9E0E9A
:10A8D000F66E20EEE6F0F5EC65F013EC66F081B272
:10A8E0007BEF54F0A0B176EF54F0F9D7FCEC61F0B7
:10A8F000230E9D6305D024C081F0030E81170CD078
:10A900002A0E9D63ECD7812B030E8161816BFC0EB7
:10A91000241681512412B8D7000E81631FD03D90B8
:10A920003D92E00EF76E8E0EF66E23EE00F0EEEC2A
:10A9300065F0DE6ADFEC65F0640EAE6F640EAD6F3D
:10A940003DB0ABEF54F03DB2A8EF54F0AD67F8D78F
:10A950003D9293EF08F03D90DDEF49F0010E8163E9
:10A9600023D1EE0EF76E8E0EF66E20EEE6F0F5ECCD
:10A9700065F026C083F027C082F075EC61F07DC0E1
:10A98000EAF07EC0EBF07FC0ECF080C0EDF081C05B
:10A99000EEF025C084F059EC61F07FC0F3F080C088
:10A9A000F4F081C0F5F013EC66F09E6B640EB06FAE
:10A9B000060EAF6F81B2D4EF49F0A0B109EF55F0A8
:10A9C000AF67F8D7200EEA6FEB6FEC6FED6FEE6FAD
:10A9D00013EC66F0640EB06F020EAF6F81B2D4EF6D
:10A9E00049F0A0B109EF55F0AF67F8D726C083F062
:10A9F00027C082F075EC61F07DC0EAF07EC0EBF01C
:10AA00007FC0ECF080C0EDF081C0EEF013EC66F09A
:10AA1000CDD7FCEC61F02A0E9D6303D0266A276A2D
:10AA2000A8D7230E9D6306D0276639D0090E266469
:10AA300033D035D09E6708D0266A276A300E7D6FE6
:10AA40007E6F7F6F806F816F7EC07DF07FC07EF0F4
:10AA500080C07FF081C080F09DC081F07DC075F026
:10AA60007EC076F07FC077F080C078F081C079F04A
:10AA70001EEC61F083C026F082C027F09E2B7DC0C3
:10AA8000EAF07EC0EBF07FC0ECF080C0EDF081C05A
:10AA9000EEF013EC66F08AD7AAEC34F06AD726C041
:10AAA00083F027C082F075EC61F07DC0EAF07EC0D3
:10AAB000EBF07FC0ECF080C0EDF081C0EEF025C07F
:10AAC00084F059EC61F07FC0F3F080C0F4F081C0F5
:10AAD000F5F013EC66F09E6B640EB06F060EAF6F70
:10AAE00081B2D4EF49F0A0B197EF55F0AF67F8D736
:10AAF000200EF36FF46FF56F13EC66F0640EB06F19
:10AB0000020EAF6F81B223EF51F0A0B197EF55F075
:10AB1000AF67F8D725C084F059EC61F07FC0F3F03F
:10AB200080C0F4F081C0F5F013EC66F0D5D7FCECF2
:10AB300061F02A0E9D6302D0256AC1D7230E9D6362
:10AB400007D0090E25641FD0700E25601CD01ED0C2
:10AB50009E6705D0256A300E7F6F806F816F80C041
:10AB60007FF081C080F09DC081F00FEC61F084C067
:10AB700025F09E2B7FC0F3F080C0F4F081C0F5F08B
:10AB800013EC66F0A9D7AAEC34F099D725C084F06D
:10AB900059EC61F07FC0F3F080C0F4F081C0F5F0B3
:10ABA00013EC66F0DDEF49F064933EEC5DF03D9010
:10ABB0003D92E00EF76E800EF66E23EE00F0EEECA6
:10ABC00065F0DE6ADFEC65F0640EAE6F640EAD6FAB
:10ABD0003DB00DEF56F03DB2F0EF55F0AD67F8D750
:10ABE0003D92EE0EF76EAE0EF66E20EED6F0F5EC60
:10ABF00065F0EE0EF76EBE0EF66E20EEE6F0F5ECAA
:10AC000065F013EC66F0AAEC34F0640EAE6F140E2F
:10AC1000AD6FAD67FED7DDEF49F0EE0EF76ECE0EED
:10AC2000F66E20EED6F0F5EC65F0EE0EF76EDE0E69
:10AC3000F66E20EEE6F0F5EC65F0070E976FCB6B45
:10AC400019EE00F0300ECB25D66F160ECB03F35065
:10AC5000E126F450E226E6CFE8F0E6CFE9F0E6CFD1
:10AC6000EAF0E6CFEBF0E6CFECF0E6CFEDF0E6CFA2
:10AC7000DBF0E6CFDCF0E6CFDDF0E6CFDEF0E6504D
:10AC8000E650E650E650E6CFF2F0E6CFF3F0E6CF3E
:10AC9000F4F0E6CFF5F0E6CFE3F0E6CFE3F0E6CF71
:10ACA000E4F0E6CFE5F013EC66F081B25CEF56F02D
:10ACB000A0B15EEF56F0F9D7DDEF49F0FCEC61F0A2
:10ACC0002A0E9D6304D0CB2B972FBAD7B6D7230E6D
:10ACD0009D636AD719EE00F0160ECB03F350E12600
:10ACE000F450E226200EE76220D0EE0EF76EEE0E54
:10ACF000F66E20EED6F0F5EC65F0EE0EF76EFE0E79
:10AD0000F66E20EEE6F0F5EC65F013EC66F081B23D
:10AD100091EF56F0A0B191EF56F0F9D7FC0E241642
:10AD2000FED5FC0E241623EF51F0EF0EF76E0E0E3B
:10AD3000F66E20EED6F0F5EC65F0EF0EF76E1E0E17
:10AD4000F66E20EEE6F0F5EC65F013EC66F019EE29
:10AD50000EF0160ECB03F350E126F450E22603EE7C
:10AD600000F0410EEE6E540EEE6E2B0EEE6E430EA4
:10AD7000EE6EEE6E450EEE6E4C0EEE6EEE6E3D0E0F
:10AD8000EE6EE6CFEEFFE6CFEEFFE6CFEEFFE6CFCC
:10AD9000EEFFEE6A5A6A6493DFEC65F0640EAE6F04
:10ADA000C80EAD6F5AB007EF57F05AB2E6EF56F043
:10ADB0005AB4E6EF56F05AB6E6EF56F05AB807EF37
:10ADC00057F05ABAE6EF56F0AD67ECD7AAEC34F07C
:10ADD0005A6AEE0EF76EEE0EF66E20EED6F0F5EC39
:10ADE00065F0EE0EF76EFE0EF66E20EEE6F0F5EC78
:10ADF00065F013EC66F081B202EF57F0A0B102EFFC
:10AE000057F0F9D7FCEC61F0FC0E241688D564836A
:10AE1000EF0EF76E2E0EF66E20EED6F0F5EC65F026
:10AE2000EF0EF76E3E0EF66E20EEE6F0F5EC65F0F6
:10AE300013EC66F081B223EF51F0A0B121EF57F08F
:10AE4000F9D7FCEC61F023EF51F01E50030B816F3A
:10AE5000000E816309D0EA0EF76E3E0EF66E20EE0C
:10AE6000E6F0F5EC65F01200010E816309D0EA0E00
:10AE7000F76E4E0EF66E20EEE6F0F5EC65F0120081
:10AE8000020E816309D0EA0EF76E5E0EF66E20EEBA
:10AE9000E6F0F5EC65F01200030E816309D0EA0ECE
:10AEA000F76E6E0EF66E20EEE6F0F5EC65F0120031
:10AEB000FC0E1E16EA0EF76E3E0EF66E20EEE6F063
:10AEC000F5EC65F01200640EAE6F0F0EAD6FAD675E
:10AED000FED781B2ECEF5BF0E80EF76E3E0EF66E39
:10AEE00020EED6F0F5EC65F0E80EF76E4E0EF66E3D
:10AEF00020EEE6F0F5EC65F013EC66F081B272EF4F
:10AF000035F0A0B185EF57F0F9D7FCEC61F0230ED6
:10AF10009D6378EF59F0E90EF76E1E0EF66E20EE87
:10AF2000D6F0F5EC65F0E90EF76E2E0EF66E20EE1B
:10AF3000E6F0F5EC65F08B6B9E6B826B8BC083F05B
:10AF4000832B75EC61F0200ED76F80C0D8F081C0E4
:10AF5000D9F004EE40F0040E8B03F350E926E86AC2
:10AF6000EA22EF380F0B7A6FEE500F0B7B6FEF3842
:10AF70000F0B7C6FEE500F0B7D6FEF380F0B7E6F5A
:10AF8000EE500F0B7F6FEF380F0B806FEE500F0BF3
:10AF9000816F22EC59F013EC66F081B2F8EF58F0B3
:10AFA000A0B1D4EF57F0F9D7FCEC61F0230E9D630C
:10AFB00005D08B2B200E8B618B6BBED72A0E9D5D2F
:10AFC00020E0370E9D5D18E0380E9D5D15E0390ECE
:10AFD0009D5D12E0310E9D5D07E0320E9D5D04E047
:10AFE000330E9D5D01E0D9D78B071F0ECB6F200E6E
:10AFF0008B61CBC08BF0A0D78B2B200E8B618B6B22
:10B000009BD79E6B640EB06F060EAF6F81B24DEF93
:10B0100058F0A0B12BEF58F0AF67F8D7200EE56FCE
:10B0200013EC66F0640EB06F020EAF6F81B24DEF9D
:10B0300058F0A0B12BEF58F0AF67F8D7480E9A6FD1
:10B040000F0E816381C09AF09AC0E5F0300EE527BB
:10B0500013EC66F0D7D7FCEC61F02A0E9D6307D0A5
:10B060000F0E816F780EE56F13EC66F0CAD7230ED2
:10B070009D5D13E0300E9D650DD0330E9D610AD0AD
:10B080000F0E9D15816F81C0E5F0300EE52713ECA2
:10B0900066F0B7D7AAEC34F0E3D7480E9A6F0F0EDC
:10B0A000816381C09AF09AC0E5F0300EE52713EC79
:10B0B00066F09E6B640EB06F060EAF6F81B2F8EF54
:10B0C00058F0A0B181EF58F0AF67F8D7200EEF6FBE
:10B0D000F06FF16FF26FF36FF46FF56F13EC66F0D2
:10B0E000640EB06F020EAF6F81B2F8EF58F0A0B1EE
:10B0F00081EF58F0AF67F8D722EC59F013EC66F007
:10B10000D9D7FCEC61F0230E9D5D4AE02A0E9D5DCF
:10B110000FE19E530DE00F0E7A6F7B6F7C6F7D6F9A
:10B120007E6F7F6F806F22EC59F013EC66F0C1D711
:10B130009E5308E10F0E7A6F7B6F7C6F7D6F7E6F81
:10B140007F6F806F070E9E611CD0010E9E6309D039
:10B15000300E9D6306D0000E7A6303D09E6B0B0EFB
:10B160009D6F0F0E9D1710EE7AF09E51E126E86A52
:10B17000E2229DC0E3FF22EC59F09E2B13EC66F017
:10B1800099D7AAEC34F00F0E7A6F7B6F7C6F7D6FCE
:10B190007E6F7F6F806F22EC59F013EC66F089D7D9
:10B1A00014EE40F0040E8B03F350E126E86AE2222D
:10B1B000200E7A6307D0FF0EE66EE66EE66EF00EA6
:10B1C000E66EF7D60F0E7A177B177C177D177E1762
:10B1D0007F17801781177A397B11E66E7C397D11D4
:10B1E000E66E7E397F11E66E80398111E66EE1D61A
:10B1F00014EE40F0040E8B03F350E126E86AE222DD
:10B20000780E7A6308D0FF0EE66EE66EE66EF00EFC
:10B21000E66E63EF57F00F0E7A177B177C177D17DA
:10B220007E177F17801781177A397B11E66E7C397C
:10B230007D11E66E7E397F11E66E80398111E66EF2
:10B2400063EF57F0480E9A6F0F0E816381C09AF03A
:10B250009AC0E5F00A0E7A6303D0FA0E9A6F0CD00A
:10B260000B0E7A6303D0FB0E9A6F06D0480E9A6FCE
:10B270000F0E7A637AC09AF09AC0EFF0F00E9A6FD0
:10B280000F0E7B637BC09AF09AC0F0F0F00E9A6FBD
:10B290000F0E7C637CC09AF09AC0F1F0F00E9A6FAA
:10B2A0000F0E7D637DC09AF09AC0F2F0F00E9A6F97
:10B2B0000F0E7E637EC09AF09AC0F3F0F00E9A6F84
:10B2C0000F0E7F637FC09AF09AC0F4F0F00E9A6F71
:10B2D0000F0E806380C09AF09AC0F5F0300EE5271B
:10B2E000EF27F027F127F227F327F427F52712009D
:10B2F000E80EF76E5E0EF66E20EED6F0F5EC65F019
:10B30000E80EF76E6E0EF66E20EEE6F0F5EC65F0E8
:10B3100013EC66F081B263EF57F0A0B191EF59F0F2
:10B32000F9D7FCEC61F0230E9D6301EF5AF0640E37
:10B33000AE6FFA0EAD6FE90EF76E3E0EF66E20EEB2
:10B34000D6F0F5EC65F0E90EF76E4E0EF66E20EED7
:10B35000E6F0F5EC65F017C084F059EC61F010EE02
:10B36000E8F080C0E6FF2E0EE66E81C0E6FF13EC2B
:10B3700066F0640EB06F060EAF6F81B2FFEF59F04A
:10B38000A0B1E4EF59F0AF67F8D710EEE8F0200E67
:10B39000E66EE66EE66E13EC66F0640EB06F020EBB
:10B3A000AF6F81B2FFEF59F0A0B1E4EF59F0AF6792
:10B3B000F8D710EEE8F080C0E6FF2E0EE66E81C0F2
:10B3C000E6FF13EC66F0D5D7FCEC61F0230E9D5D33
:10B3D00016E02A0E9D6305D0050E846F84C017F019
:10B3E000BAD717C084F0050E8427370E846103D0C6
:10B3F00084C017F0B0D7320EE8CF17F0ACD763EFA8
:10B4000057F0E80EF76E7E0EF66E20EED6F0F5ECF5
:10B4100065F0E80EF76E8E0EF66E20EEE6F0F5ECB7
:10B4200065F013EC66F081B263EF57F0A0B11AEF4C
:10B430005AF0F9D7FCEC61F0230E9D63C5EF5AF08A
:10B44000A7EC5AF093EC5AF013EC66F0640EB06F70
:10B45000060EAF6F81B291EF5AF0A0B149EF5AF0EA
:10B46000AF67F8D7200EE36FE46FE56F13EC66F07B
:10B47000640EB06F020EAF6F81B291EF5AF0A0B1BF
:10B4800049EF5AF0AF67F8D793EC5AF013EC66F037
:10B49000DDD7FCEC61F02A0E9D6302D01674D2D782
:10B4A000230E9D63D3D793EC5AF0640EB06F060E53
:10B4B000AF6F81B291EF5AF0A0B17CEF5AF0AF6755
:10B4C000F8D7E80EF76EEE0EF66E20EEE6F0F5EC2D
:10B4D00065F013EC66F0640EB06F020EAF6F81B2D0
:10B4E00091EF5AF0A0B17CEF5AF0AF67F8D7A7EC14
:10B4F0005AF013EC66F0D9D7FCEC61F02A0E9D638C
:10B500000CD09A2B030E9A171650FC0B9A11166E3C
:10B51000A7EC5AF013EC66F0C8D7230E9D63C5D78D
:10B520008FD763EF57F016B409D0E80EF76EAE0E62
:10B53000F66E20EED6F0F5EC65F01200E80EF76E30
:10B540009E0EF66E20EED6F0F5EC65F01200165069
:10B55000030B9A6F000E9A6309D0E80EF76EBE0EC9
:10B56000F66E20EEE6F0F5EC65F00ED0010E9A6373
:10B5700009D0E80EF76ECE0EF66E20EEE6F0F5EC92
:10B5800065F002D09A6BE9D71200E80EF76EFE0E56
:10B59000F66E20EED6F0F5EC65F0E90EF76E0E0EC5
:10B5A000F66E20EEE6F0F5EC65F013EC66F081B295
:10B5B00063EF57F0A0B1DEEF5AF0F9D7FCEC61F081
:10B5C000230E9D636CEF57F08FEC34F0E90EF76EAD
:10B5D0005E0EF66E20EED6F0F5EC65F018C0A2F027
:10B5E000000EA26309D0E90EF76E6E0EF66E20EE25
:10B5F000E6F0F5EC65F02ED0010EA26309D0E90E5D
:10B60000F76E7E0EF66E20EEE6F0F5EC65F022D0D9
:10B61000020EA26309D0E90EF76E8E0EF66E20EED2
:10B62000E6F0F5EC65F016D0030EA26309D0E90E42
:10B63000F76E9E0EF66E20EEE6F0F5EC65F00AD0A1
:10B64000A26B186AE90EF76E6E0EF66E20EEE6F04B
:10B65000F5EC65F013EC66F0640EB06F060EAF6F9C
:10B6600081B2EAEF5BF0A0B152EF5BF0A251186239
:10B67000F3D7AF67F5D710EEEBF00B0ECB6F200EC4
:10B68000E66ECB2FFDD713EC66F0640EB06F020EA2
:10B69000AF6F81B2EAEF5BF0A0B152EF5BF0AF6742
:10B6A000F8D79ED7FCEC61F02A0E9D6305D0A22B43
:10B6B000040EA261A26B94D7230E9D6391D7A2C002
:10B6C00018F0010EA2658CD7020EA26309D0E90E14
:10B6D000F76E8E0EF66E20EED6F0F5EC65F00BD020
:10B6E000030EA26308D0E90EF76E9E0EF66E20EEF2
:10B6F000D6F0F5EC65F0E90EF76EAE0EF66E20EEC4
:10B70000E6F0F5EC65F0826B19C083F075EC61F042
:10B710009E6B200EF46F300E806380C0F4F081C009
:10B72000F5F013EC66F0640EB06F060EAF6F81B2E9
:10B73000EAEF5BF0A0B1B9EF5BF0AF67F8D7200E8E
:10B74000F46FF56F13EC66F0640EB06F020EAF6F1E
:10B7500081B2EAEF5BF0A0B1B9EF5BF0AF67F8D769
:10B76000300E806380C0F4F081C0F5F013EC66F019
:10B77000DAD7FCEC61F0230E9D6315D0300E805FAC
:10B78000815F0A0E8003F3CF19F081511926000E54
:10B79000196403D0320E196419D7300E806F310E40
:10B7A000816F9E6BB6D72A0E9D6306D0300E806FD8
:10B7B000310E816F9E6BADD7000E9E6302D0300EAE
:10B7C000816F81C080F09DC081F09E2B030E9E632F
:10B7D000A0D7E3D763EF57F0640EAE6F0F0EAD6FD7
:10B7E000F60EF76E2E0EF66E20EED6F0F5EC65F046
:10B7F000F60EF76E3E0EF66E20EEE6F0F5EC65F016
:10B8000013EC66F0E2EC64F0AD67FED7716B81A2D9
:10B810007EEF35F065EF0FF0A06B916B926B936B41
:10B82000956B946B966B906BA083A095A09B120078
:10B8300021EC62F0A0A312000D5009E0A0A706D0F1
:10B84000A08B640EB06F0DC0AFF001D0A09B32A0F2
:10B8500016D0130E926513D0380E926110D092C09C
:10B8600084F059EC61F07F51C4EC5CF08051C4EC81
:10B870005CF08151C4EC5CF00D0EC4EC5CF08E51B8
:10B88000060F926105D08E51FA0F926501D008D053
:10B890008F51060F926112008F51FA0F92651200BC
:10B8A000A0B90BD0A0B705D092C095F0926BA0794B
:10B8B000120092C093F0926B1200A0A704D092C025
:10B8C00094F0926B120092C096F0926B9351945F39
:10B8D000D8A0946D9551965FD8A0966D0A0E94618C
:10B8E0000ED096610CD032B083EC5CF0902B050E3C
:10B8F00090651200A093A099A085906B1200A0996A
:10B90000A095906B120093C084F059EC61F07F51C8
:10B91000C4EC5CF08051C4EC5CF08151C4EC5CF090
:10B92000200EC4EC5CF095C084F059EC61F07F51BE
:10B93000C4EC5CF08051C4EC5CF08151C4EC5CF070
:10B94000200EC4EC5CF094C084F059EC61F07F519F
:10B95000C4EC5CF08051C4EC5CF08151C4EC5CF050
:10B96000200EC4EC5CF096C084F059EC61F07F517D
:10B97000C4EC5CF08051C4EC5CF08151C4EC5CF030
:10B980000D0EC4EC5CF0120000000000A4A8FDD76E
:10B990006D6E1200349034A2120038A007D04150CE
:10B9A000E842E842070B9A6F9AC0E6F0A12B030E1B
:10B9B000A117000EA16302D03D0E0BD0010EA163B2
:10B9C00002D07E0E06D0020EA16302D07C0E01D002
:10B9D0007F0E10EEECF0E76E13EC66F012009F693C
:10B9E0002A0E9D6301D01200230E9D6301D0120028
:10B9F000300E9D6303D00A0E9F6F12003A0E9D61B8
:10BA000012009D510F0B9F6F12009DC09BF0300ED6
:10BA10009D6302D00A0E1DD02A0E9D6302D00B0E2C
:10BA200018D0230E9D6302D00C0E13D0410E9D63DF
:10BA300002D00D0E0ED0420E9D6302D00E0E09D024
:10BA4000430E9D6302D00F0E04D0440E9D6302D0BE
:10BA5000000E9B6F9B510F0B1009120001EED2F0EC
:10BA6000200E976F200EEE6E972F32EF5DF01200D2
:10BA7000976F200EE66E972FFCD7120009EE00F0AC
:10BA80009A0E976F200EEE6E972FFCD71200F4C11E
:10BA90009AF0000E9A6309D0F30EF76E0E0EF66E52
:10BAA00020EEE6F0F5EC65F01200010E9A6309D085
:10BAB000F30EF76E1E0EF66E20EEE6F0F5EC65F076
:10BAC0001200020E9A6309D0F30EF76E2E0EF66E78
:10BAD00020EEE6F0F5EC65F01200030E9A6309D053
:10BAE000F30EF76E3E0EF66E20EEE6F0F5EC65F026
:10BAF0001200040E9A6309D0F30EF76E4E0EF66E26
:10BB000020EEE6F0F5EC65F01200050E9A6309D020
:10BB1000F30EF76E5E0EF66E20EEE6F0F5EC65F0D5
:10BB20001200060E9A6309D0F30EF76E6E0EF66ED3
:10BB300020EEE6F0F5EC65F01200E60EF76E0E0E64
:10BB4000F66E20EEE6F0F5EC65F0120022EE00F065
:10BB50000D0EDF5CD8B41200410EDE6204D0540E2C
:10BB6000DE6201D0120038BCE6D20000F86ADE0EB8
:10BB7000686FE40E696F68C0F7FF69C0F6FF22EED8
:10BB800000F0060E6E6F0900F55006E0F550DE5C21
:10BB900012E16E2FC3EF5DF068C0F7FF69C0F6FFDA
:10BBA000060EF626E86AF7220900F5CF6AF0000EC5
:10BBB0006A630DD01200080E6927E86A6823DF0E59
:10BBC000685DD9E1AC0E695DD6E16A6B1200010EC9
:10BBD0006A6302D03D801200FF0E6A6302D03D828C
:10BBE00012000E0E6A6302D03E8012000F0E6A63CE
:10BBF00002D03E82120022EE00F02B0EDF62120015
:10BC0000060E6A5DD8A407EF5EF038841200110EAC
:10BC10006A5DD8A414EF5EF0ABEC60F0BFEC60F0AE
:10BC20006FC040F03D821200030E6A5DD8A43DEF64
:10BC30005EF0ABEC60F0BFEC60F03DB81200000EBF
:10BC40006F6302D059801200010E6F6302D05982D7
:10BC50001200020E6F6302D059841200030E6F634C
:10BC600002D059861200040E6F6302D05988120068
:10BC7000050E6F631200598A1200020E6A5DD8A485
:10BC800091EF5EF0ABEC60F0BFEC60F03DB81200FD
:10BC9000000E6F6302D057801200010E6F6302D056
:10BCA00057821200020E6F6302D057841200030EF7
:10BCB0006F6302D057861200040E6F6302D057885C
:10BCC0001200050E6F6306D0578ABFEC60F06FC09C
:10BCD00070F01200060E6F6306D0578CBFEC60F058
:10BCE0006FC070F01200070E6F6302D0578E120003
:10BCF000080E6F6302D058801200090E6F6302D0E5
:10BD000058821200000E6F6302D0588412000B0E8E
:10BD10006F6302D0588612000C0E6F6312005888B1
:10BD20001200160E6A5DD8A4BCEF5EF0ABEC60F0BA
:10BD3000B6EC60F0BFEC60F03DB81200000E6F632F
:10BD400002D05A801200010E6F6302D05A82120094
:10BD5000020E6F6302D05A841200030E6F6302D08A
:10BD60005A861200040E6F6302D05A881200050E24
:10BD70006F6312005A8A1200070E6A5DD8A4DAEFC8
:10BD80005EF001EE8CF0120EA86F200EEE6EA82F62
:10BD9000C5EF5EF002EE08F011EE8CF0100EA86F09
:10BDA000220EEF5C05E0EECFE6FFA82FD0EF5EF0AD
:10BDB0003D861200100E6A5DD8A4F8EF5EF001EE29
:10BDC0009EF0120EA86F200EEE6EA82FE3EF5EF02D
:10BDD00002EE08F011EE9EF0100EA86F220EEF5C3E
:10BDE00005E0EECFE6FFA82FEEEF5EF03D841200F7
:10BDF000040E6A5DD8A404EF5FF0ABEC60F0BFEC1A
:10BE000060F06F51416E1200120E6A5DD8A42EEFE1
:10BE10005FF03D8C02EE07F0520EEF6202D06F6BC6
:10BE20001200530EEF6218D002EE0CF0490EEF62D2
:10BE300008D002EE0EF00D0EEF620ED0010E6F6F05
:10BE40001200550EEF6208D002EE0EF00D0EEF62FA
:10BE500003D0020E6F6F12006F691200050E6A5D4B
:10BE6000D8A472EF5FF0ABEC60F0BFEC60F0080EAE
:10BE7000A86F11EE7CF0200EE66EA82FFCD7020E04
:10BE80006F6314D001EE7CF0550EEE6E6E0EEE6E0A
:10BE9000520EEE6E650EEE6E670EEE6E690EEE6E73
:10BEA000730EEE6E2E0EEE6E3D8A120002EE0BF059
:10BEB000220EEF5C09E0050EA86F11EE7CF0EECFCC
:10BEC000E6FFA82FFCD70CD0EE5011EE7CF0080E48
:10BED000A86F220EEF5C04E0EECFE6FFA82FF9D7A3
:10BEE0003D8A1200080E6A5DD8A486EF5FF0ABECC5
:10BEF00060F0B6EC60F0C0EC60F000EE43F06FC0B4
:10BF000042F06F516FC0EBFF388A12000B0E6A5D72
:10BF1000D8A49DEF5FF0ABEC60F0B6EC60F0DE50C3
:10BF2000200EA86F08EE32F0220EDF5C04E0DECFB8
:10BF3000EEFFA82FF9D7388C12000C0E6A5DD8A43A
:10BF4000A4EF5FF03F841200130E6A5DD8A4C1EF26
:10BF50005FF0ABEC60F0DE50100EA86F08EE12F050
:10BF6000200EEE6EA82FFCD708EE12F0100EA86F70
:10BF7000DF500D0804E0DECFEEFFA82FF9D73F8693
:10BF80001200140E6A5DD8A4D0EF5FF0ABEC60F045
:10BF9000BFEC60F03F98000E6F6312003F88120004
:10BFA000150E6A5DD8A47CEF60F0ABEC60F009EE92
:10BFB00000F019EC60F0DE50B6EC60F0B6EC60F02A
:10BFC000B6EC60F0B6EC60F0B6EC60F0F5EC60F06A
:10BFD0002C0EDF621200DE5009EE16F019EC60F054
:10BFE0000D0EDE5CD8B4120009EE2CF019EC60F0F6
:10BFF0000D0EDE5CD8B4120009EE42F019EC60F0D0
:10C000000D0EDE5CD8B4120009EE58F019EC60F0A9
:10C010000D0EDE5CD8B4120009EE6EF019EC60F083
:10C020000D0EDE5CD8B4120009EE84F019EC60F05D
:10C030001200F5EC60F0200E7C6F7D6F7E6F7F6FDD
:10C04000806F816F10EE7CF0200E866386C0E6FF65
:10C05000876387C0E6FF886388C0E6FF896389C07D
:10C06000E6FFDE50F5EC60F0200E866386C0E6FF4A
:10C07000876387C0E6FF886388C0E6FF896389C05D
:10C08000E6FF7CC0EEFF7DC0EEFF7EC0EEFF7FC00E
:10C09000EEFF80C0EEFF81C0EEFFDE50B6EC60F038
:10C0A000F5EC60F086C0EEFF87C0EEFF88C0EEFFC3
:10C0B00089C0EEFFDE50F5EC60F086C0EEFF87C071
:10C0C000EEFF88C0EEFF89C0EEFFDE50F5EC60F0B9
:10C0D00086C0EEFF87C0EEFF88C0EEFF89C0EEFF8E
:10C0E000DE50F5EC60F086C0EEFF87C0EEFF88C042
:10C0F000EEFF89C0EEFF1200170E6A5DD8A48EEF26
:10C1000060F0ABEC60F0BFEC60F06FC0F2F1B6EC49
:10C1100060F0C0EC60F06FC0F3F11200180E6A5DC1
:10C12000D8A49AEF60F0ABEC60F0BFEC60F06FC0A9
:10C13000F4F112001200389C780EA86F08EE52F04D
:10C1400012EE00F00D0EE75C04E0E6CFEEFFA82F44
:10C15000F9D7EF6A120022EE00F0800E6E6F3A0EF1
:10C16000DE5C03E06E2FAFEF60F01200FF0E6E6F2B
:10C170002C0EDE5C03E06E2FB8EF60F01200DE5094
:10C180003D98300E876F886F896FDECF89F00D0E76
:10C19000DF5C13E02C0EDF5C10E089C088F0DECF9E
:10C1A00089F00D0EDF5C09E02C0EDF5C06E088C034
:10C1B00087F089C088F0DECF89F0320E876503D022
:10C1C0003D88300E876F6F6B300E875F885F895FA9
:10C1D0000A0E8703F3500A0DF3CF6FF00A0E88039F
:10C1E000F3506F2789516F271200200E866F876FDB
:10C1F000886F896F040EA86F2C0EDF5CD8B4120014
:10C200000D0EDF5CD8B4120087C086F088C087F0BE
:10C2100089C088F0DECF89F0A82FEED71200846B9A
:10C22000300E7F5D640DF3CF84F0300E805D0A0D1B
:10C23000F3508427300E815D84271200836B826B5C
:10C24000300E755F765F775F785F795F060E756198
:10C250002DD0000E756507D0100E8327270E822380
:10C26000752F2CEF61F0000E766507D0E80E83275E
:10C27000030E8223762F36EF61F0000E776507D02C
:10C28000640E8327000E8223772F40EF61F0000EAB
:10C29000786507D00A0E8327000E8223782F4AEF95
:10C2A00061F079518327E86A8223120082698369E9
:10C2B00012007F6B806B816B630E846506D0640E09
:10C2C000845F02E37F2BFBD78427090E846506D0A9
:10C2D0000A0E845F02E3802BFBD7842784C081F0A1
:10C2E000300E7F278027812712007D6B7E6B7F6B4E
:10C2F000806B816B100E835F270E825B02E37D2BC8
:10C30000F9D7100E8327270E8223E80E835F030ED2
:10C31000825B02E37E2BF9D7E80E8327030E82238C
:10C32000640E835F000E825B02E37F2BF9D7640EFD
:10C330008327000E82230A0E835F000E825B02E3D6
:10C34000802BF9D70A0E8327000E822383C081F049
:10C35000300E7D277E277F27802781271200F5EC6E
:10C3600061F0C06BC16BBF9F1200D9C9E8FF070B1A
:10C37000E8461009CE6F0C0ECF6FD5EC62F01200BC
:10C38000DBC9E8FF070BE8461009CE6F0D0ECF6F33
:10C39000D5EC62F01200DDC9E8FF070BE846100992
:10C3A000CE6F0D0ECF6FD5EC62F01200DFC9E8FF43
:10C3B000070BE8461009CE6F0E0ECF6FD5EC62F07A
:10C3C0001200120ECE6F0C0ECF6FD5EC62F0120081
:10C3D000120ECE6F0F0ECF6FD5EC62F01200CF6F42
:10C3E000160ECE6FD5EC62F01200000ECE6F000E6E
:10C3F000CF6FD5EC62F01200E9EC62F0CF510F0B79
:10C400009D6F9D6703D00F0E9D6F17D0090E9D6520
:10C4100014D00A0E9D6303D0000E9D6F0ED00B0E3C
:10C420009D6303D0FA0E9D6F08D00C0E9D6303D060
:10C43000F30E9D6F02D00F0E9D6F300E9D27A091C1
:10C440001200E9EC62F0CEB5A087CEA5A097A0912E
:10C450001200110ECE6F800ECF6FD0EC62F01E0E68
:10C46000AB6FAB6731EF62F0110ECE6F000ECF6F86
:10C47000D0EC62F0800ED16F000ED26FBFEC62F094
:10C48000CAC9D1F0CBC9D2F0BFEC62F0D6C9D1F0A5
:10C49000D7C9D2F0BFEC62F0CCC9D1F0CDC9D2F08F
:10C4A000BFEC62F0D6C9D1F0D7C9D2F0BFEC62F0D0
:10C4B000CEC9D1F0CFC9D2F0BFEC62F0D6C9D1F06D
:10C4C000D7C9D2F0BFEC62F0D0C9D1F0D1C9D2F057
:10C4D000BFEC62F0D6C9D1F0D7C9D2F0BFEC62F0A0
:10C4E000D2C9D1F0D3C9D2F0BFEC62F0D6C9D1F035
:10C4F000D7C9D2F0BFEC62F0D4C9D1F0D5C9D2F01F
:10C50000BFEC62F0D6C9D1F0D7C9D2F0BFEC62F06F
:10C510001C0ED16F680ED26FBFEC62F0240ED16F8B
:10C52000A20ED26FBFEC62F0240ED16FAD0ED26FAF
:10C53000BFEC62F0240ED16FA20ED26FBFEC62F09E
:10C54000110ECE6FF3EC62F012001E0ECE6F010ED4
:10C55000CF6FDAEC62F0110ECE6F410ECF6FD0ECE0
:10C5600062F012001E0ECE6F030ECF6FDAEC62F097
:10C57000110ECE6F440ECF6FD0EC62F01200D1C01E
:10C58000CEF0D2C0CFF0EEEC62F0020EAB6FAB6734
:10C59000C7EF62F01200010ECD6F32EC63F01200B3
:10C5A000E00ECD6F10EC63F01200E10ECD6F10ECD9
:10C5B00063F01200E20ECD6F10EC63F01200E30E98
:10C5C000CD6FF8EC62F01200E50ECD6F03EC63F076
:10C5D0001200E60ECD6F1FEC63F01200E80ECD6F77
:10C5E00010EC63F01200EC0ECD6FF8EC62F012006C
:10C5F0008498CDC0CCF032EC63F0CEC0CCF032ECFD
:10C6000063F0848812008498CDC0CCF032EC63F0E3
:10C61000000ECC6F32EC63F0CCC0CEF084881200F8
:10C620008498CDC0CCF032EC63F0CEC0CCF032ECCC
:10C6300063F0CFC0CCF032EC63F0848812008498B1
:10C64000CDC0CCF032EC63F0000ECC6F32EC63F076
:10C65000CCC0CEF0000ECC6F32EC63F0CCC0CFF08B
:10C66000848812000000000000000000080ED06F57
:10C67000D890CC37D8A08394D8B08384839200001C
:10C6800000000000000000000000000000000000AA
:10C69000838200008350010BCC1300000000D02FD8
:10C6A00038EF63F01200849C849A100EA36FA6C02A
:10C6B000A4F0A7C0A5F0D890A533A433D8A0849E39
:10C6C000D8B0848E0000000000000000848C0000C0
:10C6D0000000000000000000000000000000849C3A
:10C6E000A32F5BEF63F000000000000000000000DB
:10C6F000000000000000848A00000000000000002C
:10C700000000000000000000000000000000000029
:10C710000000000000000000849A1200000E146463
:10C72000190C010E1464250C020E1464280C030E5F
:10C730001464320C030E146E320C000E1564190CC6
:10C74000010E1564250C020E1564280C030E1564E9
:10C75000320C156A190C240EE8CFD6F9A20EE8CFD8
:10C76000D7F9D8C9FDF00F0EFD17000EFD630DD0EF
:10C77000040EE8CFCAF9AB0EE8CFCBF9050EE8CF2F
:10C78000CCF9DE0EE8CFCDF92FD0010EFD630DD030
:10C79000040EE8CFCAF9AB0EE8CFCBF9060EE8CF0E
:10C7A000CCF9000EE8CFCDF91FD0020EFD630DD0FD
:10C7B000050EE8CFCAF9550EE8CFCBF9050EE8CF44
:10C7C000CCF9DE0EE8CFCDF90FD0030EFD63D0D744
:10C7D000050EE8CFCAF9550EE8CFCBF9000EE8CF29
:10C7E000CCF9000EE8CFCDF9DAC9FDF00F0EFD1738
:10C7F000000EFD630DD0060EE8CFCEF9670EE8CF30
:10C80000CFF9080EE8CFD0F9450EE8CFD1F92FD0F7
:10C81000010EFD630DD0050EE8CFCEF9550EE8CF21
:10C82000CFF9000EE8CFD0F9000EE8CFD1F91FD034
:10C83000020EFD630DD0050EE8CFCEF9AA0EE8CFAB
:10C84000CFF9000EE8CFD0F9000EE8CFD1F90FD024
:10C85000030EFD63D0D7050EE8CFCEF9550EE8CF15
:10C86000CFF9000EE8CFD0F9000EE8CFD1F9DEC93C
:10C87000FDF00F0EFD17000EFD630DD0050EE8CF85
:10C88000D2F9DE0EE8CFD3F9060EE8CFD4F9670E61
:10C89000E8CFD5F91200010EFD630DD0050EE8CFEB
:10C8A000D2F9550EE8CFD3F9060EE8CFD4F9000E31
:10C8B000E8CFD5F91200020EFD630DD0050EE8CFCA
:10C8C000D2F9AA0EE8CFD3F9000EE8CFD4F9000EC2
:10C8D000E8CFD5F91200030EFD63D0D7050EE8CFDF
:10C8E000D2F9550EE8CFD3F9000EE8CFD4F9000EF7
:10C8F000E8CFD5F9120000EE0CF0260ECB6F030E38
:10C90000AA6E000EA96ED6EC64F009EED8F0140EF3
:10C91000CB6F030EAA6ECA0EA96ED6EC64F009EEB8
:10C920009AF0280ECB6F030EAA6E260EA96ED6ECD7
:10C9300064F001EE00F07C0ECB6F030EAA6E4E0E7B
:10C94000A96ED6EC64F004EE40F0800ECB6F000EC2
:10C95000AA6E000EA96ED6EC64F005EE00F0A00EF3
:10C96000CB6F000EAA6E800EA96ED6EC64F005EEB9
:10C97000A0F0A00ECB6F010EAA6E200EA96ED6EC11
:10C9800064F006EE40F0A00ECB6F010EAA6EC00E52
:10C99000A96ED6EC64F006EEE0F0A00ECB6F020EAE
:10C9A000AA6E600EA96ED6EC64F01200A69EA69C3C
:10C9B000A6800000A8CFEEFFA92AE86AAA22CB2F02
:10C9C000F7D7120001EE04F0180ECB6F030EAA6E1B
:10C9D000520EA96EC6EC65F0FFEC64F00AEC65F04F
:10C9E00029EC65F034EC65F053EC65F068EC65F02B
:10C9F0007DEC65F092EC65F09DEC65F0120001EEC7
:10CA000000F0040ECB6F030EAA6E4E0EA96EC6EC9C
:10CA100065F0120000EE0CF00A0ECB6F030EAA6E4A
:10CA2000000EA96EC6EC65F001EE70F00C0ECB6F37
:10CA3000030EAA6EBE0EA96EC6EC65F001EE50F0B4
:10CA4000100ECB6F030EAA6E9E0EA96EC6EC65F09B
:10CA5000120000EE16F0080ECB6F030EAA6E0A0E3F
:10CA6000A96EC6EC65F0120000EE1EF0060ECB6F4C
:10CA7000030EAA6E120EA96EC6EC65F001EE60F010
:10CA8000100ECB6F030EAA6EAE0EA96EC6EC65F04B
:10CA900001EE40F0100ECB6F030EAA6E8E0EA96E43
:10CAA000C6EC65F0120000EE24F00A0ECB6F030E08
:10CAB000AA6E180EA96EC6EC65F009EE9AF0280E63
:10CAC000CB6F030EAA6E260EA96EC6EC65F012009F
:10CAD00000EE2EF0010ECB6F030EAA6E220EA96E91
:10CAE000C6EC65F001EE1CF0240ECB6F030EAA6EAF
:10CAF0006A0EA96EC6EC65F0120000EE30F0010E71
:10CB0000CB6F030EAA6E240EA96EC6EC65F009EE7B
:10CB1000D8F0140ECB6F030EAA6ECA0EA96EC6EC27
:10CB200065F0120004EE40F0800ECB6F000EAA6E8E
:10CB3000000EA96EC6EC65F0120005EE00F0A00E26
:10CB4000CB6F000EAA6E800EA96EC6EC65F005EEE6
:10CB5000A0F0A00ECB6F010EAA6E200EA96EC6EC3F
:10CB600065F006EE40F0A00ECB6F010EAA6EC00E6F
:10CB7000A96EC6EC65F006EEE0F0A00ECB6F020EDB
:10CB8000AA6E600EA96EC6EC65F01200A69EA69C69
:10CB9000A684F29EF29CEECFA8FF550EA76EAA0EB9
:10CBA000A76EA682F28CF28EA6B2D4EF65F0A92A07
:10CBB000E86AAA22CB2FC9EF65F0A694120003EE13
:10CBC00000F0EE5005E0AD6E00009EA8FED7F9D74C
:10CBD0000D0EAD6E00009EA8FED71200F86A090087
:10CBE000F5500CE0DE6E04D01200F86A100E986F5B
:10CBF0000900F55003E0DE6E982FFAD71200100EF0
:10CC0000C76F20EED6F0200EDE6EC72F03EF66F062
:10CC10001200100EC76F20EEE6F0200EDE6EC72F5A
:10CC20000DEF66F01200080E6EEC66F0000E6EEC72
:10CC300066F0100EC76F20EED6F0DE507DEC66F089
:10CC4000C72F1DEF66F00C0E6EEC66F0000E6EEC5A
:10CC500066F0100EC76F20EEE6F0DE507DEC66F059
:10CC6000C72F2DEF66F01200030E6EEC66F0280E53
:10CC7000AB6FAB6739EF66F0030E6EEC66F00A0E31
:10CC8000AB6FAB6741EF66F0030E6EEC66F0020E21
:10CC90006EEC66F0020E6EEC66F0080E6EEC66F05E
:10CCA000000E6EEC66F0080E6EEC66F0000E6EEC98
:10CCB00066F0010E6EEC66F00A0EAB6FAB675EEFCE
:10CCC00066F0000E6EEC66F0060E6EEC66F0000E7E
:10CCD0006EEC66F00C0E6EEC66F01200E83AF00BAB
:10CCE000856E8596859485820000000085923C0EB5
:10CCF0009C6F9C2F79EF66F01200C66FF00B856E6B
:10CD0000858685948582000000008592C639F00BE7
:10CD1000856E8586859485820000000085923C0E94
:10CD20009C6F9C2F91EF66F01200F29E040E6EEC49
:10CD300066F0000E6EEC66F0000E7DEC66F0000E04
:10CD40007DEC66F0000E7DEC66F0000E7DEC66F08A
:10CD5000000E7DEC66F0000E7DEC66F0000E7DECC2
:10CD600066F0180E7DEC66F0000E7DEC66F0000EAD
:10CD70007DEC66F0000E7DEC66F0000E7DEC66F05A
:10CD8000000E7DEC66F0000E7DEC66F0180E7DEC7A
:10CD900066F0180E7DEC66F0000E7DEC66F0000E7D
:10CDA0007DEC66F0000E7DEC66F0000E7DEC66F02A
:10CDB000000E7DEC66F01C0E7DEC66F0180E7DEC2E
:10CDC00066F0180E7DEC66F0000E7DEC66F0000E4D
:10CDD0007DEC66F0000E7DEC66F0000E7DEC66F0FA
:10CDE0001C0E7DEC66F01C0E7DEC66F0180E7DECE2
:10CDF00066F0180E7DEC66F0000E7DEC66F0000E1D
:10CE00007DEC66F0000E7DEC66F01E0E7DEC66F0AB
:10CE10001C0E7DEC66F01C0E7DEC66F0180E7DECB1
:10CE200066F0180E7DEC66F0000E7DEC66F0000EEC
:10CE30007DEC66F01E0E7DEC66F01E0E7DEC66F05D
:10CE40001C0E7DEC66F01C0E7DEC66F0180E7DEC81
:10CE500066F0180E7DEC66F0000E7DEC66F01F0E9D
:10CE60007DEC66F01E0E7DEC66F01E0E7DEC66F02D
:10CE70001C0E7DEC66F01C0E7DEC66F0180E7DEC51
:10CE800066F0180E7DEC66F01F0E7DEC66F01F0E4E
:10CE90007DEC66F01E0E7DEC66F01E0E7DEC66F0FD
:10CEA0001C0E7DEC66F01C0E7DEC66F0180E7DEC21
:10CEB00066F0180E7DEC66F0F28E12000AEE00F0BD
:10CEC0000D0EEF6209D00BEE00F03F0EEE6E0D0E70
:10CED000EE6E64EC6FF01200440EEE6226D04C0E43
:10CEE000EE6223D0440EEE6220D0FF0ED16FD26FDF
:10CEF00000EED1F0020ECB6F030EAA6EFE0EA96EED
:10CF0000C6EC65F0E30EF76E7E0EF66E20EED6F000
:10CF1000F5EC65F0E30EF76E8E0EF66E20EEE6F0A1
:10CF2000F5EC65F013EC66F0FF000AEE00F0440E3D
:10CF3000EE622BD0420EEE6228D0470EEE6225D074
:10CF4000A0EC6CF0080E846180EF6CF084C0FBF004
:10CF50002C0EEE6280EF6CF0A0EC6CF0020E84619F
:10CF600080EF6CF00D0EEE6280EF6CF0FB2BD89032
:10CF700081698137FB2FFDD7815184A13216E81ECC
:10CF800084B1321248EC6FF012000AEE00F0430E4A
:10CF9000EE625AD0500EEE6257D0570EEE6254D069
:10CFA000339E00C1E8FFEE6225D001C1E8FFEE62CA
:10CFB00021D002C1E8FFEE621DD003C1E8FFEE629E
:10CFC00019D00D0EEE6216D0338E48EC6FF0B7EC30
:10CFD0006CF0CFEC6CF013EC6DF040EC6DF074EC99
:10CFE0006DF0C5EC6DF0E0EC6DF041EC6EF0ADEC89
:10CFF0006EF012000AEE03F0450EEE6280EF6CF068
:10D00000750EEE6280EF6CF0720EEE6280EF6CF0E7
:10D010006F0EEE6280EF6CF0740EEE6280EF6CF0DB
:10D02000650EEE6280EF6CF0630EEE6280EF6CF0E6
:10D03000680EEE6280EF6CF00D0EEE6280EF6CF029
:10D04000338E48EC6FF012000AEE00F0520EEE62E2
:10D050001ED0420EEE621BD0540EEE6218D0E30ECC
:10D06000F76E9E0EF66E20EED6F0F5EC65F0E30E50
:10D07000F76EAE0EF66E20EEE6F0F5EC65F013EC12
:10D0800066F0E2EC64F000000000AAEF07F00AEEA0
:10D0900000F0500EEE6224D0530EEE6221D0570EF7
:10D0A000EE621ED033AE80EF6CF0EECF7EF0EECFAE
:10D0B0007FF0EECF80F0EECF81F00D0EEE6280EFCC
:10D0C0006CF001EE00F07EC0EEFF7FC0EEFF80C08E
:10D0D000EEFF81C0EEFFFFEC64F048EC6FF0120051
:10D0E00033AE80EF6CF00AEE00F0460EEE62BBD07D
:10D0F000580EEE62B8D04F0EEE62B5D0A0EC6CF0D8
:10D1000084C000FC2C0EEE6280EF6CF0100E1CEE62
:10D1100001F038EC5DF0100EFB6F1CEE01F02C0EF0
:10D12000EF5C04E0EECFE6FFFB2FF9D72C0EEE62AA
:10D1300080EF6CF0A0EC6CF084C011FC2C0EEE6261
:10D1400080EF6CF0A0EC6CF084C012FC2C0EEE6250
:10D1500080EF6CF0A0EC6CF084C013FC2C0EEE623F
:10D1600080EF6CF0A0EC6CF084C014FC2C0EEE622E
:10D1700080EF6CF0A0EC6CF084C015FC2C0EEE621D
:10D1800080EF6CF0A0EC6CF084C016FC2C0EEE620C
:10D1900080EF6CF0A0EC6CF084C017FC2C0EEE62FB
:10D1A000AFD30C0E1CEE18F038EC5DF0080EFB6FE0
:10D1B0001CEE18F02C0EEF5C04E0EECFE6FFFB2F28
:10D1C000F9D72C0EEE629CD3040EFB6F1CEE20F000
:10D1D0002C0EEF5C04E0EECFE6FFFB2FF9D72C0E10
:10D1E000EE628ED3A0EC6CF084C024FC2C0EEE62B8
:10D1F00087D3A0EC6CF084C025FC0D0EEE6280D3CA
:10D2000000CC0CF025CC0DF011CC0EF024CC0FF09E
:10D2100012CC10F013CC11F014CC12F015CC13F08A
:10D2200016CC14F017CC15F00C0EFB6F1CEE18F09A
:10D2300001EE70F0E6CFEEFFFB2FFCD7100EFB6F78
:10D240001CEE01F001EE50F0E6CFEEFFFB2FFCD715
:10D250000AEC65F048EC6FF08EEC63F08E6F9DEC9D
:10D2600063F08F6F12000AEE00F0460EEE6253D0AC
:10D27000580EEE6250D0530EEE624DD0A0EC6CF022
:10D2800084C000FC2C0EEE623BD3A0EC6CF084C09A
:10D2900001FC2C0EEE6234D3A0EC6CF084C002FCD6
:10D2A0002C0EEE622DD3A0EC6CF084C003FC2C0E8F
:10D2B000EE6226D3A0EC6CF084C004FC2C0EEE626F
:10D2C0001FD3A0EC6CF084C005FC2C0EEE6218D3CA
:10D2D000A0EC6CF084C006FC2C0EEE6211D3A0EC26
:10D2E0006CF084C007FC0D0EEE620AD300CC16F081
:10D2F00006CC18F007CC19F001CC17F002CC1AF0CC
:10D3000003CC1BF004CC1CF005CC1DF029EC65F01F
:10D3100048EC6FF012000AEE00F0470EEE628AD081
:10D32000530EEE6287D04D0EEE6284D0A0EC6CF00E
:10D3300084C000FC2C0EEE62E3D2100E1CEE01F055
:10D3400038EC5DF0100EFB6F1CEE01F02C0EEF5C64
:10D3500004E0EECFE6FFFB2FF9D72C0EEE62D0D221
:10D36000A0EC6CF084C011FC2C0EEE62C9D2A0ECD3
:10D370006CF084C012FC2C0EEE62C2D2100E1CEEB9
:10D3800013F038EC5DF0080EFB6F1CEE13F02C0E62
:10D39000EF5C04E0EECFE6FFFB2FF9D72C0EEE6238
:10D3A000AFD2080EFB6F1CEE1BF02C0EEF5C04E0FE
:10D3B000EECFE6FFFB2FF9D72C0EEE62A1D2A0EC48
:10D3C0006CF084C023FC2C0EEE629AD2A0EC6CF0C0
:10D3D00084C024FC2C0EEE6293D2A0EC6CF084C0CE
:10D3E00025FC0D0EEE628CD200CC1EF011CC22F08A
:10D3F00012CC23F023CC20F024CC21F025CC1FF03C
:10D40000100EFB6F1CEE01F001EE60F0E6CFEEFFB8
:10D41000FB2FFCD7100EFB6F1CEE13F001EE40F05B
:10D42000E6CFEEFFFB2FFCD734EC65F0388648ECF6
:10D430006FF012000AEE00F04E0EEE62BCD0450E08
:10D44000EE62B9D0540EEE62B6D0A0EC6CF084C09F
:10D4500000FC2C0EEE6254D2A0EC6CF084C001FCF7
:10D460002C0EEE624DD283EC6CF083C002FC82C0C5
:10D4700003FC2C0EEE6244D22E0E1CEE04F038ECAF
:10D480005DF0060EFB6F1CEE04F02C0EEF5C04E06A
:10D49000EECFE6FFFB2FF9D72C0EEE62060EFB6FE8
:10D4A0001CEE0AF02C0EEF5C04E0EECFE6FFFB2F43
:10D4B000F9D72C0EEE6224D2060EFB6F1CEE12F092
:10D4C0002C0EEF5C04E0EECFE6FFFB2FF9D72C0E1D
:10D4D000EE6216D283EC6CF083C018FC82C019FC9B
:10D4E0002C0EEE620DD2060EFB6F1CEE1AF02C0E07
:10D4F000EF5C04E0EECFE6FFFB2FF9D72C0EEE62D7
:10D50000FFD183EC6CF083C020FC82C021FC2C0E88
:10D51000EE62F6D1060EFB6F1CEE22F02C0EEF5CD5
:10D5200004E0EECFE6FFFB2FF9D72C0EEE62E8D138
:10D5300083EC6CF083C028FC82C029FC2C0EEE62C8
:10D54000DFD1060EFB6F1CEE2AF02C0EEF5C04E020
:10D55000EECFE6FFFB2FF9D72C0EEE62D1D183EC94
:10D560006CF083C030FC82C031FC0D0EEE62C8D17D
:10D5700000CC24F001CC25F002CC26F003CC27F01F
:10D5800004CC28F005CC29F006CC2AF007CC2BF0EF
:10D5900008CC2CF009CC2DF0280EFB6F09EE9AF088
:10D5A0001CEE0AF0E6CFEEFFFB2FFCD753EC65F044
:10D5B00048EC6FF012000AEE00F0530EEE623FD01E
:10D5C0004D0EEE623CD0530EEE6239D0A0EC6CF002
:10D5D00084C000FC2C0EEE6293D1240E1CEE01F0F0
:10D5E00038EC5DF0100EFB6F1CEE01F02C0EEF5CC2
:10D5F00004E0EECFE6FFFB2FF9D72C0EEE6280D1D0
:10D60000100EFB6F1CEE13F00D0EEF5C04E0EECF7E
:10D61000E6FFFB2FF9D70D0EEE6272D100CC2EF093
:10D62000240EFB6F1CEE01F001EE1CF0E6CFEEFFC6
:10D63000FB2FFCD768EC65F048EC6FF012000AEEA7
:10D6400000F0500EEE6251D0520EEE624ED0460EF9
:10D65000EE624BD0A0EC6CF02C0EEE6251D1210E9C
:10D6600084614ED1000E84654BD1840784C000FCD8
:10D67000080EFB6F1CEE01F0E668FB2FFDD7070ECE
:10D68000FB6F1CEE01F02C0EEF5C05E0EE500F0B73
:10D69000E66EFB2FF8D72C0EEE6232D1A0EC6CF0C8
:10D6A00084C008FC0D0EEE622BD1040EFB6F1CEE45
:10D6B00001F004EE40F000CCE8FF040DF350E92641
:10D6C000F450EA22E638F00BEF6EE6500F0BEE1244
:10D6D000FB2FF8D71F0E006103D048EC6FF012004B
:10D6E00092EC65F048EC6FF012000AEE00F04C0E80
:10D6F000EE6253D0530EEE6250D0540EEE624DD017
:10D70000A0EC6CF02C0EEE62FBD0410E8461F8D0E0
:10D71000000E8465F5D0840784C000FC100EFB6FFA
:10D720001CEE01F0E668FB2FFDD7100EFB6F1CEE20
:10D7300001F02C0EEF5C05E0EE500F0BE66EFB2FB8
:10D74000F8D72C0EEE62DCD0A0EC6CF084C011FC9B
:10D750000D0EEE62D5D0080EFB6F1CEE01F005EE4B
:10D7600000F000CCE8FF0A0DF350E926F450EA225D
:10D77000E638F00BEF6EE6500F0BEE12FB2FF8D7EA
:10D7800011CCEFFF3F0E006103D048EC6FF01200A8
:10D790009DEC65F048EC6FF012000AEE00F0470EC9
:10D7A000EE62AED0570EEE62ABD0500EEE62A8D055
:10D7B000A0EC6CF084C000FC2C0EEE62A1D0A0ECBA
:10D7C0006CF084C001FC2C0EEE629AD0A0EC6CF0E0
:10D7D00084C002FC2C0EEE6293D0A0EC6CF084C0EE
:10D7E00003FC2C0EEE628CD0A0EC6CF084C004FC28
:10D7F0002C0EEE6285D0A0EC6CF084C005FC2C0EE3
:10D80000EE627ED0A0EC6CF084C006FC2C0EEE62C2
:10D8100077D0A0EC6CF084C007FC2C0EEE6270D0C8
:10D82000A0EC6CF084C008FC2C0EEE6269D0A0EC79
:10D830006CF084C009FC2C0EEE6262D0A0EC6CF09F
:10D8400084C00AFC2C0EEE625BD0A0EC6CF084C0AD
:10D850000BFC2C0EEE6254D0A0EC6CF084C00CFCDF
:10D860002C0EEE624DD0A0EC6CF084C00DFC2C0EA2
:10D87000EE6246D0A0EC6CF084C00EFC2C0EEE6282
:10D880003FD0A0EC6CF084C00FFC2C0EEE6238D0C0
:10D89000A0EC6CF084C010FC2C0EEE6231D0A0EC39
:10D8A0006CF084C011FC2C0EEE622AD0A0EC6CF05F
:10D8B00084C012FC2C0EEE6223D0A0EC6CF084C06D
:10D8C00013FC2C0EEE621CD0A0EC6CF084C014FC97
:10D8D0000D0EEE6215D000CC30F0140EFB6F1CEE76
:10D8E00001F009EED8F0E6CFEEFFFB2FFCD77DEC80
:10D8F00065F048EC6FF0ABEC63F029EC62F01200DD
:10D9000053EC6FF01200300E756F766F776F786F93
:10D91000796F050E976F2C0EEF5C0FE00D0EEF5C2C
:10D920000CE076C075F077C076F078C077F079C0FB
:10D9300078F0EECF79F0972FEED71EEC61F0120061
:10D94000300E7F6F806F816F030E976F2C0EEF5C30
:10D950000BE00D0EEF5C08E080C07FF081C080F02E
:10D96000EECF81F0972FF2D70FEC61F01200FF0E8F
:10D97000F76E4C0EF66E0BEE00F0560EEE6E450E88
:10D98000EE6E520EEE6E100EFA6F0900F5CFEEFF3E
:10D99000FA2FFBD70D0EEE6E64EC6FF012000BEE5B
:10D9A00000F0460EEE6E580EEE6E4F0EEE6E0CC090
:10D9B00084F013EC6FF011EE50F0100E3BEC6FF0B2
:10D9C0000EC084F011EC6FF010C084F011EC6FF019
:10D9D00011C084F011EC6FF012C084F011EC6FF004
:10D9E00013C084F011EC6FF014C084F011EC6FF0F0
:10D9F00015C084F011EC6FF011EE70F0080E3BECE6
:10DA00006FF011EE78F0040E3BEC6FF00FC084F075
:10DA100011EC6FF00DC084F011EC6FF00D0EEE6E96
:10DA200064EC6FF012000BEE00F0460EEE6E580E36
:10DA3000EE6E530EEE6E16C084F013EC6FF017C04E
:10DA400084F011EC6FF01AC084F011EC6FF01BC081
:10DA500084F011EC6FF01CC084F011EC6FF01DC06D
:10DA600084F011EC6FF018C084F011EC6FF019C065
:10DA700084F011EC6FF00D0EEE6E64EC6FF012009E
:10DA80000BEE00F0470EEE6E530EEE6E4D0EEE6E88
:10DA90001EC084F013EC6FF011EE60F0100E3BEC42
:10DAA0006FF022C084F011EC6FF023C084F011EC11
:10DAB0006FF011EE40F0080E3BEC6FF011EE48F005
:10DAC000080E3BEC6FF020C084F011EC6FF021C029
:10DAD00084F011EC6FF01FC084F011EC6FF00D0EAC
:10DAE000EE6E64EC6FF012000BEE00F04E0EEE6E78
:10DAF000450EEE6E540EEE6E24C084F013EC6FF003
:10DB000025C084F011EC6FF026C083F027C082F0AE
:10DB100022EC6FF0060E10EE28F03BEC6FF019EEE1
:10DB20009AF0060E3BEC6FF019EEA2F0060E3BECFD
:10DB30006FF0A8C983F0A9C982F022EC6FF019EE4A
:10DB4000AAF0060E3BEC6FF0B0C983F0B1C982F0C9
:10DB500022EC6FF019EEB2F0060E3BEC6FF0B8C994
:10DB600083F0B9C982F022EC6FF019EEBAF0060E1C
:10DB70003BEC6FF0C0C983F0C1C982F022EC6FF0BA
:10DB80000D0EEE6E64EC6FF012000BEE00F0530E13
:10DB9000EE6E4D0EEE6E530EEE6E2EC084F013EC54
:10DBA0006FF011EE1CF0100E3BEC6FF011EE2EF04A
:10DBB000100E3BEC6FF00D0EEE6E64EC6FF0120089
:10DBC0000BEE00F0470EEE6E570EEE6E500EEE6E40
:10DBD00030C084F013EC6FF0D8C984F011EC6FF012
:10DBE000D9C984F011EC6FF0DAC984F011EC6FF050
:10DBF000DBC984F011EC6FF0DCC984F011EC6FF03C
:10DC0000DDC984F011EC6FF0DEC984F011EC6FF027
:10DC1000DFC984F011EC6FF0E0C984F011EC6FF013
:10DC2000E1C984F011EC6FF0E2C984F011EC6FF0FF
:10DC3000E3C984F011EC6FF0E4C984F011EC6FF0EB
:10DC4000E5C984F011EC6FF0E6C984F011EC6FF0D7
:10DC5000E7C984F011EC6FF0E8C984F011EC6FF0C3
:10DC6000E9C984F011EC6FF0EAC984F011EC6FF0AF
:10DC7000EBC984F011EC6FF00D0EEE6E64EC6FF0FA
:10DC80001200200EFC6F14EE40F00BEE00F0500E70
:10DC9000EE6E520EEE6E460EEE6ED880210EFC55E4
:10DCA000846F59EC61F080C0EEFF81C0EEFF2C0E56
:10DCB000EE6EE7380F0B7A6F0A0E7A6302D02A0EE7
:10DCC00007D00B0E7A6302D02B0E02D0300E7A25CD
:10DCD0007A6FE6500F0B300F7B6FE7380F0B300F6A
:10DCE0007C6FE6500F0B300F7D6FE7380F0B300F56
:10DCF0007E6FE6500F0B300F7F6FE7380F0B300F42
:10DD0000806FE6500F0B300F816F3A0E7A611AD098
:10DD10007AC0EEFF7B6116D07BC0EEFF7C6112D033
:10DD20007CC0EEFF7D610ED07DC0EEFF7E610AD02B
:10DD30007EC0EEFF7F6106D07FC0EEFF806102D023
:10DD400080C0EEFF2C0EEE6E81C0EEFF0D0EEE6E6B
:10DD500064EC6FF0FC2F99D71200400EFC6F15EEAB
:10DD600000F00BEE00F04C0EEE6E530EEE6E540E05
:10DD7000EE6ED880410EFC55846F59EC61F080C086
:10DD8000EEFF81C0EEFF2C0EEE6EE6CF7AF0E6CF0E
:10DD90007BF0E6CF7CF0E6CF7DF0E6CF7EF0E6CFFD
:10DDA0007FF0E6CF80F0E6CF81F0E6CF79F0E65065
:10DDB0007A390F0B300FFD6F3C0EFD6127D03B0E03
:10DDC000FD5DD8B4FD99FDC0EEFF7A510F0B300F09
:10DDD0007A6F3A0E7A611AD07AC0EEFF070EFB6FA7
:10DDE00020EE7BF0DF380F0B300FFD6F3A0EFD6138
:10DDF0000DD0FDC0EEFFDE500F0B300FFD6F3A0E61
:10DE0000FD6104D0FDC0EEFFFB2FECD779C084F09C
:10DE100011EC6FF00D0EEE6E64EC6FF0FC2FA1D7DD
:10DE200012002C0EEE6E59EC61F0300E7F6303D0C1
:10DE3000806303D004D07FC0EEFF80C0EEFF81C0BE
:10DE4000EEFF12002C0EEE6E75EC61F0300E7D636D
:10DE500007D07E6307D07F6307D0806307D008D0E8
:10DE60007DC0EEFF7EC0EEFF7FC0EEFF80C0EEFF04
:10DE700081C0EEFF1200FA6F2C0EEE6E01D0FA6F29
:10DE8000200EE75C04E0E6CFEEFFFA2FF9D7120090
:10DE90000BEE00F04F0EEE6E4B0EEE6E0D0EEE6EB4
:10DEA00064EC6FF012000BEE00F0450EEE6E520EB9
:10DEB000EE6E520EEE6E4F0EEE6E520EEE6E0D0EBA
:10DEC000EE6E64EC6FF01200EF6AF96B0BEE00F08F
:10DED000A4A8FED7EE5003E06D6EF92FF9D7A4A8E1
:10DEE000FED7120041540000000000004F4B00001C
:10DEF000000001002B57494E443A02002B43524583
:10DF0000473A03002B4353513A2004002B434F5010
:10DF1000533A05002B4352494E4706002B434C49C8
:10DF2000503A07002B434D54493A08002B434D47C4
:10DF3000573A09002B434D53533A0A002B434D47A0
:10DF4000523A0B002B434D47533A0C004E4F2041A1
:10DF50004E530E004255535900000F002B434357B8
:10DF6000413A10002B434D45000011002B4350490E
:10DF70004E3A12004552524F5200FF002B57494D66
:10DF8000454913002B5744574C3A14002B43434543
:10DF9000443A15002B4343454C4C16002B57565220
:10DFA0003A2017002B574D42533A1800000000004A
:10DFB000000000004154000041544531000041542C
:10DFC0004800000041544100000041542B434D459E
:10DFD000453D3100000041542B434C49503D310038
:10DFE000000041542B434C49503D30000000415447
:10DFF0002B434C49523D3000000041542B434C49C7
:10E00000523D3100000041542B434C49523D3200F7
:10E01000000041542B4950523D3936303000000049
:10E0200041542B4950523D31393230300000415477
:10E030002B4946433D302C30000041542B5753565A
:10E04000473D3100000041542B57494E443D31308B
:10E050003233000041542B57494E443D3F000000ED
:10E0600041542B43474D5200000041542B57445715
:10E070004C00000041542B57494D45493F000000DA
:10E0800041542B434345443D302C33000000415460
:10E090002B4343454C4C3D30000041542B434655E7
:10E0A0004E3D3100000041542B574344503D310058
:10E0B000000041542B435245473D3000000041547D
:10E0C0002B435245473D3100000041542B435245FC
:10E0D000473D3200000041542B434345443D312C21
:10E0E0003800000041542B4352433D31000041545D
:10E0F0002B434943423D3200000041542657000063
:10E1000041542B434F50533D3000000041542B43AA
:10E110004F50533D3200000041542B434F50533D6C
:10E12000332C3000000041542B434F50533D332CCF
:10E130003100000041542B434F50533F00004154E5
:10E140002B4343494400000041542B43494D4900AF
:10E15000000041542B434E554D00000041542B43C9
:10E160004C49523D3000000041542B434C49523F32
:10E17000000041542B434357413D312C312C310099
:10E18000000041542B4350494E3F000041542B574F
:10E1900056523F00000041542B574D42533F000060
:10E1A00041542B434D45523D2C30000041542B45EA
:10E1B00043484F3D312C332C33302C383030302C09
:10E1C00032353000000041542B53494445543D3111
:10E1D0002C33000041542B535045414B45523D30A8
:10E1E000000041542B57464D3D312C333300000085
:10E1F00041542B5647543D30000041542B56475450
:10E200003D343000000041542B5647523D36340017
:10E21000000041542B4543484F3D312C362C3330C0
:10E220002C35302C36342C3230302C3535302C31E6
:10E23000352C33323736372C353030302C323734BA
:10E2400038342C33383639372C373331312C3400CD
:10E25000000041542B53494445543D300000415483
:10E260002B535045414B45523D30000041542B57F4
:10E27000464D3D312C333300000041542B4543487B
:10E280004F3D312C332C33302C383030302C32355C
:10E290003600000041542B53494445543D312C3342
:10E2A000000041542B535045414B45523D31000035
:10E2B00041542B57464D3D312C333300000041541F
:10E2C0002B43534D533D3000000041542B434D47E9
:10E2D000463D3100000041542B434E4D493D322C08
:10E2E000312C302C302C3000000041542B434D4752
:10E2F000443D000041542B434D47443D312C3400F4
:10E30000000041542B434D47523D000041542B43E4
:10E310004D53533D000041542B434D47573D0000A2
:10E3200041542B434D47533D000041542B43484C2F
:10E33000443D3200000041542B43484C443D3132AF
:10E34000000041542B43484C443D330000002A2038
:10E35000474154455741592047534D20202A4C6F7F
:10E36000616465722050617373776F726420436FCC
:10E3700064653A2020202020202020202020476192
:10E380007465776179206973207265616479746F4F
:10E3900020746865207570646174696E67215361CB
:10E3A00076696E6720506172616D65746572205286
:10E3B000657374617274696E6720475720204753F4
:10E3C0004D3A202D506F776572204F4E2D20202022
:10E3D000202D506F776572204F46462D20204E65C8
:10E3E00074776F726B3A2020202020202020534920
:10E3F0004D783A204175746F6D617469632053499B
:10E400004D783A20204D616E75616C202020455278
:10E41000524F523A20204D6F64756C6520202020A9
:10E42000206E6F7420616E737765722020204552D4
:10E43000524F523A202020202020202020204154DA
:10E4400020436F6D6D616E64206661696C2E2020C3
:10E450002053494D202063617264202020202069D0
:10E4600073206E6F742070726573656E7420202047
:10E470007761732072656D6F76656420202020209F
:10E4800077617320696E7365727465642020202043
:10E490002020496E73657274202020202020496E50
:10E4A000736572742053494D2020636172644E6518
:10E4B00074776F726B20776173206C6F737447533E
:10E4C0004D3A202020202D496E69742D2020204EA9
:10E4D0006574776F726B2064656E69656420204394
:10E4E00068616E6765207468652053494D2020532C
:10E4F000494D20756E6B6E6F776E202020204E6523
:10E5000074776F726B20697320666F756E6420205C
:10E51000204E6574776F726B20202020202020779A
:10E520006173206E6F7420666F756E642020526F69
:10E53000616D696E6720697320666F756E644E65E4
:10E5400074776F726B3A20756E6B6E6F776E4E6577
:10E5500074776F726B3A20202020202020205349AE
:10E560004D783A2053657474696E67202020204DE1
:10E57000616E75616C2053656C65637420204E6517
:10E5800074776F726B3A20202020202020204E6567
:10E5900074776F726B3A20202020202020202020CA
:10E5A00069732073656C6563746564202020202086
:10E5B0006E6F7420616C6C6F77656420202020433F
:10E5C0006F6465206F66204E6574776F726B2020D4
:10E5D000697320616473656E742E20202020204EA4
:10E5E0006574776F726B7320636F6465732020208E
:10E5F00061726520616273656E7420202020566F01
:10E6000069636520524154453A78782C7878202007
:10E610002047534D2042616E64203F20202020453A
:10E620006E7465722050617373776F726420496EE7
:10E6300076616C69642050617373776F7264537490
:10E64000657020323A20436F6D6D616E642020202A
:10E6500020697320696E76616C69642E202044699C
:10E66000616C3A2046585320506F727420205269D2
:10E670006E673A20202047534D2E53494D3144694F
:10E68000616C3A20202047534D2E53494D31436150
:10E690006C6C3A20202047534D2E53494D31576121
:10E6A00069743A20202047534D2E53494D3154610F
:10E6B0006C6B3A20202047534D2E53494D3120207A
:10E6C00047534D204469616C696E672020202044C7
:10E6D0006972656374204469616C696E672E204FAE
:10E6E0006E6C7920546F6E65204469616C2E202019
:10E6F0002020505249564154452020202020434993
:10E7000044206973206E6F7420666F756E6444696F
:10E71000616C3A2046584F20506F7274202054612B
:10E720006C6B3A2046584F20506F72742020446919
:10E73000616C3A20464F4C4C4F57204D4520546158
:10E740006C6B3A20464F4C4C4F57204D4520446946
:10E75000616C3A6E6F7420737570706F72742020E4
:10E760005245504C4143494E472053494D2053494F
:10E770004D313A206C6F6164696E672020205349E7
:10E780004D323A206C6F6164696E672020204572BB
:10E79000726F72206F66205265616464722E4D65DF
:10E7A0006E75202320312E30202020202020202094
:10E7B0002046585320504F525420202020204D6591
:10E7C0006E75202320322E30202020202020202073
:10E7D0002047534D204E4554574F524B20204D65F6
:10E7E0006E75202320332E30202020202020202052
:10E7F0002046584F20504F525420202020204D6555
:10E800006E75202320342E30202020202020202030
:10E8100020204741544557415920202020204D6554
:10E820006E75202320352E302020202020202053DC
:10E830004D5320504152414D4554455253204D6552
:10E840006E75202320312E31202020202020507270
:10E8500065666978657320666F722047534D4D6514
:10E860006E75202320312E322020202020202020D1
:10E87000204449414C2050415553452020204D65AE
:10E880006E75202320312E33202020202020204789
:10E89000656E65726174696F6E20434C49204765EF
:10E8A0006E65726174696F6E3A20204F4E20476525
:10E8B0006E65726174696F6E3A20204F4646434C14
:10E8C000493A202042656C6C636F72652020434C8E
:10E8D000493A204254204F6E2D686F6F6B20434C95
:10E8E000493A20562E323320202020202020434C2D
:10E8F000493A2020202020202020202020204D6563
:10E900006E75202320312E342020202020205245D7
:10E91000564552534520504F4C4152495459237843
:10E9200078782020666F722053494D3A2078205025
:10E930007265666978203A787878787878782044B3
:10E9400069616C6C696E6720506175736520202069
:10E95000782E78207365636F6E6473202020526573
:10E96000766572736520506F6C6172697479547941
:10E9700070653A2044697361626C65202020547987
:10E9800070653A4261742E5265766572736554798A
:10E9900070653A44626C2E5265762E506F6C5479D5
:10E9A00070653A427265616B204C696E652031304A
:10E9B000306D7320782054696D653A2020204D65B4
:10E9C0006E75202320322E3120202020202020553B
:10E9D0004E4C49535445442043414C4C2020205533
:10E9E0006E6C69737465642043616C6C20202041F7
:10E9F0006363657074202D20656E61626C652041D3
:10EA00006363657074202D64697361626C65204175
:10EA10006363657074202D202020202020204D6508
:10EA20006E75202320322E322020202020204753B4
:10EA30004D20414343455353204D4F44453A44698B
:10EA4000726563746C7920746F2046585320446952
:10EA5000726563746C7920746F2046584F20475359
:10EA60004D2F46584F2043616C6C4261636B2047C9
:10EA7000534D20436F6E666572656E63652020207E
:10EA80002020202020202020202020202020417510
:10EA9000746F6469616C206E756D626572204D657E
:10EAA0006E75202320322E3320202020202020208D
:10EAB0005245504541542043414C4C202020526542
:10EAC000706561742063616C6C2046584F206672DB
:10EAD0006F6D2047534D3A20656E61626C656672BA
:10EAE0006F6D2047534D3A64697361626C654D6583
:10EAF0006E75202320322E3420202020202020203C
:10EB00002043414C4C4241434B20202020202043B5
:10EB1000414C4C4241434B20534554555020436196
:10EB20006C6C6261636B3A656E61626C6520436117
:10EB30006C6C6261636B3A64697361626C654361BA
:10EB40006C6C6261636B3A202020202020204341BE
:10EB50004C4C4241434B2077696C6C20626576696E
:10EB6000613A20202047534D202020202020766924
:10EB7000613A20202046584F20202020202076690E
:10EB8000613A202020202020202020202020204109
:10EB9000646465642043414C4C4241434B20766998
:10EBA0006120534D53203A64697361626C657669E4
:10EBB0006120534D53203A20656E61626C65766921
:10EBC0006120534D53203A202020202020204D65E5
:10EBD0006E75202320322E35202020202020204139
:10EBE000434345535320766961204C495354204197
:10EBF000636365737320766961204C697374766909
:10EC000061204C4953543A2020202020202076694E
:10EC100061204C4953543A20656E61626C65766997
:10EC200061204C4953543A64697361626C654D6567
:10EC30006E75202320322E3620202020202047539E
:10EC40004D204E554D42455253204C495354475345
:10EC50004D204E756D62657273204C6973746B65DF
:10EC6000793A2A2D4164642C232D456469742378F4
:10EC7000783A53544154453D2030303030304D6166
:10EC8000782E20616D6F756E74206F662020746819
:10EC900065206E756D62657273203D2036344D655A
:10ECA0006E75202320322E37202020202020205255
:10ECB000494E474241434B20544F4E45202020525D
:10ECC000696E674261636B20546F6E6520206672C7
:10ECD0006F6D2047534D3A64697361626C6566726B
:10ECE0006F6D2047534D3A656E61626C65206672A8
:10ECF0006F6D2047534D3A202020202020204D6565
:10ED00006E75202320322E38202020202020434CD6
:10ED1000495220616E64205052495641544520208A
:10ED20004D79204E756D6265723A20202020207347
:10ED30006574206279204E6574776F726B20206451
:10ED4000697361626C6564206E756D626572202006
:10ED5000656E61626C6564206E756D62657250727D
:10ED600069766174652063616C6C20746F204C6FF0
:10ED700063616C204C6E3A656E61626C65204C6F0D
:10ED800063616C204C6E3A64697361626C654C6FB0
:10ED900063616C204C6E3A202020202020204D659D
:10EDA0006E75202320322E39202020202020204E56
:10EDB00045542F43454C4C2053454C454354204E1D
:10EDC0004554574F524B2053454C45435420202027
:10EDD000204175746F2053656C656374202020504A
:10EDE0006572696F6469632053656C65637478202C
:10EDF0004E6574776F726B3A20202020202050657A
:10EE000072696F642F7365633A2020202020204DA3
:10EE1000616E75616C2053656C6563742020204DB4
:10EE2000616E75616C2053656C65637420204E655E
:10EE300074776F726B3A2020202020202020202021
:10EE400043454C4C2053454C4543542020204365BA
:10EE50006C6C2053656C6563742066726F6D4E65D3
:10EE600074776F726B3A20202020202020202020F1
:10EE7000204175746F2053656C65637420202050A9
:10EE80006572696F6469632053656C656374507261
:10EE9000643D78787878782C52783D787878204D71
:10EEA000616E75616C2053656C65637420204552FA
:10EEB000524F523A202020202020202020202020A5
:10EEC00043656C6C2053656C65637420202078204A
:10EED000434C3A787878782C52783A7878784E3A69
:10EEE0007878787878782C43483A7878787820530E
:10EEF000656C65637465642043656C6C2020697380
:10EF0000206E6F7420617661696C61626C65576117
:10EF10006974696E673A202020202020202020205C
:10EF200043656C6C2053656C65637420202020530E
:10EF3000656C65637465642043656C6C20202020DB
:10EF40002020776173207365742E202020204D656A
:10EF50006E75202320332E312020202020202046B3
:10EF6000584F20414343455353204D4F4445465845
:10EF70004F20416363657373204D6F64653A446944
:10EF8000726563746C7920746F204658532044690D
:10EF9000726563746C7920746F2047534D2020276D
:10EFA000464F4C4C4F57204D4527202020202020F5
:10EFB000202020202020202020202020202020472A
:10EFC000534D2053656C656374696F6E20206279C0
:10EFD0002050726566697865733A205945536279A5
:10EFE0002050726566697865733A20204E4F202064
:10EFF0002020546F205465737420202020204E75EB
:10F000006D626572204C6973743A205945534E7590
:10F010006D626572204C6973743A20204E4F4D65C5
:10F020006E75202320332E32202020202020202007
:10F0300027464F4C4C4F57204D452720202020205D
:10F0400027466F6C6C6F77204D6527202020275254
:10F05000696E677327204E756D6265723A20466F40
:10F060006C6C6F77204D65274E756D6265724D65CE
:10F070006E75202320332E332020202020202020B6
:10F080004449414C494E47204D4F44452020204D96
:10F09000696E2E204469616C6C696E672020204483
:10F0A00069676974733A2020202020207878204DE9
:10F0B00061782E204469616C6C696E672020204461
:10F0C00069676974733A20202020202078782044D2
:10F0D00069616C6C696E67205061757365202020D2
:10F0E000782E78207365636F6E647320202020541F
:10F0F000696D652057616974696E67206F66646920
:10F10000616C6C696E6728736563293A7878205062
:10F1100053544E2F4578742E204C696E65204469F7
:10F12000616C696E6720203A20546F6E65204469D7
:10F13000616C696E6720203A2050756C73652020E1
:10F1400020436F756E747279202020202020204388
:10F150006F646520203A20202020202020204E614E
:10F1600074696F6E616C20446972656374204469D0
:10F17000616C696E672F4E44443A20202020506114
:10F18000757365206166746572206469616C204ED8
:10F19000444420283120736563202A293A204D6594
:10F1A0006E75202320332E34202020202020505321
:10F1B000544E2F4578742E4C20546F6E657320206A
:10F1C0004275737920546F6E653A202020204F4E8F
:10F1D0002F4F46463A20353030206D7365632052FC
:10F1E000656F7264657220546F6E653A20204F4ED1
:10F1F0002F4F46463A20323530206D7365634D659A
:10F200006E75202320332E352020202020202052F0
:10F21000494E4720504152414D455445525320528A
:10F22000696E67204672657175656E63792020206E
:10F230002020202020203A2078787820487A4D65B8
:10F240006E75202320342E312020202020202020E5
:10F250004761696E20436F6E74726F6C202053702B
:10F2600065616B6572202020203A202D78204D6941
:10F2700063726F70686F6E65203A202B78204D6541
:10F280006E75202320342E32202020202020566F1F
:10F2900069636520526174652054797065204F75EB
:10F2A0007420436F64696E6720203A202020496EE5
:10F2B00020436F64696E672020203A20202020546C
:10F2C00068697320566F69636520526174652020F8
:10F2D000206E6F7420737570706F72742E204D6580
:10F2E0006E75202320342E33202020202020202043
:10F2F0002047534D2042616E64202020202046721A
:10F30000657175656E63792042616E643A204D6F58
:10F310006E6F3A20202020383530204D487A4D6FCE
:10F320006E6F3A20202039303045204D487A4D6F9D
:10F330006E6F3A20202031383030204D487A4D6FA2
:10F340006E6F3A20202031393030204D487A447594
:10F35000616C3A3835302F313930304D487A447548
:10F36000616C3A3930302F313830304D487A44753D
:10F37000616C3A3930302F313930304D487A2020A5
:10F380002020202020202020202020202020205449
:10F390006869732047534D2042616E64202020200D
:10F3A0006E6F7420616C6C6F7765642E20204D65E4
:10F3B0006E75202320342E34202020202020534519
:10F3C0005454494E472050415353574F52442045BF
:10F3D0006E746572206E65772050535720204D65FE
:10F3E0006E75202320342E352020202020205345E8
:10F3F0005454494E472050494E20434F4445202005
:10F40000202053657474696E6720202020205049A5
:10F410004E20434F444520666F722053494D4D6541
:10F420006E75202320342E362020202020202020FE
:10F4300020205550444154494E47202020204D65FE
:10F440006E75202320342E372020202020204D6F61
:10F4500064756C6520494420284D4944292043683F
:10F46000616E67696E67204D49442020202020206E
:10F470002020776173206661696C656420212020FB
:10F4800043757272656E74204D49442020204552A8
:10F49000524F523A20202020202020202020526548
:10F4A0006164696E67206F66204D4944212043687E
:10F4B000616E67696E67206F66204D494420636FF7
:10F4C0006E6669726D3A2020202020202020456E33
:10F4D000746572206E6577204D49443A20204D496D
:10F4E000442073686F756C642068617665206F6670
:10F4F0002031342F3135206469676974732E2053AD
:10F50000657474696E67206F66204D4944204368B6
:10F51000616E67696E67206F66204D4944202077D1
:10F52000617320636F6D706C657465642021436F37
:10F530006E6669726D20746865206F6C64204D4939
:10F5400044205053573A20202020202020202045BE
:10F550006E74657220746865206E657720204D4951
:10F5600044205053573A20202020202020202020C3
:10F570004E6577204D4944205053572020202020AD
:10F580002077617320736574212020202020456E30
:10F590007465726564204D4944205053572020699A
:10F5A0007320494E56414C49442021212120456E6B
:10F5B0007465726564206E657720505357202077FC
:10F5C000617320756E636F72726563742E204D6572
:10F5D0006E75202320342E38202020202020524FEA
:10F5E0005554455220574F524B204D4F44452057BC
:10F5F0006F726B204D6F64653A2020202020202000
:10F60000566F696365204D6F64652020202020209F
:10F610002044617461204D6F6465202020202020EB
:10F6200020202020202020202020202020202020DA
:10F63000536176696E672020202020202020202022
:10F6400020504152414D4554455253202020202006
:10F6500047534D207C2054656C2E4C696E652020EC
:10F660006E6F742070726573656E7420202020495F
:10F670006E636F6D696E672043616C6C2020202083
:10F68000746F2046584F20506F72742E20204658B9
:10F690004F3A2020496E636F6D696E6720202020ED
:10F6A00020202020202020202020202020205269DF
:10F6B0006E673A4E6574776F726B2047534D2050DA
:10F6C00053544E2F465853206973206E6F74636FE6
:10F6D0006E6E656374656420746F2046584F2050C9
:10F6E00053544E2F46585320206973202020636FB7
:10F6F0006E6E656374656420746F2046584F466F64
:10F700006C6C6F77204D65274E756D626572206950
:10F7100073206E6F742070726573656E742120445F
:10F720006973636F6E6E656374696F6E2020206607
:10F73000726F6D2046585320506F72742020204401
:10F740006973636F6E6E656374696F6E20202066E7
:10F75000726F6D2046584F20506F727420202044E5
:10F760006973636F6E6E656374696F6E20202066C7
:10F77000726F6D2043454C4C554C415220204658E9
:10F780004F2043616C6C20746F2047534D204175AE
:10F79000746F6469616C20746F2046584F20204656
:10F7A000584F2F204578742E204C696E6520776164
:10F7B0007320646973636F6E6E656374656443611F
:10F7C0006C6C4261636B207669612046584F20471C
:10F7D000534D206E6F7420616E7377657220202008
:10F7E00047534D20496E636F6D696E67202020631B
:10F7F000616C6C207761732064656E696564436C2D
:10F800006261636B3A2047534D2E53494D78205324
:10F81000494D20697320626C6F636B65642E534998
:10F820004D2050494E20726571756972656453654B
:10F830007474696E672050494E2053494D78504981
:10F840004E2053494D3A2020202020202020457270
:10F85000726F723A3E203820646967697473204978
:10F860006E636F72726563742050494E2020534955
:10F870004D2050554B207265717569726564205238
:10F8800045504C4143452053494D20212121202002
:10F8900020526563656976656420202020204552EA
:10F8A000524F523A2020202020202020202053494F
:10F8B0004D312069732070726573656E742E456DCD
:10F8C00070747920736F636B657420312E205349F7
:10F8D0004D322069732070726573656E742E456DAC
:10F8E00070747920736F636B657420322E204C6FB7
:10F8F0006164696E67207468652053494D314C6FAF
:10F900006164696E67207468652053494D324658BA
:10F910004F206E6F7420666F756E642E20204465D4
:10F920006E6965642046584F2043616C6C204465C5
:10F930006E6965642047534D2043616C6C2E202016
:10F9400053494D206661696C7572652E20202052E6
:10F9500045504C4143452053494D20212121202031
:10F9600020204661696C75726520202020206F661A
:10F9700020737769746368696E672053494D20531B
:10F98000494D2072657175697265206F66206F74CC
:10F9900068657220706172616D65746572212050B6
:10F9A000756C7365206469616C6C696E673A206D73
:10F9B00075737420626520646967697473202049D7
:10F9C0006E6974696C697A6174696F6E2020202099
:10F9D0006F6620534D53204D4F44452020205265E3
:10F9E0006164696E6720534D53206661696C697369
:10F9F000206E6F7420636F6E6669726D656420633C
:10FA00006F6D6D616E64206572726F7220202020B0
:10FA10004C6973742069732066756C6C2020534D9B
:10FA200053206E6F74207072697661746520207740
:10FA30006173206E6F7420666F756E642020436C56
:10FA40006F7365642043616C6C6261636B204D650C
:10FA50006E75202320352E31202020202020434F7A
:10FA60004E54524F4C2076696120534D53204D65C2
:10FA70006E75202320352E32202020202020507229
:10FA800069766174652050617373776F7264536532
:10FA90007474696E6720666F722020534D53436FF4
:10FAA0006E6669726D3A20202020202020202020C0
:10FAB000456E74657265642050535720202020697C
:10FAC0007320494E56414C49442021212120436F47
:10FAD0006E6669726D206F6C64205053573A2045F2
:10FAE0006E746572206E657720505357203A4E65CC
:10FAF00077205052495641544520505357202020DA
:10FB000020776173207365742E2020202020436F9E
:10FB10006E74726F6C206279204C49535420766960
:10FB20006120534D53203A64697361626C65766954
:10FB30006120534D53203A656E61626C6520766991
:10FB40006120534D53203A202020202020202043A4
:10FB50006F6E6669726D2020616374696F6E76697D
:10FB60006120534D53203A64697361626C65766914
:10FB70006120534D53203A656E61626C65202050C0
:10FB8000726976617465206E756D62657220666F4C
:10FB90007220534D53203A64697361626C65666FDD
:10FBA0007220534D53203A656E61626C6520456E3C
:10FBB0007465726564206E657720505357202077F6
:10FBC000617320756E636F72726563742E202053AB
:10FBD0004D5320436F6E6669726D696E67202020F9
:10FBE000776173206661696C65642E202020205047
:10FBF000726976617465204E756D6265722020436E
:10FC00006F6E74726F6C20446967697473205365FA
:10FC100072766963652053657474696E672E5365E7
:10FC200072766963652053657474696E672E436FDD
:10FC30006E6669726D3A202020202020202020202E
:10FC4000456E7465726564205053572020202069EA
:10FC50007320494E56414C494420212121202053F4
:10FC6000657276696365204E756D626572202054F9
:10FC70004553542052494E472046584F2020506546
:10FC800072696F643A202020202020206D7320208C
:10FC9000534D5320434F4E54524F4C202020202090
:10FCA00020697320636C6F7365642E202020464D9D
:10FCB000453A204E4F5420414E5357455220464D11
:10FCC000453A204E4F542043415252494552464DE9
:10FCD000453A202042555359202020202020464DCF
:10FCE000453A4E6574776F726B206C6F7373524137
:10FCF0003A20204E4F5420414E53574552205241F6
:10FD00003A20204E4F5420434152524945525241CD
:10FD10003A202020425553592020202020205241B3
:10FD20003A204E6574776F726B206C6F7373525408
:10FD3000523A204E4F5420414E5357455220525470
:10FD4000523A204E4F542043415252494552525448
:10FD5000523A20204255535920202020202052542E
:10FD6000523A4E6574776F726B206C6F7373434CAD
:10FD7000423A204E4F5420414E5357455220434C57
:10FD8000423A204E4F542043415252494552434C2F
:10FD9000423A20204255535920202000434C423AF9
:10FDA0004E6574776F726B206C6F7373434F4E4662
:10FDB0004552454E43453A2043616C6C436F6E6635
:10FDC0006572656E6365206D6F64652020207761C4
:10FDD000732066696E69736865642E20434F4E46D2
:10FDE0004552454E43453A2057616974434F4E464C
:10FDF0004552454E43453A2042757379434F4E462E
:10FE00002E3A4E6F7420416E73776572434F4E46A3
:10FE10004552454E43453A2054616C6B20436F6E0A
:10FE2000666572656E6365204D6F646520202020D5
:10FE30004552524F522021212120202020202020D5
:10FE400047534D2043616C6C2020202020206E6F92
:10FE50007420616C6C6F7765642E20202050726571
:10FE600066697820776173206E6F742020666F75E5
:10FE70006E6420696E207461626C652E4552524F2B
:10FE8000523A20205365747570206F6673706565F3
:10FE900064203D31393230302062707352342E305C
:10FEA000202D44415441204D4F44452D20202020F9
:10FEB0003139323030206270732020204552524F49
:10FEC000523A2020274543484F2720202020205207
:10FED000455354415254494E472020202743616CDA
:10FEE0006C4261636B27206D6F64652020776173BE
:10FEF000206E6F7420736574212121202053494D99
:10FF0000206E6F7420737570706F74202743616C5E
:10FF10006C6261636B27204D6F6465204669726D6A
:10FF2000776172652056657273696F6E50726F6784
:10FF300072616D6D2056657273696F6E5254522DE9
:10FF4000342E39392D52342E302D422D4757343925
:0CFF50003952342E302D3035313130372D
:06FFFA0080FF8A3B630456
:020000040030CA
:0600010022001E83838033
:0600080000800F800F4094
:0200000400F00A
:10000000052FFFF1050FFFF2FFFFFFF1FFFFFFF1EB
:10001000FFFFFFF1FFFFFFF1FFFFFFF1FFFFFFF128
:10002000FFFFFFF1FFFFFFF1FFFFFFF1FFFFFFF118
:10003000FFFFFFF1FFFFFFF1FFFFFFF1FFFFFFF108
:10004000FFFFFFF2FFFFFFF2FFFFFFF2FFFFFFF2F4
:10005000FFFFFFF2FFFFFFF2FFFFFFF2FFFFFFF2E4
:10006000FFFFFFF2FFFFFFF2FFFFFFF2FFFFFFF2D4
:10007000FFFFFFF2FFFFFFF2FFFFFFF2FFFFFFF2C4
:10008000FFFFFFFFFFFFFFFF00FFFFFFFFFFFFFF7F
:10009000FFFF00FFFFFFFFFFFFFFFFFF00FFFFFF6E
:1000A000FFFFFFFFFFFF00FFFFFFFFFFFFFFFFFF5F
:1000B00000FFFFFFFFFFFFFFFFFF00FFFFFFFFFF4E
:1000C000FFFFFFFF00FFFFFFFFFFFFFFFFFF00FF3E
:1000D000FFFFFFFFFFFFFFFF00FFFFFFFFFFFFFF2F
:1000E000FFFF00FFFFFFFFFFFFFFFFFF00FFFFFF1E
:1000F000FFFFFFFFFFFF00FFFFFFFFFFFFFFFFFF0F
:1001000000FFFFFFFFFFFFFFFFFF00FFFFFFFFFFFD
:10011000FFFFFFFF00FFFFFFFFFFFFFFFFFF00FFED
:10012000FFFFFFFFFFFFFFFF00FFFFFFFFFFFFFFDE
:10013000FFFF00FFFFFFFFFFFFFFFFFF00FFFFFFCD
:10014000FFFFFFFFFFFF00FFFFFFFFFFFFFFFFFFBE
:1001500000FFFFFFFFFFFFFFFFFF00FFFFFFFFFFAD
:10016000FFFFFFFF00FFFFFFFFFFFFFFFFFF00FF9D
:10017000FFFFFFFFFFFFFFFF00FFFFFFFFFFFFFF8E
:10018000FFFF00FFFFFFFFFFFFFFFFFF00FFFFFF7D
:10019000FFFFFFFFFFFF00FFFFFFFFFFFFFFFFFF6E
:1001A00000FFFFFFFFFFFFFFFFFF00FFFFFFFFFF5D
:1001B000FFFFFFFF00FFFFFFFFFFFFFFFFFF00FF4D
:1001C000FFFFFFFFFFFFFFFF00FFFFFFFFFFFFFF3E
:1001D000FFFF00FFFFFFFFFFFFFFFFFF00FFFFFF2D
:1001E000FFFFFFFFFFFF00FFFFFFFFFFFFFFFFFF1E
:1001F00000FFFFFFFFFFFFFFFFFF00FFFFFFFFFF0D
:10020000FFFFFFFF00FFFFFFFFFFFFFFFFFF00FFFC
:10021000FFFFFFFFFFFFFFFF00FFFFFFFFFFFFFFED
:10022000FFFF00FFFFFFFFFFFFFFFFFF00FFFFFFDC
:10023000FFFFFFFFFFFF00FFFFFFFFFFFFFFFFFFCD
:1002400000FFFFFFFFFFFFFFFFFF00FFFFFFFFFFBC
:10025000FFFFFFFF00FFFFFFFFFFFFFFFFFF00FFAC
:10026000FFFFFFFFFFFFFFFF00FFFFFFFFFFFFFF9D
:10027000FFFF00FFFFFFFFFFFFFFFFFF00FFFFFF8C
:10028000FFFFFFFFFFFF00FFFFFFFFFFFFFFFFFF7D
:1002900000FFFFFFFFFFFFFFFFFF00FFFFFFFFFF6C
:1002A000FFFFFFFF00FFFFFFFFFFFFFFFFFF00FF5C
:1002B000FFFFFFFFFFFFFFFF00FFFFFFFFFFFFFF4D
:1002C000FFFF00FFFFFFFFFFFFFFFFFF00FFFFFF3C
:1002D000FFFFFFFFFFFF00FFFFFFFFFFFFFFFFFF2D
:1002E00000FFFFFFFFFFFFFFFFFF00FFFFFFFFFF1C
:1002F000FFFFFFFF00FFFFFFFFFFFFFFFFFF00FF0C
:1003000000320000030A323203000032000F32963E
:100310000000000501013000400C100E30202020AC
:10032000202000000000202020202020000020208D
:1003300020202020100E202020202020100E202001
:1003400020202020100E202020202020100E3030D1
:10035000303034323338363738333132333435365F
:1003600037383132333435363738202020202020BA
:10037000202020202020202020202020202020207D
:10038000202020202020202020202020202020206D
:10039000202020202020202020202020202020205D
:1003A000202020202020202020202020202020204D
:1003B000202020202020202020202020202020203D
:1003C00020202020202020202020000100010001EA
:0E03D000000132323232191919196496009662
:0403FC00FAFF000004
:00000001FF
